S01800006375705F646973635F625F626F6172642E737265639A
S3150802000000000A2009630208454E02084D4E0208FE
S31508020010554E02085D4E0208654E020859630208EB
S315080200200000000000000000000000006D4E0208FB
S315080200307B4E020800000000894E0208974E02080D
S315080200405963020859630208596302085963020888
S315080200505963020859630208596302085963020878
S315080200605963020859630208596302085963020868
S315080200705963020859630208596302085963020858
S315080200805963020859630208596302085963020848
S315080200905963020859630208596302085963020838
S315080200A05963020859630208596302085963020828
S315080200B05963020859630208596302085963020818
S315080200C05963020859630208596302085963020808
S315080200D0000000005963020859630208A54E020887
S315080200E059630208596302085963020859630208E8
S315080200F059630208B94E020859630208596302088D
S3150802010059630208CD4E0208596302085963020868
S3150802011059630208596302085963020859630208B7
S315080201205963020859630208E14E02085963020834
S315080201305963020859630208596302085963020897
S315080201405963020859630208596302085963020887
S315080201505963020859630208596302085963020877
S315080201605963020859630208596302085963020867
S315080201705963020859630208596302085963020857
S315080201805963020859630208596302085963020847
S315080201905963020859630208596302085963020837
S315080201A05963020859630208596302085963020827
S315080201B05963020859630208596302085963020817
S315080201C05963020859630208596302085963020807
S315080201D059630208596302085963020859630208F7
S315080201E059630208596302085963020859630208E7
S315080201F059630208596302085963020859630208D7
S31508020200596302085963020859630208000000008C
S315080202100000000059630208000000005963020842
S3150802022059630208596302085963020859630208A6
S315080202305963020859630208596302085963020896
S31508020240596302085963020859630208000000004C
S3150802025010B5054C237833B9044B13B10448AFF3F0
S3150802026000800123237010BD8407002000000000CF
S315080202707C88030808B5034B1BB103490348AFF34F
S31508020280008008BD00000000880700207C8803085B
S31508020290034613F8012B002AFBD1181A01387047B6
S315080202A081F0004102E000BF83F0004330B54FEA17
S315080202B041044FEA430594EA050F08BF90EA020F84
S315080202C01FBF54EA000C55EA020C7FEA645C7FEA17
S315080202D0655C00F0E2804FEA5454D4EB5555B8BF3A
S315080202E06D420CDD2C4480EA020281EA030382EAAB
S315080202F0000083EA010180EA020281EA0303362D3D
S3150802030088BF30BD11F0004F4FEA01314FF4801C0F
S315080203104CEA113102D0404261EB410113F0004F21
S315080203204FEA03334CEA133302D0524263EB4303D8
S3150802033094EA050F00F0A780A4F10104D5F1200E76
S315080203400DDB02FA0EFC22FA05F2801841F10001D1
S3150802035003FA0EF2801843FA05F359410EE0A5F1A5
S3150802036020050EF1200E012A03FA0EFC28BF4CF0D6
S31508020370020C43FA05F3C01851EBE37101F000458C
S3150802038007D54FF0000EDCF1000C7EEB00006EEB99
S315080203900101B1F5801F1BD3B1F5001F0CD3490823
S315080203A05FEA30004FEA3C0C04F101044FEA44527A
S315080203B012F5800F80F09A80BCF1004F08BF5FEA01
S315080203C0500C50F1000041EB045141EA050130BDE1
S315080203D05FEA4C0C404141EB0101013C28BFB1F5F3
S315080203E0801FE9D291F0000F04BF01460020B1FA3E
S315080203F081F308BF2033A3F10B03B3F120020CDA11
S315080204000C3208DD02F1140CC2F10C0201FA0CF0EE
S3150802041021FA02F10CE002F11402D8BFC2F1200C53
S3150802042001FA02F120FA0CFCDCBF41EA0C01904009
S31508020430E41AA2BF01EB0451294330BD6FEA040452
S315080204401F3C1CDA0C340EDC04F11404C4F120023D
S3150802045020FA04F001FA02F340EA030021FA04F34F
S3150802046045EA030130BDC4F10C04C4F1200220FAA6
S3150802047002F001FA04F340EA0300294630BD21FAE4
S3150802048004F0294630BD94F0000F83F4801306BFAA
S3150802049081F480110134013D4EE77FEA645C18BF9E
S315080204A07FEA655C29D094EA050F08BF90EA020F35
S315080204B005D054EA000C04BF1946104630BD91EA2D
S315080204C0030F1EBF0021002030BD5FEA545C05D130
S315080204D04000494128BF41F0004130BD14F580046F
S315080204E03CBF01F5801130BD01F0004545F0FE41E3
S315080204F041F470014FF0000030BD7FEA645C1ABF18
S31508020500194610467FEA655C1CBF0B46024650EA4E
S31508020510013406BF52EA033591EA030F41F400217A
S3150802052030BD00BF90F0000F04BF0021704730B500
S315080205304FF4806404F132044FF000054FF00001D5
S3150802054050E700BF90F0000F04BF0021704730B596
S315080205504FF4806404F1320410F0004548BF40426B
S315080205604FF000013EE700BF42004FEAE2014FEAC0
S3150802057031014FEA02701FBF12F07F4393F07F4F9B
S3150802058081F06051704732F07F4208BF704793F09E
S315080205907F4F04BF41F40021704730B54FF46074B1
S315080205A001F0004521F000411CE700BF50EA0102B4
S315080205B008BF704730B54FF000050AE050EA01025D
S315080205C008BF704730B511F0004502D5404261EBCD
S315080205D041014FF4806404F132045FEA915C3FF40E
S315080205E0D8AE4FF003025FEADC0C18BF03325FEAAB
S315080205F0DC0C18BF033202EBDC02C2F1200300FA5C
S3150802060003FC20FA02F001FA03FE40EA0E0021FA80
S3150802061002F11444BDE600BF70B54FF0FF0C4CF46E
S31508020620E06C1CEA11541DBF1CEA135594EA0C0F20
S3150802063095EA0C0F00F0DEF82C4481EA030621EA5B
S315080206404C5123EA4C5350EA013518BF52EA033596
S3150802065041F4801143F4801338D0A0FB02CE4FF048
S315080206600005E1FB02E506F00042E0FB03E54FF078
S315080206700006E1FB03569CF0000F18BF4EF0010E70
S31508020680A4F1FF04B6F5007F64F5407404D25FEA6C
S315080206904E0E6D4146EB060642EAC62141EA55511F
S315080206A04FEAC52040EA5E504FEACE2EB4F1FD0C61
S315080206B088BFBCF5E06F1ED8BEF1004F08BF5FEADF
S315080206C0500E50F1000041EB045170BD06F0004691
S315080206D046EA010140EA020081EA0301B4EB5C043E
S315080206E0C2BFD4EB0C0541EA045170BD41F4801136
S315080206F04FF0000E013C00F3AB8014F1360FDEBF5B
S31508020700002001F0004170BDC4F10004203C35DA36
S315080207100C341BDC04F11404C4F1200500FA05F3B9
S3150802072020FA04F001FA05F240EA020001F000425A
S3150802073021F0004110EBD37021FA04F642EB0601D0
S315080207405EEA430E08BF20EAD37070BDC4F10C04FA
S31508020750C4F1200500FA04F320FA05F001FA04F2BE
S3150802076040EA020001F0004110EBD37041F10001AA
S315080207705EEA430E08BF20EAD37070BDC4F12005B5
S3150802078000FA05F24EEA020E20FA04F301FA05F21D
S3150802079043EA020321FA04F001F0004121FA04F2C5
S315080207A020EA020000EBD3705EEA430E08BF20EA95
S315080207B0D37070BD94F0000F0FD101F000464000CF
S315080207C041EB010111F4801F08BF013CF7D041EA51
S315080207D0060195F0000F18BF704703F00046520055
S315080207E043EB030313F4801F08BF013DF7D043EA26
S315080207F00603704794EA0C0F0CEA135518BF95EADC
S315080208000C0F0CD050EA410618BF52EA4306D1D162
S3150802081081EA030101F000414FF0000070BD50EA81
S31508020820410606BF1046194652EA430619D094EA0B
S315080208300C0F02D150EA013613D195EA0C0F05D1F5
S3150802084052EA03361CBF104619460AD181EA030149
S3150802085001F0004141F0FE4141F470014FF0000001
S3150802086070BD41F0FE4141F4780170BD70B54FF09C
S31508020870FF0C4CF4E06C1CEA11541DBF1CEA13551C
S3150802088094EA0C0F95EA0C0F00F0A7F8A4EB0504FE
S3150802089081EA030E52EA03354FEA013100F08880F5
S315080208A04FEA03334FF0805545EA131343EA1263BE
S315080208B04FEA022245EA111545EA10654FEA002673
S315080208C00EF000419D4208BF964244F1FD0404F52C
S315080208D0407402D25B084FEA3202B61A65EB030588
S315080208E05B084FEA32024FF480104FF4002CB6EB45
S315080208F0020E75EB030E22BFB61A754640EA0C00C5
S315080209005B084FEA3202B6EB020E75EB030E22BF04
S31508020910B61A754640EA5C005B084FEA3202B6EB45
S31508020920020E75EB030E22BFB61A754640EA9C0004
S315080209305B084FEA3202B6EB020E75EB030E22BFD4
S31508020940B61A754640EADC0055EA060E18D04FEA92
S31508020950051545EA16754FEA06164FEAC30343EA32
S3150802096052734FEAC2025FEA1C1CC0D111F4801FFF
S315080209700BD141EA00014FF000004FF0004CB6E7F8
S3150802098011F4801F04BF01430020B4F1FD0C88BF97
S31508020990BCF5E06F3FF6AFAEB5EB030C04BFB6EBA2
S315080209A0020C5FEA500C50F1000041EB045170BD95
S315080209B00EF0004E4EEA113114EB5C04C2BFD4EBC2
S315080209C00C0541EA045170BD41F480114FF0000E46
S315080209D0013C90E645EA060E8DE60CEA135594EAC2
S315080209E00C0F08BF95EA0C0F3FF43BAF94EA0C0FC5
S315080209F00AD150EA01347FF434AF95EA0C0F7FF43A
S31508020A0025AF104619462CE795EA0C0F06D152EA8D
S31508020A1003353FF4FDAE1046194622E750EA410671
S31508020A2018BF52EA43067FF4C5AE50EA41047FF482
S31508020A300DAF52EA43057FF4EBAE12E74FF0FF3CE7
S31508020A4006E000BF4FF0010C02E000BF4FF0010CB8
S31508020A504DF804CD4FEA410C7FEA6C5C4FEA430C31
S31508020A6018BF7FEA6C5C1BD001B050EA410C0CBF80
S31508020A7052EA430C91EA030F02BF90EA020F0020E2
S31508020A80704710F1000F91EA030F58BF994208BF49
S31508020A9090422CBFD8176FEAE37040F00100704706
S31508020AA04FEA410C7FEA6C5C02D150EA013C07D15D
S31508020AB04FEA430C7FEA6C5CD6D152EA033CD3D0A8
S31508020AC05DF8040B704700BF8446104662468C46A2
S31508020AD01946634600E000BF01B5FFF7B7FF0028D5
S31508020AE048BF10F1000F01BD4DF808EDFFF7F4FFFE
S31508020AF00CBF012000205DF808FB00BF4DF808ED89
S31508020B00FFF7EAFF34BF012000205DF808FB00BFAB
S31508020B104DF808EDFFF7E0FF94BF012000205DF8CD
S31508020B2008FB00BF4DF808EDFFF7CEFF94BF012082
S31508020B3000205DF808FB00BF4DF808EDFFF7C4FF7B
S31508020B4034BF012000205DF808FB00BF4FEA410CC4
S31508020B507FEA6C5C02D150EA013C0AD14FEA430CA7
S31508020B607FEA6C5C02D152EA033C02D14FF00000E4
S31508020B7070474FF0010070474FEA410212F5001222
S31508020B8015D211D56FF47873B3EB625212D94FEAC4
S31508020B90C12343F0004343EA505311F0004F23FAAE
S31508020BA002F018BF404270474FF00000704750EA03
S31508020BB0013005D111F0004008BF6FF000407047C0
S31508020BC04FF00000704700BF4A0011D212F500121A
S31508020BD011D20DD56FF47873B3EB62520ED44FEA85
S31508020BE0C12343F0004343EA505323FA02F0704705
S31508020BF04FF00000704750EA013002D14FF0FF3043
S31508020C0070474FF0000070474FEA4102B2F1E043E5
S31508020C1024BFB3F5001CDCF1FE5C0DD901F0004CD3
S31508020C204FEAC0024CEA5070B2F1004F40EB830023
S31508020C3008BF20F00100704711F0804F21D113F14F
S31508020C403872BCBF01F00040704741F480114FEA88
S31508020C505252C2F11802C2F1200C10FA0CF320FA11
S31508020C6002F018BF40F001004FEAC1234FEAD3232E
S31508020C7003FA0CFC40EA0C0023FA02F34FEA430398
S31508020C80CCE77FEA625307D150EA01331EBF4FF021
S31508020C90FE4040F44000704701F0004040F0FE403C
S31508020CA040F40000704700BF53B94AB9002908BF8B
S31508020CB000281CBF4FF0FF314FF0FF3000F0B4B9E7
S31508020CC0ADF1080C6DE904CE00F03CF8DDF804E05D
S31508020CD0DDE9022304B0704738B500220023044632
S31508020CE00D46FFF70BFF28B920462946BDE83840CE
S31508020CF000F00AB8204605F1004100F005F8404226
S31508020D0061EB410138BD00BFD0B500220B4B064648
S31508020D100F46FFF781FCFFF757FF0446FFF702FC71
S31508020D200022074BFFF778FC02460B463046394647
S31508020D30FFF7BAFAFFF748FF2146D0BD0000F03D9B
S31508020D400000F0412DE9F04F099D0C46002B4DD1CC
S31508020D508A420F4684469646B2FA82F360D94BB166
S31508020D6002FA03FEC3F120029F4000FA03FC20FAAE
S31508020D7002F217434FEA1E461FFA8EF44FEA1C4246
S31508020D80B7FBF6F106FB117701FB04F042EA0742CC
S31508020D90904208D91EEB020201F1FF3702D29042B5
S31508020DA000F22D813946121A1FFA8CFCB2FBF6F0B4
S31508020DB006FB102200FB04F44CEA024C644508D9EF
S31508020DC01EEB0C0C00F1FF3202D2644500F21A81C6
S31508020DD0104640EA0140ACEB040C002125B12CFA7E
S31508020DE003F30022C5E90032BDE8F08F8B4205D92C
S31508020DF00DB1C5E9000100210846F5E7B3FA83F10A
S31508020E0000294DD1A342C0F0F280904280F0EF80D3
S31508020E10064623460846002DE6D0C5E90063E3E701
S31508020E20002B40F0A2808A1A4FEA1E471FFA8EF656
S31508020E300121B2FBF7F407FB14204FEA1C4242EAEF
S31508020E40004206FB04F090420FD91EEB020204F19F
S31508020E50FF382CBF4FF001094FF00009904203D921
S31508020E60B9F1000F00F0C8804446121A1FFA8CFC2A
S31508020E70B2FBF7F007FB102200FB06F64CEA024C1F
S31508020E80664508D91EEB0C0C00F1FF3202D2664504
S31508020E9000F2BB801046ACEB060C40EA04409DE724
S31508020EA0C1F120068B4004FA01FE22FA06F720FA5F
S31508020EB006FCF4408A401F434EEA0C0300FA01FE80
S31508020EC04FEA17484FEA13491FFA87FCB4FBF8F0B2
S31508020ED008FB104449EA044400FB0CF9A1450ED963
S31508020EE03C1900F1FF3A2CBF4FF0010B4FF0000BF3
S31508020EF0A14503D9BBF1000F00F093805046A4EB3D
S31508020F0009041FFA83F9B4FBF8F308FB134403FB3D
S31508020F100CFC49EA0444A44506D93C1903F1FF38F6
S31508020F2001D2A4457AD8434643EA0040A4EB0C040E
S31508020F30A0FB02984445CC46434602D306D1CE4589
S31508020F4004D20138B9EB020C68EB07035DB1BEEBBC
S31508020F500C0264EB030404FA06F622FA01F3CC4007
S31508020F601E43C5E9006400213EE702FA03FEC3F107
S31508020F70200104FA03F200FA03FCCC404FEA1E47AA
S31508020F8020FA01F11FFA8EF6B4FBF7F00A4307FBC3
S31508020F901044110C41EA044100FB06F48C420ED9B6
S31508020FA01EEB010100F1FF382CBF4FF001094FF08B
S31508020FB000098C4202D9B9F1000F2CD04046091B10
S31508020FC092B2B1FBF7F407FB141142EA014204FBA1
S31508020FD006F1914207D91EEB020204F1FF3801D24B
S31508020FE0914215D84446521A44EA004121E7861A24
S31508020FF064EB030301200EE7023C724435E702392B
S315080210007244D0E6F4440238E3E6F444023842E78E
S31508021010023C7244E7E702387144D0E7023B3C449B
S3150802102082E702383C446AE7704700BF80B582B05F
S3150802103000AF03F0EFFF0346184604F03AF878606B
S3150802104024220021786814F057F9054805F0E8F8D3
S315080210507B68044A1A6000BF0837BD4680BD00BFD8
S31508021060A08803080245434980B588B000AFF860F6
S31508021070B9601346FB710023FB6100233B61BB6821
S315080210807B617B69BB610023FB6110E0FA69FB683F
S315080210901344184611F0E6FD03463B613A69BB69FB
S315080210A01A60BB690433BB61FB690433FB61FB79D4
S315080210B0FA699A42EADB012318462037BD4680BD03
S315080210C080B58CB000AF002387F82F3003F0A2FF5B
S315080210D00346184603F0EDFFB86224220021B86AD7
S315080210E014F00AF93B1D24220021184614F004F9CB
S315080210F03B1D242219460F48FFF7B6FF7B680E4AA6
S31508021100934205D0FFF792FF002387F82F300BE0B2
S315080211103B1D24221946B86A14F0A5F9074805F0BA
S315080211207FF8012387F82F3097F82F301846303783
S31508021130BD4680BD00C01F0802454349B88803085A
S3150802114090B589B000AF0023FB6103F063FF034645
S31508021150184603F0AEFF78617B69BB61FE2011F089
S31508021160B0FD0023FB611CE03B1D1022002118463E
S3150802117014F0C2F8BB693C1D186859689A68DB689E
S315080211800FC4FB6903F1016303F57C233A1D11467B
S31508021190184611F07BFDBB691033BB61FB6910333E
S315080211A0FB61FB69232BDFD9012318462437BD4689
S315080211B090BD000080B483B000AF0346FB71FB7993
S315080211C0002B02D1194B1B682AE0FB79012B02D1AD
S315080211D0174B1B6824E0FB79022B02D1154B1B68BF
S315080211E01EE0FB79032B02D1134B1B6818E0FB792F
S315080211F0042B02D1114B1B6812E0FB79052B02D195
S315080212000F4B1B680CE0FB79062B02D10D4B1B68B2
S3150802121006E0FB79072B02D10B4B1B6800E0002383
S3150802122018460C37BD465DF8047B7047A0070020B8
S31508021230A4070020A8070020AC070020B00700205A
S31508021240B4070020B8070020BC07002080B483B08A
S3150802125000AF03463960FB71FB79002B03D11D4AA7
S315080212603B6813602FE0FB79012B03D11A4A3B68CE
S31508021270136028E0FB79022B03D1184A3B681360F6
S3150802128021E0FB79032B03D1154A3B6813601AE068
S31508021290FB79042B03D1134A3B68136013E0FB79ED
S315080212A0052B03D1104A3B6813600CE0FB79062B29
S315080212B003D10E4A3B68136005E0FB79072B02D17E
S315080212C00B4A3B68136000BF0C37BD465DF8047BCA
S315080212D0704700BFA0070020A4070020A807002027
S315080212E0AC070020B0070020B4070020B80700208A
S315080212F0BC07002080B586B000AFF8600B467A605E
S31508021300FB720023FB752D4804F08AFF0023FB7548
S315080213104CE0FB7D2A4A4FF48E7101FB03F313441A
S315080213201B78012B3FD1FB7D4FF48E7202FB03F330
S31508021330234A134402331946224804F071FF22480D
S3150802134004F06EFFFB7D4FF48E7202FB03F3183333
S315080213501B4A1344043319461A4804F061FF1B4812
S3150802136004F05EFFFB7D164A4FF48E7101FB03F310
S3150802137013449C331B782D2B12D0154804F050FFCA
S31508021380FB7D4FF48E7202FB03F398330C4A134427
S31508021390043319460B4804F043FF0C4804F040FF97
S315080213A00A4804F03DFFFB7D0133FB75FB7D042BE8
S315080213B0AFD900BF00BF1837BD4680BDC88803082D
S315080213C000000020F0880308F4880308F888030858
S315080213D0FC88030880B586B000AFF8600B467A60D1
S315080213E0FB7200237B617B6803F5007303221649AF
S315080213F0184613F089FF0346002B21D17B6803F5B3
S3150802140000731846FEF744FF0346032B18D17B6880
S3150802141003F58063184612F06DFE78617B69002B2E
S3150802142007D003F0F7FD03460121184604F064F8D5
S3150802143006E003F0EFFD03460121184604F079F8A9
S3150802144000BF1837BD4680BD0889030880B584B039
S3150802145000AFF8600B467A60FB727B6803F500738F
S315080214600422A949184613F04FFF0346002B08D158
S315080214707B6803F500731846FEF70AFF0346042B3A
S3150802148013D07B6803F500731A78A04B1B78D31A1E
S31508021490002B40F0D7807B6803F500731846FEF7E9
S315080214A0F7FE0346012B40F0CD807B6803F5806387
S315080214B01A78974B1B78D31A002B0FD17B6803F542
S315080214C080631846FEF7E4FE0346012B06D19148CF
S315080214D004F0A6FE002000F0BFFEB2E07B6803F52A
S315080214E080631A788C4B1B78D31A002B0FD17B6832
S315080214F003F580631846FEF7CBFE0346012B06D199
S31508021500864804F08DFE012000F0A6FE99E07B686D
S3150802151003F580631A78824B1B78D31A002B0FD1F6
S315080215207B6803F580631846FEF7B2FE0346012B75
S3150802153006D17C4804F074FE022000F08DFE80E09D
S315080215407B6803F580631A78774B1B78D31A002BCE
S315080215500FD17B6803F580631846FEF799FE0346AA
S31508021560012B06D1714804F05BFE032000F074FEDD
S3150802157067E07B6803F580631A786D4B1B78D31A8C
S31508021580002B0FD17B6803F580631846FEF780FEB1
S315080215900346012B06D1674804F042FE042000F0F8
S315080215A05BFE4EE07B6803F580631A78624B1B7814
S315080215B0D31A002B0FD17B6803F580631846FEF712
S315080215C067FE0346012B06D15C4804F029FE052076
S315080215D000F042FE35E07B6803F580631A78584BC3
S315080215E01B78D31A002B0FD17B6803F58063184644
S315080215F0FEF74EFE0346012B06D1524804F010FEB2
S31508021600062000F029FE1CE07B6803F580631A7841
S315080216104D4B1B78D31A002B0FD17B6803F58063D9
S315080216201846FEF735FE0346012B06D1474804F055
S31508021630F7FD072000F010FE03E0454804F0F0FD30
S3150802164030E32FE37B6803F500730322414918460A
S3150802165013F05AFE0346002B40F006817B6803F519
S3150802166000731846FEF714FE0346032B40F0FC806F
S315080216707B6803F580631A78254B1B78D31A002BEF
S315080216800FD17B6803F580631846FEF701FE034611
S31508021690012B06D1304804F0C3FD002000F074FF88
S315080216A0E1E07B6803F580631A781B4B1B78D31A33
S315080216B0002B0FD17B6803F580631846FEF7E8FD19
S315080216C00346012B06D1254804F0AAFD012000F0A5
S315080216D05BFFC8E07B6803F580631A78104B1B78BA
S315080216E0D31A002B3ED17B6803F580631846FEF7B2
S315080216F0CFFD0346012B35D1194804F091FD02208E
S3150802170000F042FFAFE000BF0C8903081489030802
S31508021710188903081C8903084089030844890308B1
S31508021720688903086C890308908903089489030861
S31508021730B8890308BC890308E0890308E489030811
S31508021740088A03080C8A0308308A0308348A0308BD
S31508021750588A03086C8A0308708A03088C8A030865
S31508021760AC8A03087B6803F580631A78AF4B1B784B
S31508021770D31A002B0FD17B6803F580631846FEF750
S3150802178087FD0346012B06D1A94804F049FD03202B
S3150802179000F0FAFE67E07B6803F580631A78A54BCA
S315080217A01B78D31A002B0FD17B6803F58063184682
S315080217B0FEF76EFD0346012B06D19F4804F030FD65
S315080217C0042000F0E1FE4EE07B6803F580631A7898
S315080217D09A4B1B78D31A002B0FD17B6803F58063CB
S315080217E01846FEF755FD0346012B06D1944804F028
S315080217F017FD052000F0C8FE35E07B6803F5806317
S315080218001A78904B1B78D31A002B0FD17B6803F5F5
S3150802181080631846FEF73CFD0346012B06D18A482B
S3150802182004F0FEFC062000F0AFFE1CE07B6803F520
S3150802183080631A78854B1B78D31A002B0FD17B68E5
S3150802184003F580631846FEF723FD0346012B06D1EE
S315080218507F4804F0E5FC072000F096FE03E07D4889
S3150802186004F0DEFC1EE21DE27B6803F50073042227
S315080218707949184613F048FD0346002B11D17B68B7
S3150802188003F500731846FEF703FD0346042B08D139
S31508021890724804F0C5FCFFF753FC714804F0C0FC1B
S315080218A000E27B6803F5007305226E49184613F0B9
S315080218B02BFD0346002B40F05F817B6803F500731E
S315080218C01846FEF7E5FC0346052B40F055817B6872
S315080218D003F580631A78644B1B78D31A002B19D147
S315080218E07B6803F580631846FEF7D2FC0346012B94
S315080218F010D15E4804F094FC002000F00DFD10EEB5
S31508021900103A1846FEF730FE02460B46584804F0CF
S3150802191087FC30E17B6803F580631A78554B1B78A0
S31508021920D31A002B19D17B6803F580631846FEF794
S31508021930AFFC0346012B10D14F4804F071FC01207D
S3150802194000F0EAFC10EE103A1846FEF70DFE0246C3
S315080219500B464A4804F064FC0DE17B6803F5806394
S315080219601A78474B1B78D31A002B19D17B6803F5D3
S3150802197080631846FEF78CFC0346012B10D14148BA
S3150802198004F04EFC022000F0C7FC10EE103A18468E
S31508021990FEF7EAFD02460B463B4804F041FCEAE044
S315080219A07B6803F580631A78204B1B78D31A002BC1
S315080219B019D17B6803F580631846FEF769FC03466E
S315080219C0012B10D1314804F02BFC032000F0A4FCB3
S315080219D010EE103A1846FEF7C7FD02460B462C488B
S315080219E004F01EFCC7E07B6803F580631A78114B86
S315080219F01B78D31A002B51D17B6803F580631846EE
S31508021A00FEF746FC0346012B48D1224804F008FC9F
S31508021A10042000F081FC10EE103A1846FEF7A4FDE9
S31508021A2002460B461C4804F0FBFBA4E09089030817
S31508021A30CC8A0308B8890308708A0308E089030870
S31508021A40EC8A0308088A03080C8B0308308A030801
S31508021A502C8B0308588A03084C8B0308548B0308FB
S31508021A60708B0308908B030818890308988B030860
S31508021A70B88B030840890308D48B0308F48B030840
S31508021A8068890308108C0308308C03084C8C0308F9
S31508021A906C8C0308888C0308A88C03087B6803F5FA
S31508021AA080631A78814B1B78D31A002B19D17B686D
S31508021AB003F580631846FEF7EBFB0346012B10D1AC
S31508021AC07B4804F0ADFB052000F026FC10EE103A28
S31508021AD01846FEF749FD02460B46764804F0A0FB77
S31508021AE049E07B6803F580631A78734B1B78D31A2F
S31508021AF0002B19D17B6803F580631846FEF7C8FBED
S31508021B000346012B10D16D4804F08AFB062000F02B
S31508021B1003FC10EE103A1846FEF726FD02460B465F
S31508021B20674804F07DFB26E07B6803F580631A7834
S31508021B30644B1B78D31A002B19D17B6803F5806393
S31508021B401846FEF7A5FB0346012B10D15E4804F0A2
S31508021B5067FB072000F0E0FB10EE103A1846FEF786
S31508021B6003FD02460B46594804F05AFB03E058485F
S31508021B7004F056FB96E095E07B6803F500730722AE
S31508021B805449184613F0C0FB0346002B40F08680E2
S31508021B907B6803F500731846FEF77AFB0346072BA4
S31508021BA07CD17B6803F580631A784B4B1B78D31A72
S31508021BB0002B14D17B6803F580631846FEF768FB91
S31508021BC00346012B0BD1454804F02AFB002000F0FE
S31508021BD067FA03461946424804F022FB5DE07B6831
S31508021BE003F580631A783F4B1B78D31A002B14D15E
S31508021BF07B6803F580631846FEF74AFB0346012B0A
S31508021C000BD1394804F00CFB012000F049FA0346CF
S31508021C101946364804F004FB3FE07B6803F5806307
S31508021C201A78334B1B78D31A002B14D17B6803F529
S31508021C3080631846FEF72CFB0346012B0BD12D4871
S31508021C4004F0EEFA022000F02BFA034619462A4857
S31508021C5004F0E6FA21E07B6803F580631A78274BDD
S31508021C601B78D31A002B14D17B6803F580631846B8
S31508021C70FEF70EFB0346012B0BD1214804F0D0FADE
S31508021C80032000F00DFA034619461E4804F0C8FA66
S31508021C9003E00F4804F0C4FA04E003E00C4804F039
S31508021CA0BFFA00BF1037BD4680BD00BFE0890308F2
S31508021CB0C48C0308E48C0308088A0308008D030809
S31508021CC0208D0308308A03083C8D03085C8D0308BF
S31508021CD0588A0308788D030818890308808D030833
S31508021CE0A08D030840890308B88D0308D88D030818
S31508021CF068890308F08D0308108E03089089030883
S31508021D00288E0308488E030880B584B000AFF860B1
S31508021D100B467A60FB7203F07DF90346184603F018
S31508021D209FF900BF1037BD4680BD000090B585B04B
S31508021D3000AF78600023BB730023FB734FF4A052F5
S31508021D400021204813F0D8FA07F10E030A221D498A
S31508021D5078680FF0FBFB0346012B2ED10023FB7399
S31508021D6028E0FB7B4FF48E7202FB03F3164A1344F8
S31508021D709C1C1448FEF78CFA03461A46114920465B
S31508021D8013F0C2FA0346002B11D1FB7B0E4A4FF41D
S31508021D908E7101FB03F3134418331B68B97B094A96
S31508021DA000209847094804F03BFA012306E0FB7B2A
S31508021DB00133FB73FB7B042BD3D900231846143754
S31508021DC0BD4690BDC007002000000020F888030821
S31508021DD080B582B000AF0346FB71FB790D2B24D187
S31508021DE04F4B00221A704F4804F01AFA4E4B1B78D2
S31508021DF0002B16D04D48FFF799FF0346012B08D151
S31508021E00F02200214A4813F077FA4849484813F065
S31508021E1014FB454B00221A70F0220021434813F0A6
S31508021E206BFA444804F0FCF976E0FB790A2B03D1F5
S31508021E303B4B00221A706FE0FB791B2B03D1384B00
S31508021E4001221A7068E0FB795B2B07D1344B1B78A9
S31508021E50012B03D1324B02221A705DE0FB79412B2A
S31508021E601FD12F4B1B78022B1BD12D4B00221A7028
S31508021E702D4B1B78002B4FD12D492F4804F0D0F952
S31508021E802B48FEF705FA0346DAB2274B1A70F022F8
S31508021E900021264813F030FA2549244813F0CDFAD2
S31508021EA03AE0FB79082B02D0FB797F2B16D11C4B23
S31508021EB000221A701C4B1B78002B2DD01A4B1B784C
S31508021EC0013BDAB2184B1A70174B1B781A46174B96
S31508021ED000219954194804F0A3F91DE0124B1B7806
S31508021EE05A1CD1B2104A11701946104AFB7953543A
S31508021EF00D4B1A78124BA3FB0213D9090B461B0189
S31508021F005B1A1B01D31ADAB2074B1A70FB79194608
S31508021F100C4804F085F9FFE700BF0837BD4680BDC7
S31508021F20A11D0020F8880308A01D0020B01C00206F
S31508021F30C01B0020608E0308F0880308648E03081D
S31508021F4089888888688E030880B58AB004AF00231A
S31508021F507B6100233B610023FB600023BB600023F7
S31508021F607B6003F057F80346184603F0A2F80346C7
S31508021F70184603F0B9F8786103F04CF80346184698
S31508021F8003F097F80346184603F0C9F8386103F0D8
S31508021F9041F80346184603F08CF80346184603F040
S31508021FA0D9F8F86003F036F80346184603F081F8C4
S31508021FB00346184603F0E9F8B86003F02BF803461F
S31508021FC0184603F076F80346184603F0F9F87860DF
S31508021FD00020FFF7EFF802467B690293019220235D
S31508021FE00093254B1022244924480FF021F8022099
S31508021FF0FFF7E0F802463B69029301924FF4007339
S3150802200000931F4B4FF480721D491E480FF010F8BB
S315080220100420FFF7CFF80246FB68029301924FF4B9
S3150802202000630093184B4FF48062174917480EF065
S31508022030FFFF0520FFF7BEF80246BB68029301922E
S3150802204040230093124B2022114912480EF0F0FF4A
S315080220500620FFF7AFF802467B6802930192022335
S3150802206000930D4B01220C490C480EF0E1FF00BF0C
S315080220701837BD4680BD00BF00080242A41D0020D5
S31508022080000C0242C01D002000180242DC1D00207E
S3150802209000040242F81D002000140242141E002009
S315080220A080B582B000AF0346FB71FB79002B04D1E1
S315080220B017480EF0F1FF034626E0FB79012B22D0E2
S315080220C0FB79022B04D113480EF0E6FF03461BE008
S315080220D0FB79032B17D0FB79042B04D10E480EF09B
S315080220E0DBFF034610E0FB79052B04D10B480EF003
S315080220F0D3FF034608E0FB79062B04D108480EF005
S31508022100CBFF034600E0002318460837BD4680BDCC
S31508022110A41D0020C01D0020DC1D0020F81D002083
S31508022120141E002080B582B000AF03460A46FB7132
S315080221301346BB71FB79002B06D1BB7919461C489D
S315080221400EF0FCFF03462EE0FB79012B2AD0FB7921
S31508022150022B06D1BB79194616480EF0EFFF034645
S3150802216021E0FB79032B1DD0FB79042B06D1BB7921
S31508022170194611480EF0E2FF034614E0FB79052BD7
S3150802218006D1BB7919460D480EF0D8FF03460AE078
S31508022190FB79062B06D1BB79194609480EF0CEFF04
S315080221A0034600E0002318460837BD4680BD00BF37
S315080221B0A41D0020C01D0020DC1D0020F81D0020E3
S315080221C0141E002080B582B000AF0346FB71FB796E
S315080221D0002B08D10020FEF7EDFF034619461A48E0
S315080221E00EF0CFFF2BE0FB79012B28D0FB79022BCF
S315080221F008D10220FEF7DEFF0346194613480EF001
S31508022200C0FF1CE0FB79032B19D0FB79042B08D1FC
S315080222100420FEF7CFFF034619460D480EF0B1FF1C
S315080222200DE0FB79052B0AD0FB79062B07D1062090
S31508022230FEF7C0FF0346194606480EF0A2FF00BF86
S315080222400837BD4680BD00BFA41D0020C01D002062
S31508022250DC1D0020141E002080B584B000AF0346A2
S31508022260FB710023FB60FB79002B0CD105210020B2
S31508022270FFF758FFF860F9680020FEF7E7FF00202D
S31508022280FFF7A0FF44E0FB79012B41D0FB79022B33
S315080222900CD105210220FFF745FFF860F9680220F4
S315080222A0FEF7D4FF0220FFF78DFF31E0FB79032BFF
S315080222B02ED0FB79042B0CD105210420FFF732FF1F
S315080222C0F860F9680420FEF7C1FF0420FFF77AFFD9
S315080222D01EE0FB79052B0CD105210520FFF722FF0D
S315080222E0F860F9680520FEF7B1FF0520FFF76AFFD7
S315080222F00EE0FB79062B0BD105210620FFF712FF0C
S31508022300F860F9680620FEF7A1FF0620FFF75AFFD4
S3150802231000BF1037BD4680BD80B586B000AF034604
S31508022320FB714FF000037B614FF000033B614FF0F6
S315080223300003FB604FF00003BB60FB79002B2ED134
S315080223400020FFF7ADFE07EE900AF8EEE77AC7ED32
S31508022350047A0020FEF72EFF07EE900AF8EEE77AD7
S31508022360C7ED037A02F056FE0346184602F0A1FEAE
S315080223700346184602F0B8FE07EE900AF8EEE77A28
S31508022380C7ED027A02F046FE0346D7ED047AFCEE62
S31508022390E77A17EE901A184602F0E6FFCEE0FB79C6
S315080223A0012B00F0CB80FB79022B2ED10220FFF7FE
S315080223B077FE07EE900AF8EEE77AC7ED047A02206E
S315080223C0FEF7F8FE07EE900AF8EEE77AC7ED037A0B
S315080223D002F020FE0346184602F06BFE0346184634
S315080223E002F09DFE07EE900AF8EEE77AC7ED027A4A
S315080223F002F010FE0346D7ED047AFCEEE77A17EEF2
S31508022400901A184602F0D7FF98E0FB79032B00F0E2
S315080224109580FB79042B2ED10420FFF741FE07EEA7
S31508022420900AF8EEE77AC7ED047A0420FEF7C2FEB0
S3150802243007EE900AF8EEE77AC7ED037A02F0EAFDAC
S315080224400346184602F035FE0346184602F082FE97
S3150802245007EE900AF8EEE77AC7ED027A02F0DAFD9D
S315080224600346D7ED047AFCEEE77A17EE901A184679
S3150802247002F0C8FF62E0FB79052B2ED10520FFF793
S315080224800FFE07EE900AF8EEE77AC7ED047A052002
S31508022490FEF790FE07EE900AF8EEE77AC7ED037AA2
S315080224A002F0B8FD0346184602F003FE0346184634
S315080224B002F06BFE07EE900AF8EEE77AC7ED027AAB
S315080224C002F0A8FD0346D7ED047AFCEEE77A17EE8A
S315080224D0901A184602F0B1FF30E0FB79062B2DD18F
S315080224E00620FFF7DDFD07EE900AF8EEE77AC7ED5C
S315080224F0047A0620FEF75EFE07EE900AF8EEE77A01
S31508022500C7ED037A02F086FD0346184602F0D1FDAE
S315080225100346184602F054FE07EE900AF8EEE77AEA
S31508022520C7ED027A02F076FD0346D7ED047AFCEE91
S31508022530E77A17EE901A184602F09AFFD7ED027A52
S31508022540F5EE407AF1EE10FA10D097ED047AD7ED4F
S31508022550037A77EE676A97ED027AC6EE877A9FED77
S31508022560097A67EE877AC7ED057A02E04FF000032B
S315080225707B617B6907EE903AB0EE670A1837BD466B
S3150802258080BD00BF0000484390B585B000AF034642
S31508022590FB710023FB60FB79002B25D11E2100204D
S315080225A0FFF7C0FD04460020FEF704FE0346E31AC1
S315080225B0FB6002F02FFD0346184602F07AFD034639
S315080225C0F968184602F081FD02F024FD034601214E
S315080225D0184602F074FF0346002B00F0AB80F96838
S315080225E0564803F01DFEA5E0FB79012B00F0A280F8
S315080225F0FB79022B24D11E210220FFF793FD044604
S315080226000220FEF7D7FD0346E31AFB6002F002FD3D
S315080226100346184602F04DFD0346F968184602F0CD
S315080226206FFD02F0F7FC03460121184602F047FF48
S315080226300346002B7ED0F968404803F0F1FD79E0A5
S31508022640FB79032B76D0FB79042B24D11E21042097
S31508022650FFF768FD04460420FEF7ACFD0346E31ABD
S31508022660FB6002F0D7FC0346184602F022FD034639
S31508022670F968184602F05FFD02F0CCFC0346012118
S31508022680184602F01CFF0346002B53D0F9682B4864
S3150802269003F0C6FD4EE0FB79052B24D11E21052049
S315080226A0FFF740FD04460520FEF784FD0346E31ABC
S315080226B0FB6002F0AFFC0346184602F0FAFC03463A
S315080226C0F968184602F052FD02F0A4FC03460121FD
S315080226D0184602F0F4FE0346002B2BD0F968174879
S315080226E003F09EFD26E0FB79062B23D11E21062048
S315080226F0FFF718FD04460620FEF75CFD0346E31ABB
S31508022700FB6002F087FC0346184602F0D2FC034639
S31508022710F968184602F045FD02F07CFC03460121E1
S31508022720184602F0CCFE0346002B03D0F96803488C
S3150802273003F076FD00BF1437BD4690BD748E0308BC
S3150802274080B400AF034B1B681846BD465DF8047B90
S31508022750704700BF301E002080B500AF4FF40062FC
S315080227600E490F480EF05CFF4FF400620D490E4801
S315080227700EF056FF4FF400720C490D480EF050FF4A
S315080227804FF400620B490C480EF04AFF4FF4006200
S315080227900A490B480EF044FF00BF80BD441E0020C4
S315080227A0341E00205426002044260020882E0020AD
S315080227B0782E0020C83000208830002008390020F2
S315080227C0C838002080B483B000AF78607B68002BDD
S315080227D001D1002346E07B68012B01D1012341E0A8
S315080227E07B68022B01D102233CE07B68032B01D1D3
S315080227F0032337E07B68042B01D1042332E07B688C
S31508022800052B01D105232DE07B68062B01D1062372
S3150802281028E07B68072B01D1072323E07B68082B76
S3150802282001D108231EE07B68092B01D80C2319E085
S315080228307B680A2B01D8102314E07B680B2B01D87E
S3150802284014230FE07B680C2B01D818230AE07B6857
S315080228500D2B01D8202305E07B680E2B01D83023E7
S3150802286000E0402318460C37BD465DF8047B7047E6
S3150802287080B483B000AF0346FB80FB88002B01D1EE
S31508022880002346E0FB88012B01D1012341E0FB88A6
S31508022890022B01D102233CE0FB88032B01D103233F
S315080228A037E0FB88042B01D1042332E0FB88052B91
S315080228B001D105232DE0FB88062B01D1062328E04A
S315080228C0FB88072B01D1072323E0FB88082B01D1BC
S315080228D008231EE0FB880C2B01D8092319E0FB8884
S315080228E0102B01D80A2314E0FB88142B01D80B23DA
S315080228F00FE0FB88182B01D80C230AE0FB88202B53
S3150802290001D80D2305E0FB88302B01D80E2300E001
S315080229100F2318460C37BD465DF8047B7047000046
S3150802292084B0B0B400AF07F10C0484E80F00074B7B
S315080229301D4607F10C040FCC0FC50FCC0FC5236833
S315080229402B6000BFBD46B0BC04B07047542E0020B1
S3150802295080B586B000AF78600B467B800023FB7596
S3150802296000233B610023FB600023BB6000F002FDED
S315080229700346002B0BD0444BD3F844323B61424BFF
S31508022980D3F8843AFB607B681B68BB600AE03E4B5F
S31508022990D3F844323B613C4BD3F8843AFB607B68FC
S315080229A01B68BB603A69BB689A4227D1364B93F8D3
S315080229B06832002B0AD1344BD3F850227B88134451
S315080229C0314AC2F850320123FB7558E02E4BB3F850
S315080229D06C321A467B881344B3F5006F0BDA2A4B1E
S315080229E0B3F86C227B8813449AB2274BA3F86C225D
S315080229F00123FB7543E00023FB7540E0FA68BB68D8
S31508022A009A4227D1204B93F8A83A002B0AD11E4B9B
S31508022A10D3F850227B8813441B4AC2F85032022349
S31508022A20FB752CE0184BB3F8AC3A1A467B8813446C
S31508022A30B3F5006F0BDA144BB3F8AC2A7B88134450
S31508022A409AB2114BA3F8AC2A0223FB7517E00023AE
S31508022A50FB7514E03B69002B07D1242279680B48E1
S31508022A6012F001FD0123FB7509E0FB68002B06D174
S31508022A7024227968064812F0F6FC0223FB75FB7DD0
S31508022A8018461837BD4680BD542E002098300020BF
S31508022A90D838002080B584B000AF03463960FB7190
S31508022AA01346BB800023FB81FB79012B12D100233D
S31508022AB0FB810AE0FB893A68134401221946124847
S31508022AC00EF054FEFB890133FB81FA89BB889A42D0
S31508022AD0F0D314E0FB79022B11D10023FB810AE023
S31508022AE0FB893A6813440122194608480EF03EFE4D
S31508022AF0FB890133FB81FA89BB889A42F0D300BF6E
S31508022B001037BD4680BD00BF88300020C838002077
S31508022B1080B582B000AF0346FB71FB1D0122194640
S31508022B2003480EF023FE00BF0837BD4680BD00BF2E
S31508022B30782E0020B0B5B6B000AFF860B9607A60FA
S31508022B40002387F8CF30002387F8D730F86804F0D7
S31508022B5054F8C7F8D000002387F8CF3004E097F876
S31508022B60CF30013387F8CF300721F86804F05AF9D5
S31508022B700346002BF3D17A68B968F86803F0F9FFBF
S31508022B800346002B3AD097F8D730013387F8D73067
S31508022B9002F040FA03460121184602F090FC034669
S31508022BA0002B02D06A4803F03BFB6A4B1B78012BC9
S31508022BB024D0684B01221A7007F1CC03012118466A
S31508022BC00FF0BEFB07F1880207F1CC03114618463F
S31508022BD00FF005FF0FF0CEFF044607F188031846EB
S31508022BE00FF00EFC054607F1880318460FF014FC91
S31508022BF003461A462946204611F0C8F997F8D730EF
S31508022C00002B28D1534B1B78002B24D0514B002282
S31508022C101A7007F1CC03002118460FF091FB07F151
S31508022C20880207F1CC03114618460FF0D8FE0FF0BA
S31508022C30A1FF044607F1880318460FF0E1FB054693
S31508022C4007F1880318460FF0E7FB03461A4629469A
S31508022C50204611F09BF9F86800F0E6FA03461A4690
S31508022C603D4B9A60F86800F0A9FA03463A4A13609F
S31508022C70F86800F0BBFA0346374A5360364B9B683E
S31508022C80002B1CD002F0C6F903460121184602F0B1
S31508022C9016FC0346002B12D02F4B1A682E4B5B6884
S31508022CA007F114002D4912F093FA07F11403184696
S31508022CB003F0B6FA284B9B68184600F0FDFA0C2278
S31508022CC02549274812F008FB0346002B36D0224B2B
S31508022CD01B68DAB207F15803114618460FF0DFFAF5
S31508022CE01D4B5B68DAB207F15803114618460FF016
S31508022CF0F1FA194B9B68DAB207F1580311461846DE
S31508022D000FF003FB07F1140207F1580311461846A0
S31508022D100FF036FE0FF02EFF044607F1140318468D
S31508022D200FF06EFB054607F1140318460FF074FB05
S31508022D3003461A462946204611F028F9084B064A40
S31508022D4007CA83E8070000BFD837BD46B0BD00BF33
S31508022D50988E03082041002008410020BC8E0308F3
S31508022D601441002080B592B000AF3B4640220021B4
S31508022D70184612F0C1FA0023A7F8423000237B64F2
S31508022D809C480EF0D7FC034683F00103DBB2002B06
S31508022D9000F0C480984B93F86832002B50D1964BBA
S31508022DA0D3F850329AB2944BA3F86C22924B0F2264
S31508022DB0C3F8502210233B703B785AB28E4BB3F8B5
S31508022DC06C321B0A9BB25BB203F00F035BB213436E
S31508022DD05BB2DBB23B70884BB3F86C32DBB27B700A
S31508022DE03B4602333E22194682480EF0FAFC034657
S31508022DF0002B00F0FC80FFF7A3FC3B461A467F49EE
S31508022E00FFF798FE7C4BB3F86C323E3B9AB27A4B8C
S31508022E10A3F86C22784BB3F86A3201339AB2764B2E
S31508022E20A3F86A22744B012283F86822724BFF22A6
S31508022E3083F86E22704B4FF4FA62C3F87022D6E01A
S31508022E406D4B93F86E32002B05D06B4B93F86E32AE
S31508022E50012B40F0CC80684BB3F86C323E2B02D97A
S31508022E6040237B6404E0644BB3F86C3201337B6421
S31508022E7020233B703B785AB25F4BB3F86A325BB297
S31508022E8003F00F035BB213435BB2DBB23B707B6C9E
S31508022E905A1E3B460133194656480EF0A2FC034613
S31508022EA0002B00F0A4807B6C9BB21846FFF7E0FC6F
S31508022EB00346514AC2F85032FFF742FC3B461A46CD
S31508022EC04E49FFF737FE4C4BB3F86C227B6C9BB22C
S31508022ED0D31A9BB201339AB2474BA3F86C22464BDC
S31508022EE0B3F86A3201339AB2434BA3F86A22424BC9
S31508022EF0B3F86C32002B7AD1242200213F4812F013
S31508022F00FBF93D4B002283F868223B4B0022A3F8CB
S31508022F106A22394BFF2283F86E2268E038480EF09F
S31508022F2009FC034683F00103DBB2002B5FD03B4664
S31508022F300122194632480EF054FC0346002B53D0A0
S31508022F403B781B09DBB2032B14D13B460133022221
S31508022F5019462B480EF045FC0346002B47D0264B54
S31508022F600322DA60FFF7ECFB3B461A462249FFF7D3
S31508022F70E1FD3CE03B781B09DBB2002B37D13B462F
S31508022F800133012219461E480EF02BFC0346002B7C
S31508022F902CD03B781B029BB203F47063A7F842302D
S31508022FA07B781A46B7F842301343A7F84230B7F887
S31508022FB042203B460233194611480EF012FC0346DC
S31508022FC0002B14D0B7F8423002339BB21846FFF7EB
S31508022FD04FFC0346084AD360FFF7B2FB3B461A4644
S31508022FE00549FFF7A7FD02E000BF00E000BF48372A
S31508022FF0BD4680BD88300020542E0020983000201F
S31508023000782E002080B59AB000AF3B466822002190
S31508023010184612F071F90E480EF08CFB034683F03F
S315080230200103DBB2002B0ED004E03B4668211846AA
S3150802303000F010F83B466822194605480EF0D1FB07
S315080230400346002BF1D100BF6837BD4680BD00BFDD
S315080230504426002080B582B000AF78600B467B809C
S31508023060786800F0E7FB00BF0837BD4680BD000060
S3150802307080B500AF174B93F86832002B28D0154B52
S3150802308093F86E32FF2B23D1124BD3F87032002BF2
S3150802309007D0104BD3F87032013B0E4AC2F8703291
S315080230A016E0242200210C4812F026F94FF4006299
S315080230B00A490B480EF0B4FA064B002283F8682236
S315080230C0044B0022A3F86A22024BFF2283F86E22DF
S315080230D000BF80BD542E002098300020C830002042
S315080230E08830002080B582B000AF78600B467B80BE
S315080230F0786800F0C5FA00BF0837BD4680BD0000F3
S3150802310080B582B000AF78600B467B807B881A4612
S31508023110796803480EF02AFB00BF0837BD4680BD12
S31508023120341E002080B59AB000AF3B4668220021C3
S31508023130184612F0E1F80E480EF0FCFA034683F040
S315080231400103DBB2002B0ED004E03B466821184689
S31508023150FFF7C8FF3B466822194605480EF041FBB1
S315080231600346002BF1D100BF6837BD4680BD00BFBC
S31508023170341E002080B582B000AF78600B4A7B68A7
S315080231801360FFF7E9FA24220021094812F0B4F87D
S3150802319024220021074812F0AFF82422002106480B
S315080231A012F0AAF800BF0837BD4680BD301E0020BF
S315080231B0542E002098300020D838002080B485B0DC
S315080231C000AF78607B681B681B6CBB600023FB60E2
S315080231D0BB68DBB2002B02D0BB68DBB2FB60FB68C4
S315080231E018461437BD465DF8047B704780B485B02F
S315080231F000AF78607B681B681B6CBB600023FB60B2
S31508023200BB6803F4FE43002B06D0BB6803F4FE43F7
S31508023210FB60FB681B0AFB60FB6818461437BD4651
S315080232205DF8047B7047000080B485B000AF786013
S315080232307B681B685B6CBB600023FB60BB6803F0A2
S315080232400703002B2FD0BB6803F00703013B052BAE
S3150802325020D801A252F823F0713202087732020806
S315080232607D32020883320208893202088F32020846
S315080232700123FB600FE00223FB600CE00323FB60E3
S3150802328009E00423FB6006E00523FB6003E006234E
S31508023290FB6000E000BF7B681B685A6C7B681B6892
S315080232A022F007025A64FB68DBB218461437BD4699
S315080232B05DF8047B704700BF80B582B000AF7860C6
S315080232C001F0A8FE03460121184602F0F8F8034663
S315080232D083F00103DBB2002B2AD17B68013B052B65
S315080232E027D801A252F823F001330208093302084B
S315080232F01133020819330208213302082933020856
S315080233000D4802F08DFF14E00C4802F089FF10E028
S315080233100B4802F085FF0CE00A4802F081FF08E03C
S31508023320094802F07DFF04E0084802F079FF00E050
S3150802333000BF0837BD4680BDE08E0308F08E03083D
S31508023340008F0308188F0308308F0308488F030875
S3150802335080B483B000AF0346FB71054AFB7913704C
S31508023360012318460C37BD465DF8047B704700BF3B
S315080233708C05002080B400AF034B1B781846BD4667
S315080233805DF8047B704700BF8C05002080B500AF4E
S31508023390FFF7F0FF0346002B02D04FF4807301E0DB
S315080233A04FF48073184680BD80B500AFFFF7E2FF81
S315080233B00346002B02D04FF4006301E04FF400638A
S315080233C0184680BD80B500AFFFF7D4FF0346002B31
S315080233D002D040F2031301E040F20313184680BDFF
S315080233E0B0B5A4B006AFF860B9601346FB800023F7
S315080233F0A7F87630FB683B65FFF7BCFF0346002B50
S3150802340003D04FF080437B6501E000237B650023F0
S31508023410BB65FB8802339BB21846FFF729FA0346B7
S31508023420FB6500233B664FF480137B664FF400135B
S31508023430BB660023FB6600233B6700233B743B7C89
S315080234405AB2FB881B0A9BB25BB203F00F035BB24C
S3150802345013435BB2DBB23B74FB88DBB27B74022399
S31508023460A7F8763010E0B7F87630023BBA681A4405
S31508023470B7F87630127878333B4403F8682CB7F8F5
S3150802348076300133A7F87630B7F87620FB88013311
S315080234909A42E8DD0023A7F876300DE0B7F87630D1
S315080234A078333B4413F8683C1846FFF731FBB7F804
S315080234B076300133A7F87630B7F87620FB880133E1
S315080234C09A42EBDD6D4607F160040FCC0FC52368FF
S315080234D02B6007F150030FCBFFF722FA00BF7837AC
S315080234E0BD46B0BD80B58EB000AFF860B960134670
S315080234F0FB80002387F83730FB683B61FFF73AFF0A
S315080235000346002B03D04FF080437B6101E0002382
S315080235107B610023BB61FB88FB6100233B624FF49E
S3150802352080137B624FF40013BB620023FB62002305
S315080235303B63FA8807F1100311461846FFF708FAA3
S31508023540034687F8373097F83730002B06D0FA88C3
S3150802355097F83730B9681846FFF79CFA00BF38372C
S31508023560BD4680BDB0B5A2B006AF78600846114622
S315080235701A460346FB700B46BB7013467B70002344
S3150802358087F86F307B68BB64FFF7F4FE0346002BAF
S3150802359003D04FF08043FB6401E00023FB64002361
S315080235A03B6503237B650023BB654FF48013FB65EC
S315080235B04FF400133B6600237B660023BB66302369
S315080235C03B723B7A5AB297F9033003F00F035BB2A8
S315080235D013435BB2DBB23B72BB787B727B78BB72FE
S315080235E0002387F86F300DE097F86F3070333B444D
S315080235F013F8683C1846FFF78BFA97F86F300133D1
S3150802360087F86F3097F86F30022BEDD96D4607F1C0
S3150802361058040FCC0FC523682B6007F148030FCB5C
S31508023620FFF77EF900BF7037BD46B0BD80B582B0E0
S3150802363000AF78600023002200217868FFF792FF26
S3150802364000BF0837BD4680BD80B584B000AFF860BC
S31508023650B9601346FB80FB883E2B06D8FB881A46C0
S31508023660B968F868FFF7BCFE05E0FB881A46B96830
S31508023670F868FFF737FF00BF1037BD4680BD000068
S3150802368080B588B000AF7860FF23FB7600237B61A4
S315080236900023FB6100237B827B68FB60FB6893F84F
S315080236A028301B09FB76FB681B687B61FFF77CFEEB
S315080236B002467B69934202D1FFF784FEF861FB7EDC
S315080236C0032B00F2A78001A252F823F0DD36020886
S315080236D01F37020869370208B7370208FB6893F8EA
S315080236E0283003F00F039AB24C4B1A804B4B1B88B7
S315080236F01B029AB2494B1A80FB6893F829301A467C
S31508023700464B1B8813439AB2444B1A80FB682A33EA
S31508023710424A12881146184600F0C8FB7AE0FB684E
S3150802372093F8283003F00F039AB23C4B1A803B4BAE
S315080237301B881B029AB2394B1A80FB6893F8293008
S315080237401A46364B1B8813439AB2344B1A80344BAB
S3150802375001221A70FB682A333E21184600F0A6FB9E
S31508023760F869FFF763FF55E02D4B1B781A46FB688D
S3150802377093F8283003F00F039A4248D1FB68DB68B6
S315080237801846FFF71FF80346013B7B82FB6829337D
S315080237907A8A1146184600F089FB214B1B780133B9
S315080237A0DAB21F4B1A701E4B1B780F2B2FD91C4BE4
S315080237B000221A702BE01B4BD3F84432FA699A425C
S315080237C00FD1FB6893F8283003F00F03DAB2154BD2
S315080237D083F86E22FB6893F82920124B83F86F222E
S315080237E017E0104BD3F8843AFA699A4211D1FB686A
S315080237F093F8283003F00F03DAB20A4B83F8AE2A9D
S31508023800FB6893F82920074B83F8AF2A01E000BF2B
S3150802381000E000BF00BF2037BD4680BD2241002020
S3150802382024410020542E002080B500AF0FF034FF4B
S3150802383000BF80BD80B584B000AF78607B68FB604E
S31508023840FFF798FD0346002B0AD0FB681B68B3F501
S31508023850806F10D1FB6893F82830002B0BD10AE051
S31508023860FB681B68B3F5806F05D1FB6893F82830AF
S31508023870002B00D100BF00BF1037BD4680BD000037
S3150802388080B500AF4022034903480DF0C9FE012363
S31508023890184680BD384100202841002080B500AF77
S315080238A005480DF047FF0346002B01D0012300E02F
S315080238B00023184680BD00BF2841002080B582B08B
S315080238C000AF78600B46FB70FB781A4679680448A5
S315080238D00EF0BBF8012318460837BD4680BD00BF67
S315080238E02841002080B584B000AF78600023FB73BE
S315080238F0796805480EF0BAF80346FB73FB7B18464F
S315080239001037BD4680BD00BF2841002090B593B050
S3150802391000AF002387F84730FFF7C0FF0346002BA6
S3150802392040F09B8101F076FB03460121184601F01F
S31508023930C6FD0346002B02D0CA4802F071FC3B1DA5
S3150802394040220021184611F0D7FC3B1D1846FFF706
S31508023950C9FF034687F847303B79012B40F07D8142
S3150802396097F84730002B00F078817B79082B17DC13
S31508023970022BC0F26B81023B062B00F2678101A281
S3150802398052F823F0BB3902084D3C02081B3B0208D9
S315080239902D3A0208F13A02084D3C0208073C020891
S315080239A0FF2B40F05381B04802F03AFC01F032FB9B
S315080239B00346184601F054FB4FE13B1D0233AB495F
S315080239C018460EF09EFEA9480EF05EFB03461946FF
S315080239D0A74802F025FCA5480EF056FB0346012B24
S315080239E007D101F017FB03460121184601F052FBE5
S315080239F00CE09E480EF048FB0346022B06D101F066
S31508023A0009FB03460021184601F044FB0FF0B4FDFA
S31508023A10034618460FF0C6FD044694480EF034FBDA
S31508023A200346194620460EF054F916E13B1D0233A9
S31508023A30904918460EF0FEFE8E480EF067FB0346C6
S31508023A4019468D4802F0ECFB0FF096FD0346184620
S31508023A500FF0A8FD0346142118460EF0DCF800F014
S31508023A60C9FA84480EF052FB0346013B072B27D8B6
S31508023A7001A252F823F000BF993A0208D33A020883
S31508023A80A13A0208D33A0208A93A0208B13A020848
S31508023A90B93A0208D33A02080020FEF7DDFB19E01C
S31508023AA00220FEF7D9FB15E00420FEF7D5FB11E04C
S31508023AB00520FEF7D1FB0DE00620FEF7CDFB09E057
S31508023AC06C480EF023FB034619466C4802F0A8FB25
S31508023AD000E000BF00F08EFA0FF04EFD03461846CE
S31508023AE00FF060FD0346152118460EF094F8B4E06F
S31508023AF03B1D0233624918460EF090FF60480EF0ED
S31508023B002EFC03461C465E480EF044FC03461A4643
S31508023B1021465C4802F084FB9FE03B1D02335A496A
S31508023B2018460EF055FE58480EF0D5FA03461946C1
S31508023B30564802F075FB0FF01FFD034618460FF0B4
S31508023B4031FD0346162118460EF065F84E480EF06A
S31508023B50C2FA0346012B03D10020FEF715FD44E005
S31508023B6049480EF0B8FA0346022B03D10120FEF7A4
S31508023B700BFD3AE044480EF0AEFA0346032B03D196
S31508023B800220FEF701FD30E03F480EF0A4FA034694
S31508023B90042B03D10320FEF7F7FC26E03A480EF081
S31508023BA09AFA0346052B03D10420FEF7EDFC1CE026
S31508023BB035480EF090FA0346062B03D10520FEF788
S31508023BC0E3FC12E030480EF086FA0346072B03D1CF
S31508023BD00620FEF7D9FC08E02B480EF07CFA0346CD
S31508023BE0082B02D10720FEF7CFFCFDF7A9FA0FF042
S31508023BF0C3FC034618460FF0D5FC034617211846A0
S31508023C000EF009F829E03B1D0233214918460EF049
S31508023C1058FF1F480EF0D9FB034619461D4802F005
S31508023C20FFFA1B480EF0D1FB0346002B14D10FF006
S31508023C30A3FC034618460FF0B5FC034600211846B6
S31508023C400EF004F8144802F0EBFA05E07B791946FF
S31508023C50124802F0E5FA00E000BF00BF4C37BD4645
S31508023C6090BD00BF548F0308808F03087841002057
S31508023C709C8F030880410020E08F03082C900308DC
S31508023C80844100205C9003087C410020B090030820
S31508023C9088410020FC9003083C9103085C910308C4
S31508023CA080B582B000AF78600B467B8009480DF07C
S31508023CB0E3FC02467B889A4207D37B881A467968D0
S31508023CC004480DF0C2FE012300E000231846083717
S31508023CD0BD4680BD8C41002080B5C4B000AF024607
S31508023CE007F58873A3F209131A70002387F80F31B0
S31508023CF023E007F10C034FF480720021184611F0F5
S31508023D00FBFA07F10C03194615480DF015FF034691
S31508023D1087F80F3107F10C03194611480DF0A6FE74
S31508023D20034687F80F31FFF74DFB97F80F319AB222
S31508023D3007F10C031946FFF787FC09480DF0FAFC50
S31508023D40034683F00103DBB2002B03D0054B1B7835
S31508023D50002BCED000BF07F58877BD4680BD00BFD1
S31508023D608C4100209C41002080B483B000AF78606B
S31508023D700B467B8000BF00BF0C37BD465DF8047B4F
S31508023D807047000080B582B000AF0023FB712A4B52
S31508023D901B78002B48D0294B1B780133DAB2274B04
S31508023DA01A70264B1B78092B41D9244B00221A700C
S31508023DB0214B5B78012B17D81F4B5B780133DAB29C
S31508023DC01D4B5A70FFF7FEFA03461B4A92F88320E8
S31508023DD01B491846FFF738FC01F01CF90346012176
S31508023DE0184601F06CFB22E001F014F903460121A2
S31508023DF0184601F064FB0346002B0BD00023FB7127
S31508023E0002E0FB790133FB710B4B93F88330FA79A5
S31508023E109A42F6D30A490B480DF028FE842200215D
S31508023E20054811F069FA02E0044B00221A7000BF35
S31508023E300837BD4680BD00BF9C41002020420020B5
S31508023E409F4100208C41002080B582B000AF786087
S31508023E5039603B68DBB21946786800F04BF800BF58
S31508023E600837BD4680BD80B582B000AF786039603C
S31508023E703B689BB219467868FFF712FF00BF0837FE
S31508023E80BD4680BD80B582B000AF78603960064B0A
S31508023E901B683A6892B2796818460DF0BBF900BFFA
S31508023EA00837BD4680BD00BF9005002080B582B0A8
S31508023EB000AF78603960054B1B683A68796818461E
S31508023EC00DF042FA00BF0837BD4680BD90050020B6
S31508023ED080B500AF044B1868044B054A00210DF063
S31508023EE05EF900BF80BD00BF90050020673E02084C
S31508023EF0493E020890B585B000AF78600B46FB7064
S31508023F0001F088F8F860FB789BB219467868FFF7E3
S31508023F102BFF7B681B780F2B23D00F2B48DC012B3A
S31508023F2002D0052B31D043E0244B9B78194624480E
S31508023F300EF0C0FF214BDB78194621480EF0D6FF5A
S31508023F4020491F480EF044FF1E480EF08FFF044614
S31508023F501C480EF097FF034619462046FFF792FFC4
S31508023F6027E0194B01221A70164917480EF053FF1B
S31508023F7014480EF07BFF044612480EF083FF0346F0
S31508023F8019462046FFF77EFF13E0F86801F068F845
S31508023F900C480EF059FF0B480EF068FF0446094814
S31508023FA00EF070FF034619462046FFF76BFF00E046
S31508023FB000BF00BF1437BD4690BD00BFE0BF1F0853
S31508023FC058530020505200205453002080B500AFA9
S31508023FD003480BF045F802480AF002FF00BF80BD0D
S31508023FE02054002080B500AF00F0C2F902F008F9AB
S31508023FF000BF80BD80B500AF01F00CF80346184635
S3150802400001F022F80346002B02D1024804F01EF8FA
S3150802401000BF80BDC053002080B582B000AF304BD0
S31508024020304A9A6062B600BF02F098F900F076F854
S3150802403000F0EAF900F0DCF800F022F900F042F9A3
S3150802404000F048F900F094F927480AF06BF802F0F4
S31508024050D7F82648FFF78EF800F098FCFFF738FFE6
S315080240600FF018FFFFF70CFCFDF72AF80346FB7161
S31508024070FDF76AFFFB79002B2CD01D4802F0D0F819
S315080240800020FEF7E9F81B4802F0CAF81A4802F0BF
S31508024090C7F80220FEF7E0F8184802F0C1F81848F7
S315080240A002F0BEF80420FEF7D7F8164802F0B8F870
S315080240B0154802F0B5F80520FEF7CEF8134802F0C7
S315080240C0AFF8134802F0ACF80620FEF7C5F8114817
S315080240D002F0A6F8104802F0A3F801F0CFFBFCE7BD
S315080240E000ED00E000600008D45300205C53002075
S315080240F088910308A8910308C8910308E891030860
S31508024100089203082892030848920308689203084B
S3150802411088920308A8920308C892030880B59CB03F
S3150802412000AF07F1200350220021184611F0E4F8E7
S3150802413007F1080300221A605A609A60DA601A6167
S315080241405A612A4B1B69294A43F030031361274BEC
S315080241501B6903F030037B607B6800BF234B5B69F6
S3150802416003F00803082BF9D109233B624FF4803385
S315080241707B624FF08063BB630223BB640323FB6449
S3150802418003233B657D237B650223BB650223FB650F
S3150802419002233B6608237B660023BB660023FB6675
S315080241A007F12003184603F061FF0346002B01D0EE
S315080241B000F0AAFA1F23BB600323FB6000233B61BE
S315080241C000237B610023BB610023FB6107F108031F
S315080241D00521184604F082FB0346002B01D000F0A5
S315080241E093FA00BF7037BD4680BD00BF000802447F
S315080241F080B500AF204B214A1A601F4B00225A6035
S315080242001D4B4FF440729A601B4B0022DA601A4B20
S3150802421000221A74184B00225A74174B00229A74F9
S31508024220154B05225A61144B0A229A61124B272210
S31508024230DA61114B0A221A620F4B05225A620E4B99
S3150802424002229A620C4B0722DA620B4B02221A638B
S31508024250094B01225A63084B01229A63064B002234
S31508024260DA63054802F078FA0346002B01D000F01B
S315080242704BFA00BF80BD00BF5C53002000A400407B
S3150802428080B500AF0D4B0E4A1A600C4B05225A60D8
S315080242900A4B40F2EE22DA60084B40F2EE229A60AE
S315080242A0064B00221A61054803F048FE0346002B16
S315080242B001D000F029FA00BF80BD00BFC05300201C
S315080242C00030004080B400AF00BFBD465DF8047BF5
S315080242D07047000080B588B000AF07F110030022CE
S315080242E01A605A609A60DA603B1D00221A605A60A8
S315080242F09A601E4B4FF080421A601C4B40F6C3125E
S315080243005A601A4B00229A60184B6322DA60174BDE
S3150802431000221A61154B00229A61144809F0AAFE76
S315080243200346002B01D000F0EFF94FF480533B61AE
S3150802433007F1100319460D480AF0ECF80346002B5C
S3150802434001D000F0E1F900237B600023FB603B1DEE
S31508024350194606480AF0DEFB0346002B01D000F098
S31508024360D3F900BF2037BD4680BD00BFD453002015
S3150802437080B500AF224B234A1A60214B4FF4E13233
S315080243805A601F4B00229A601D4B0022DA601C4BB2
S3150802439000221A611A4B0C225A61194B00229A61A1
S315080243A0174B0022DA61164B00221A62144B0022BE
S315080243B05A62134B00229A6211480AF0C1FC03465C
S315080243C0002B01D000F0A0F900210D480CF031FDB8
S315080243D00346002B01D000F097F9002108480CF09B
S315080243E066FD0346002B01D000F08EF904480CF056
S315080243F0E7FC0346002B01D000F086F900BF80BD1A
S31508024400205400200038014080B58EB000AF07F175
S31508024410240300221A605A609A60DA601A61A74B6E
S31508024420D3F88C30A54A43F02003C2F88C30A34B4C
S31508024430D3F88C3003F020033B623B6A9F4BD3F8D8
S315080244408C309E4A43F08003C2F88C309B4BD3F8DB
S315080244508C3003F08003FB61FB69984BD3F88C30F0
S31508024460964A43F00403C2F88C30944BD3F88C3046
S3150802447003F00403BB61BB69904BD3F88C308F4AB7
S3150802448043F04003C2F88C308C4BD3F88C3003F0DF
S3150802449040037B617B69894BD3F88C30874A43F0AA
S315080244A01003C2F88C30854BD3F88C3003F0100316
S315080244B03B613B69814BD3F88C30804A43F0080351
S315080244C0C2F88C307D4BD3F88C3003F00803FB60BE
S315080244D0FB687A4BD3F88C30784A43F00103C2F86A
S315080244E08C30764BD3F88C3003F00103BB60BB6883
S315080244F0724BD3F88C30714A43F00203C2F88C30FF
S315080245006E4BD3F88C3003F002037B607B68002283
S315080245104FF481716A4803F0DFFC002220216948C2
S3150802452003F0DAFC002240F62101674803F0D4FCC6
S3150802453000224FF40051654803F0CEFC00224FF4E6
S315080245400071634803F0C8FC00224021614803F069
S31508024550C3FC81237B620023BB620023FB6207F153
S3150802456024031946564803F091FA4FF481737B6285
S315080245700123BB620023FB6203233B6307F1240387
S3150802458019464F4803F082FA10237B620023BB6266
S315080245900023FB6207F1240319464A4803F076FA18
S315080245A020237B620123BB620023FB6203233B6356
S315080245B007F124031946434803F068FA01237B628C
S315080245C00123BB620023FB6200233B6307F124033A
S315080245D019463D4803F05AFA4FF480537B6200238A
S315080245E0BB620023FB6207F124031946374803F02E
S315080245F04DFA4FF400537B620123BB620023FB6230
S3150802460003233B6307F124031946304803F03EFAB5
S315080246104FF480737B620023BB620023FB6207F1BF
S31508024620240319462A4803F031FA4FF400737B62D1
S315080246300123BB620023FB6203233B6307F12403C6
S315080246401946234803F022FA4FF482637B62002359
S31508024650BB620023FB6207F1240319461A4803F0DA
S3150802466015FA4FF402637B620123BB620023FB62E5
S3150802467003233B6307F124031946134803F006FA9A
S3150802468020237B620023BB620023FB6207F124031B
S315080246901946104803F0FAF940237B620123BB62EC
S315080246A00023FB6203233B6307F1240319460948E7
S315080246B003F0ECF900BF3837BD4680BD000C024452
S315080246C00014024200080242001802420010024286
S315080246D0000C02420004024280B582B000AF786044
S315080246E07B681B68074A934201D101F05DFE7B682D
S315080246F01B68B3F1804F01D100F0F0FF00BF083705
S31508024700BD4680BD0010004080B400AF72B600BF3F
S3150802471000BFFDE7B0B596B000AF786039600023F8
S315080247207B6545E0644B654A4021786802F072FA77
S315080247300346002B0DD000F06DFC034601211846F6
S3150802474000F0BDFE0346002B32D05D4801F068FD3D
S315080247502EE0FEF70FFE0346002B03D0574B1B68CD
S315080247607B6502E0554B1B687B65FEF71DFE02461C
S315080247707B6D934204D168215048FEF7C1FC17E0CD
S315080247800EF0DEF902467B6D934205D00EF0E5F98E
S3150802479002467B6D93420BD1484BDB681846FEF7FF
S315080247A011F80346DBB21A464349786D0FF0B8FB97
S315080247B04021786802F04CFB0346002BB2D1786898
S315080247C0FEF732FD03461A463E4B9A607868FEF7B4
S315080247D0F5FC03463B4A13607868FEF707FD034675
S315080247E0384A5360374B9B68002B1CD000F012FCEA
S315080247F003460121184600F062FE0346002B12D03A
S31508024800304B1A682F4B5B6807F10C002E4910F0E3
S31508024810DFFC07F10C03184601F002FD294B9B68E1
S315080248201846FEF749FD0C222649284810F054FD81
S315080248300346002B36D0234B1B68DAB207F1500326
S31508024840114618460DF02BFD1E4B5B68DAB207F1CE
S315080248505003114618460DF03DFD1A4B9B68DAB215
S3150802486007F15003114618460DF04FFD07F10C02E9
S3150802487007F15003114618460EF082F80EF07AF93F
S31508024880044607F10C0318460DF0BAFD054607F172
S315080248900C0318460DF0C0FD03461A462946204663
S315080248A00FF074FB094B074A07CA83E8070000BFE3
S315080248B05837BD46B0BD00BFDC540020B4540020B2
S315080248C0F0920308084100201093030814410020BF
S315080248D080B58AB002AF78600B467B8013463B8070
S315080248E00023BB600023FB607B683B6101237B617D
S315080248F07B88BB613B88FB6107F1080319460748B9
S3150802490002F084F8012300930123022202210348BC
S3150802491002F0D6F800BF2037BD4680BD5C530020A2
S3150802492080B58CB002AFF860B9607A604FF0804308
S315080249303B6100237B61FB68BB610123FB61BB68AA
S315080249403B627B687B6207F110031946074802F04F
S315080249505DF801230093012302220221034802F093
S31508024960AFF800BF2837BD4680BD00BF5C530020A4
S3150802497080B500AF044802F0D4F8002201210248AB
S3150802498002F084FA00BF80BD5C53002080B500AFF8
S31508024990FEF7F0FC0346002B09D0FEF705FD034699
S315080249A01A466FF060410220FFF7BAFF09E0FEF7E8
S315080249B0FBFC03469BB21A464FF6FF710220FFF72D
S315080249C087FFFFF7D5FF00BF80BD000080B58EB018
S315080249D000AFF860B9601346FB71FB79002B02D071
S315080249E0FB79402B01D9002330E007F11403242276
S315080249F00021184610F080FCFB687B61FEF7BAFCC2
S31508024A000346002B03D04FF08043BB6101E000232D
S31508024A10BB610023FB61FB799BB21846FDF728FFB1
S31508024A2003463B6200237B624FF48013BB624FF45A
S31508024A300013FB6200233B6300237B6307F1140325
S31508024A40BA6819460348FEF775F801231846383737
S31508024A50BD4680BD5C53002080B400AF00BFBD4692
S31508024A605DF8047B7047000080B5CCB000AF07F54F
S31508024A709873A3F59673186007F58E7300221A6069
S31508024A805A609A60DA601A6107F59873A3F590730B
S31508024A9018464FF484731A46002110F02DFC07F5C8
S31508024AA09873A3F596731B681B68384A934267D1B5
S31508024AB007F59873A3F590714FF000024FF00403BF
S31508024AC0C1E9002307F59873A3F590734FF4807232
S31508024AD0C3F8BC2007F11003184604F079FA034616
S31508024AE0002B01D0FFF710FE294BD3F8A030284A35
S31508024AF043F40073C2F8A030254BD3F8A03003F470
S31508024B00007207F59873A3F592731A6007F59873FE
S31508024B10A3F592731B681E4BD3F88C301C4A43F0DC
S31508024B200103C2F88C301A4BD3F88C3003F0010219
S31508024B3007F59873A3F594731A6007F59873A3F5A6
S31508024B4094731B684FF4C053C7F81C310223C7F885
S31508024B5020310023C7F824310323C7F82831092353
S31508024B60C7F82C3107F58E7319460A4802F08EFFEC
S31508024B7000220021272001F013FD272001F02AFD3B
S31508024B8000BF07F59877BD4680BD00BF00A4004068
S31508024B90000C02440000024280B584B000AF78607F
S31508024BA07B681B68B3F1804F16D10D4BD3F89C3046
S31508024BB00B4A43F00103C2F89C30094BD3F89C30E8
S31508024BC003F00103FB60FB68002200212D2001F09F
S31508024BD0E7FC2D2001F0FEFC00BF1037BD4680BD64
S31508024BE0000C024480B5CCB000AF07F59873A3F564
S31508024BF09673186007F58E7300221A605A609A60D7
S31508024C00DA601A6107F59873A3F5907318464FF49C
S31508024C1084731A46002110F06FFB07F59873A3F503
S31508024C2096731B681B68374A934265D107F59873D2
S31508024C30A3F590714FF001024FF00003C1E900237A
S31508024C4007F59873A3F590730022DA6507F1100346
S31508024C50184604F0BDF90346002B01D0FFF754FDB0
S31508024C60294BD3F8A430284A43F48043C2F8A43027
S31508024C70254BD3F8A43003F4804207F59873A3F5BD
S31508024C8092731A6007F59873A3F592731B681E4B05
S31508024C90D3F88C301C4A43F00103C2F88C301A4B05
S31508024CA0D3F88C3003F0010207F59873A3F59473D1
S31508024CB01A6007F59873A3F594731B684FF4C063DB
S31508024CC0C7F81C310223C7F820310023C7F824315C
S31508024CD00323C7F828310723C7F82C3107F58E7343
S31508024CE019460A4802F0D2FE002200213A2001F0B3
S31508024CF057FC3A2001F06EFC00BF07F59877BD46CF
S31508024D0080BD00BF00380140000C02440000024288
S31508024D1080B582B000AF78607B681B680B4A934205
S31508024D200FD10B4BD3F8A430094A23F48043C2F8B7
S31508024D30A4304FF4C061074802F0FAFF3A2001F0A6
S31508024D4057FC00BF0837BD4680BD00BF003801408A
S31508024D50000C02440000024280B58EB000AF7860B3
S31508024D60334BD3F89C30324A43F01003C2F89C30D6
S31508024D702F4BD3F89C3003F01003BB60BB6807F1D6
S31508024D800C0207F110031146184604F0E9F8FB690C
S31508024D90FB62FB6A002B03D104F0A0F8786304E0F7
S31508024DA004F09CF803465B007B637B6B5B09214A34
S31508024DB0A2FB0323DB09013BBB621F4B1F4A1A6096
S31508024DC01D4B6322DA601C4ABB6A53601A4B0022E7
S31508024DD01A61194B00229A60174809F04BF90346E3
S31508024DE087F8333097F83330002B18D1124809F078
S31508024DF099F9034687F8333097F83330002B0ED1EA
S31508024E007B680F2B08D800227968312001F0C8FB8D
S31508024E100B4A7B68136002E0012387F8333031209E
S31508024E2001F0D8FB97F8333018463837BD4680BDAF
S31508024E30000C0244C55A7C0A1C550020001000408A
S31508024E409805002080B400AF00BFFDE780B400AF2C
S31508024E5000BFFDE780B400AF00BFFDE780B400AF36
S31508024E6000BFFDE780B400AF00BFFDE780B400AF26
S31508024E7000BFBD465DF8047B704780B400AF00BF33
S31508024E80BD465DF8047B704780B400AF00BFBD46DF
S31508024E905DF8047B704780B400AF00BFBD465DF87D
S31508024EA0047B704780B500AF024802F0D5F800BF10
S31508024EB080BD00BF5C53002080B500AF024809F0F0
S31508024EC0DFF900BF80BD00BFD453002080B500AF14
S31508024ED0024809F0D5F900BF80BD00BF1C55002065
S31508024EE080B500AF02480AF06FF900BF80BD00BF67
S31508024EF02054002080B400AF01231846BD465DF851
S31508024F00047B704780B582B000AF7860396010F0D4
S31508024F1067FA034616221A604FF0FF331846083717
S31508024F20BD4680BD80B582B000AF78604FF0FF31D4
S31508024F307868FFF7E7FF00BFFDE780B586B000AFE8
S31508024F40F860B9607A6000237B610AE0AFF30080FB
S31508024F500146BB685A1CBA60CAB21A707B69013329
S31508024F607B617A697B689A42F0DB7B681846183758
S31508024F70BD4680BD80B586B000AFF860B9607A607C
S31508024F8000237B6109E0BB685A1CBA601B78184685
S31508024F90AFF300807B6901337B617A697B689A4249
S31508024FA0F1DB7B6818461837BD4680BD80B483B0EE
S31508024FB000AF78604FF0FF3318460C37BD465DF8F0
S31508024FC0047B704780B483B000AF786039603B6871
S31508024FD04FF400525A60002318460C37BD465DF856
S31508024FE0047B704780B483B000AF7860012318460B
S31508024FF00C37BD465DF8047B704780B485B000AFB8
S31508025000F860B9607A60002318461437BD465DF821
S31508025010047B704780B500AF094B1B78DBB2002BC7
S315080250200AD1074B01221A706C220021054810F09A
S3150802503063F90120FEF78CF9024B184680BD00BFC2
S31508025040D45500206855002080B483B000AF78603C
S315080250507B681B7818460C37BD465DF8047B70479B
S3150802506080B483B000AF78607B6801221A7001238E
S3150802507018460C37BD465DF8047B704780B483B08A
S3150802508000AF78607B685B7818460C37BD465DF8DA
S31508025090047B704780B483B000AF78600B46FB7020
S315080250A07B68FA785A7000BF0C37BD465DF8047BF8
S315080250B0704780B483B000AF78607B6804331846C3
S315080250C00C37BD465DF8047B704780B483B000AFE9
S315080250D0786039607B683A685A60012318460C374B
S315080250E0BD465DF8047B704780B483B000AF786034
S315080250F07B685B6818460C37BD465DF8047B7047CB
S3150802510080B483B000AF786039607B683A68DA6049
S31508025110012318460C37BD465DF8047B704780B4F8
S3150802512083B000AF78607B68DB6818460C37BD46EB
S315080251305DF8047B704780B483B000AF786039604D
S315080251407B683A685A61012318460C37BD465DF8F2
S31508025150047B704780B483B000AF78607B685B6974
S3150802516018460C37BD465DF8047B704780B483B099
S3150802517000AF786039607B683A689A6101231846FD
S315080251800C37BD465DF8047B704780B483B000AF28
S3150802519078607B689B6918460C37BD465DF8047BC8
S315080251A0704780B483B000AF786039607B683A682C
S315080251B0DA61012318460C37BD465DF8047B704751
S315080251C080B483B000AF78607B68DB6918460C3719
S315080251D0BD465DF8047B704780B483B000AF786043
S315080251E087ED000A7B683A689A62012318460C37EB
S315080251F0BD465DF8047B704780B483B000AF786023
S315080252007B689B6A07EE903AB0EE670A0C37BD4692
S315080252105DF8047B704780B483B000AF78607B6822
S31508025220DB6A07EE903AB0EE670A0C37BD465DF8C0
S31508025230047B704780B483B000AF786087ED000ABC
S315080252407B683A681A63012318460C37BD465DF82F
S31508025250047B704780B483B000AF78607B681B6BB1
S3150802526007EE903AB0EE670A0C37BD465DF8047B46
S31508025270704780B483B000AF78607B685B6B07EEDB
S31508025280903AB0EE670A0C37BD465DF8047B704764
S3150802529080B483B000AF786087ED000A7B683A680D
S315080252A09A63012318460C37BD465DF8047B70479E
S315080252B080B483B000AF78607B689B6B07EE903A48
S315080252C0B0EE670A0C37BD465DF8047B704780B4BA
S315080252D083B000AF786087ED000A7B683A68DA63C4
S315080252E0012318460C37BD465DF8047B704780B427
S315080252F083B000AF78607B68DB6B07EE903AB0EE5E
S31508025300670A0C37BD465DF8047B704780B483B0E4
S3150802531000AF786087ED000A7B683A681A64012351
S3150802532018460C37BD465DF8047B704780B483B0D7
S3150802533000AF78607B681B6C07EE903AB0EE670A9E
S315080253400C37BD465DF8047B704780B483B000AF66
S3150802535078607B685B6C07EE903AB0EE670A0C37AA
S31508025360BD465DF8047B704780B483B000AF7860B1
S3150802537039607B683A689A64012318460C37BD4639
S315080253805DF8047B704780B483B000AF78607B68B1
S315080253909B6C18460C37BD465DF8047B704780B493
S315080253A083B000AF78607B68DB6C18460C37BD4665
S315080253B05DF8047B704780B483B000AF78603960CB
S315080253C07B683A681A65012318460C37BD465DF8AC
S315080253D0047B704780B483B000AF78607B681B6D2E
S315080253E018460C37BD465DF8047B704780B483B017
S315080253F000AF78607B685B6D18460C37BD465DF872
S31508025400047B704780B483B000AF786039607B68EC
S315080254103A689A65012318460C37BD465DF8047B3F
S31508025420704780B483B000AF78607B689B6D18467E
S315080254300C37BD465DF8047B704780B483B000AF75
S31508025440786039607B683A68DA65012318460C3752
S31508025450BD465DF8047B704780B483B000AF7860C0
S315080254607B68DB6D18460C37BD465DF8047B7047D2
S3150802547080B483B000AF786039607B683A681A6690
S31508025480012318460C37BD465DF8047B704780B485
S3150802549083B000AF78607B681B6E18460C37BD4632
S315080254A05DF8047B704780B483B000AF78607B6890
S315080254B05B6E18460C37BD465DF8047B704780B4B0
S315080254C085B000AF78600B46FB70FB78002B01D1E4
S315080254D000230BE07B6893F86820FB781340DBB265
S315080254E0002B14BF01230023FB73FB7B18461437DA
S315080254F0BD465DF8047B704780B483B000AF786020
S315080255000B46FB70FB78002B01D100230BE07B686E
S3150802551093F86820FB781343DAB27B6883F868202D
S315080255207B6893F8683018460C37BD465DF8047BED
S31508025530704780B483B000AF78600B46FB70FB7887
S31508025540002B01D1002310E07B6893F868305AB229
S3150802555097F90330DB435BB213405BB2DAB27B687E
S3150802556083F868207B6893F8683018460C37BD467E
S315080255705DF8047B7047000080B586B000AF78609E
S31508025580144A154BD31A7B617B693B61134B1B6823
S31508025590002B02D1114B124A1A60104B1A687B680B
S315080255A013443A699A4207D20FF01AFF03460C22AD
S315080255B01A604FF0FF3309E0084B1B68FB60074B84
S315080255C01A687B681344054A1360FB68184618373D
S315080255D0BD4680BD00000A2000040000D855002000
S315080255E0F85F002080B483B000AF354BD3F888301B
S315080255F0334A43F47003C2F88830324B01221A60E8
S31508025600304B0022DA612F4B00221A622D4B1A68A0
S315080256102C492D4B13400B602A4B00229A62294BC8
S315080256200022DA62274B00221A63264B274A5A635C
S31508025630244B00229A63234B244ADA63214B002225
S315080256401A64204B214A5A641E4B00229A641D4B47
S315080256501B681C4A23F4802313601A4B00221A651E
S31508025660174B4FF000629A60194B9B6903F060432F
S315080256707B607B68B3F1604F03D07B68B3F1404F20
S3150802568017D1134BDB6903F00103002B05D0104B2E
S31508025690104ADA600E4B104ADA600D4BDB690C4A87
S315080256A043F00203D3610A4BDB69094A43F001035B
S315080256B0D36100BF0C37BD465DF8047B704700BF57
S315080256C000ED00E0000C0244E3EAE2EA800201018E
S315080256D0002002403B2A19087F6E5D4C80B400AF59
S315080256E0214B1B8801339AB21F4B1A801F4B01228A
S315080256F01A701D4B1A881E4BA3FB0213D9080B46B8
S315080257009B000B445B00D31A9BB2002B02D1194BA8
S3150802571001221A70144B1B88174AA2FB031252095C
S31508025720642101FB02F29B1A9BB2002B02D1134B96
S3150802573001221A700C4B1B88114AA2FB031292090A
S315080257404FF47A7101FB02F29B1A9BB2002B05D128
S315080257500C4B01221A70044B00221A8000BFBD4668
S315080257605DF8047B704700BFDC550020DE5500203B
S31508025770CDCCCCCCDF5500201F85EB51E05500205F
S31508025780D34D6210E155002098B500AFFEF732FC02
S31508025790FFF740FC04460020FCF7BEFDF0EE407A17
S315080257A0B0EE670A2046FFF717FDFEF723FCFFF760
S315080257B031FC04460220FCF7AFFDF0EE407AB0EE6B
S315080257C0670A2046FFF736FDFEF714FCFFF722FCB0
S315080257D004460420FCF7A0FDF0EE407AB0EE670A14
S315080257E02046FFF755FDFEF705FCFFF713FC0446B6
S315080257F00520FCF791FDF0EE407AB0EE670A2046E6
S31508025800FFF765FDFEF7F6FBFFF704FC04460620E4
S31508025810FCF782FDF0EE407AB0EE670A2046FFF703
S3150802582075FDFEF7E7FB00BF98BD0000B0B592B064
S3150802583000AF114B1A883B46114618460CF014FD68
S315080258403A1D3B46114618460DF07BF80DF092F9C3
S3150802585004463B1D18460CF0D3FD05463B1D18466B
S315080258600CF0DAFD03461A46294620460EF08EFB50
S3150802587000BF4837BD46B0BDEA550020B0B592B064
S3150802588000AFC24B1B78002B13D0C04B00221A70F4
S31508025890FEF73CF8FDF746FCFDF7B4FBFDF762FAA6
S315080258A0FDF7E6FB0DF04EFF0EF02CF90020FEF791
S315080258B013FAB74B1B78002B08D0B54B00221A7087
S315080258C0B44B1B780133DAB2B24B1A70B14B1B7860
S315080258D0042B02D9AF4B00221A70AF4B1B78002B50
S315080258E060D0AD4B00221A70AC4B1B780133DAB28A
S315080258F0AA4B1A700EF0C0F80EF008F80EF09CFAD1
S315080259000EF0E4F9FEF73EFAA54800F0F9FBFFF7B8
S3150802591081FB03461846FFF7B1FB0346012B03D169
S31508025920FFF732FF00F003FA0DF026FE034618468B
S315080259300DF038FE0346012118460CF0A2F903467B
S31508025940002B29D10DF018FE034618460DF02AFE43
S315080259500346022118460CF094F90346002B1BD184
S315080259600DF00AFE034618460DF01CFE03460421F6
S3150802597018460CF086F90346002B0DD10DF0FCFDF6
S31508025980034618460DF00EFE0346082118460CF08B
S3150802599078F90346002B03D00421824802F0B4FAB0
S315080259A0FEF728FB7D4B1B78012B11D97B4B002276
S315080259B01A7000F097F9FFF72DFB03461846FFF712
S315080259C05DFB0346002B03D1FFF7DEFE00F0AFF9BD
S315080259D0754B1B78002B00F02681734B00221A7038
S315080259E0724B1B780133DAB2704B1A70704B1B7804
S315080259F00133DAB26E4B1A706E4B1B780133DAB288
S31508025A006C4B1A706C4B1B780133DAB26A4B1A70FC
S31508025A106A4B1B780133DAB2684B1A70684B1B88DB
S31508025A2001339AB2664B1A800DF0A6FD0346184654
S31508025A300DF0B8FD0346012118460CF022F903467B
S31508025A4083F00103DBB2002B36D00DF095FD034639
S31508025A5018460DF0A7FD0346022118460CF011F967
S31508025A60034683F00103DBB2002B25D00DF084FD3B
S31508025A70034618460DF096FD0346042118460CF017
S31508025A8000F9034683F00103DBB2002B14D00DF0B4
S31508025A9073FD034618460DF085FD03460821184690
S31508025AA00CF0EFF8034683F00103DBB2002B03D0B8
S31508025AB004213C4802F028FAFFF7ACFA0346012112
S31508025AC01846FFF7FCFC0346002B0FD0FFF7A2FA95
S31508025AD003461846FFF790FB10EE103A1846FAF7F7
S31508025AE043FD02460B46374800F09AFBFFF792FA47
S31508025AF0034601211846FFF7E2FC0346002B0FD0A6
S31508025B00FFF788FA03461846FFF7A4FB10EE103A89
S31508025B101846FAF729FD02460B462B4800F080FB89
S31508025B20FFF778FA034601211846FFF7C8FC034631
S31508025B30002B02D0254800F073FBFFF76BFA0346E9
S31508025B4001211846FFF7BBFC0346002B02D020486A
S31508025B5000F066FBFFF75EFA034601211846FFF7D7
S31508025B60AEFC0346002B37D00DF006FD0346184659
S31508025B700DF018FD0346012118460CF082F803467B
S31508025B801946144800F04CFB26E000BFDE550020FB
S31508025B90DF550020E8550020E0550020E755002093
S31508025BA0F53F020800040242E1550020E2550020B2
S31508025BB0E3550020E4550020E5550020E95500206C
S31508025BC0EA550020349303084493030854930308C0
S31508025BD05893030864930308FFF71CFA0346012146
S31508025BE01846FFF76CFC0346002B0FD00DF0C4FCD9
S31508025BF0034618460DF0D6FC0346042118460CF057
S31508025C0040F8034619462F4800F00AFBFFF702FA46
S31508025C10034601211846FFF752FC0346002B02D021
S31508025C20294800F0FDFA294B1B78012B02D9274B8C
S31508025C3000221A70264B1B78022B25D9244B0022E8
S31508025C401A70244B1B78002B1ED1224B01221A7084
S31508025C5000F074F901233B703A1D3B46114618467B
S31508025C600CF097FD0CF086FF04463B1D18460CF017
S31508025C70C7FB05463B1D18460CF0CEFB03461A46E3
S31508025C80294620460EF082F9134B1B78042B02D9BB
S31508025C90114B00221A70114B1B780E2B04D90F4B8D
S31508025CA000221A70FDF7C0FD0D4B1B783B2B04D959
S31508025CB00B4B00221A70FFF7B9FD00BF4837BD46E5
S31508025CC0B0BD00BF6493030854930308E25500204D
S31508025CD0E3550020E6550020E4550020E55500204E
S31508025CE0E9550020B0B592B000AF0DF045FC034669
S31508025CF018460DF057FC02463B1D194610460CF095
S31508025D0013FC0CF044FF04463B1D18460CF078FBC6
S31508025D1005463B1D18460CF07FFB03461A462946E4
S31508025D2020460EF033F900BF4837BD46B0BDB0B5C0
S31508025D30A2B000AF07F148034022002118460FF02F
S31508025D40DBFAFFF767F903461846FFF755FAF0EE4E
S31508025D50407A07F14803B0EE670A18460BF0E3FFEC
S31508025D60FFF758F903461846FFF755FAF0EE407A58
S31508025D7007F14803B0EE670A18460BF0F2FFFFF781
S31508025D8049F903461846FFF765FAF0EE407A07F135
S31508025D904803B0EE670A18460CF001F8FFF73AF91D
S31508025DA003461846FFF765FAF0EE407A07F148030C
S31508025DB0B0EE670A18460CF010F8FFF72BF90346FF
S31508025DC01846FFF775FAF0EE407A07F14803B0EE87
S31508025DD0670A18460CF01FF8FFF71CF9034618461F
S31508025DE0FFF785FAF0EE407A07F14803B0EE670A44
S31508025DF018460CF02EF8FFF70DF903461846FFF77A
S31508025E0095FAF0EE407A07F14803B0EE670A1846AB
S31508025E100CF03DF8FFF7FEF803461846FFF795FA29
S31508025E20F0EE407A07F14803B0EE670A18460CF01E
S31508025E304CF8FFF7EFF803461846FFF7A4FA0246AE
S31508025E4007F14803114618460CF05AF8FFF7E2F82C
S31508025E5003461846FFF7A3FA024607F14803114616
S31508025E6018460CF067F8FFF7D5F803461846FFF709
S31508025E70B1FA024607F14803114618460CF074F8BF
S31508025E80FFF7C8F803461846FFF7B0FA024607F1C5
S31508025E904803114618460CF081F8FFF7BBF803468B
S31508025EA01846FFF7BEFA024607F148031146184696
S31508025EB00CF08EF8FFF7AEF803461846FFF7CCFA51
S31508025EC0024607F14803114618460CF09BF8FFF7FD
S31508025ED0A1F803461846FFF7DAFA024607F148031D
S31508025EE0114618460CF0A8F8FFF794F80346184628
S31508025EF0FFF7D9FA024607F14803114618460CF08D
S31508025F00B5F83A1D07F14803114618460CF044FB4A
S31508025F100CF04CFE04463B1D18460CF071FA054679
S31508025F203B1D18460CF078FA03461A4629462046BF
S31508025F300EF02CF800BF8837BD46B0BDB0B594B098
S31508025F4000AF5C4BD3F8F430002B09DA5A4800F05C
S31508025F5067F907F14803062118460CF0FEF85DE0DA
S31508025F60544BD3F8F43003F08043002B09D053483E
S31508025F7000F056F907F14803052118460CF0EDF82A
S31508025F804CE04C4BD3F8F43003F00053002B09D005
S31508025F904B4800F045F907F14803042118460CF06E
S31508025FA0DCF83BE0434BD3F8F43003F08053002B84
S31508025FB009D0444800F034F907F14803032118468A
S31508025FC00CF0CBF82AE03B4BD3F8F43003F000632D
S31508025FD0002B09D03C4800F023F907F148030221B7
S31508025FE018460CF0BAF819E0324BD3F8F43003F03D
S31508025FF08063002B09D0354800F012F907F14803EF
S31508026000012118460CF0A9F808E0314800F008F911
S3150802601007F14803002118460CF09FF8254BD3F8E0
S31508026020F430244A43F40003C2F8F43029480CF049
S3150802603004FE03461B0ADAB207F14803114618465C
S315080260400CF0A6F823480CF0F8FD0346DAB207F17D
S315080260504803114618460CF0B6F81F4B9A7807F112
S315080260604803114618460CF0C9F81B4BDA7807F1B3
S315080260704803114618460CF0DCF83A1D07F14803A6
S31508026080114618460CF01EFC0CF074FD04463B1D26
S3150802609018460CF0B5F905463B1D18460CF0BCF936
S315080260A003461A46294620460DF070FF00BF5037B0
S315080260B0BD46B0BD000C02446C93030888930308DE
S315080260C0A4930308C0930308E0930308F89303080C
S315080260D010940308F05F0008E0BF1F0880B582B07D
S315080260E000AF0346FB71FB1D0122194603480BF05C
S315080260F03DFB00BF0837BD4680BD00BFEC550020FA
S3150802610080B584B000AF78600023FB730023BB73AD
S3150802611024480BF00FFB034683F00103DBB2002B86
S3150802612019D00DE07B689847BB7B1846FBF750FEF3
S315080261300023BB73FB7B0133FB73FB7B3F2B2CD802
S3150802614007F10E030122194616480BF04AFB0346CD
S31508026150002BE7D122E0144809F02AFB0346202B3C
S315080261600DD1114B0122A3F85C200F4B0122A3F893
S315080261705E2001220D490C4808F010FF0EE00A4B7A
S31508026180B3F85C20084BB3F85E309BB29A4205D04E
S31508026190FDF71CFFFDF726FF00E000BF00BF103722
S315080261A0BD4680BDEC550020205400203C560020F8
S315080261B080B582B000AF78600B467B807A884FF450
S315080261C07A737968034808F04AFE012318460837A5
S315080261D0BD4680BD2054002080B500AF4022064946
S315080261E006480BF01DFAFEF715FF034680211846EE
S315080261F0FFF782F900BF80BDFC550020EC55002050
S3150802620080B500AFFFF7E8FF01220349034808F00B
S31508026210C5FE00BF80BD00BF3C56002020540020AA
S315080262200FB480B582B000AF4FF4807200211548D2
S315080262300FF062F84FF48072002113480FF05CF8F1
S3150802624007F114033B603A6839690F480FF03AF8C8
S3150802625078600D4A0D490B480EF0BAFF0948FAF75D
S3150802626017F803469BB219460648FFF7A1FF0346ED
S315080262707B607B6818460837BD46BDE8804004B097
S31508026280704700BF44560020445700202C94030848
S3150802629080B582B000AF78607B681B68094A934272
S315080262A00CD1094B1B781846FFF718FF064B00223C
S315080262B01A7001220449054808F070FE00BF083723
S315080262C0BD4680BD003801403C56002020540020BF
S315080262D080B582B000AF7860786809F07EFA034626
S315080262E0074A13607B681B68064A934203D1FDF787
S315080262F06DFEFDF777FE00BF0837BD4680BD00BFBD
S3150802630040560020003801400D488546FFF76AF9D5
S315080263100C480D490D4A002302E0D458C4500433F0
S31508026320C4188C42F9D30A4A0A4C002301E01360C6
S315080263300432A242FBD30FF059F8FDF76DFEFEE7D1
S3150802634000000A20000000208407002090A303080A
S3150802635084070020F45F0020FEE7000080B500AF46
S31508026360032000F012F902F071FC02460B4B1B6A7D
S3150802637003F00F030A49CB5C22FA03F3094A1360B6
S315080263800F20FEF7E9FC0346002B01D0012302E0A9
S31508026390FEF762FB0023184680BD00BF000C0244CC
S315080263A0E09E03089405002080B400AF064B1B78D4
S315080263B01A46064B1B681344044A136000BFBD46BF
S315080263C05DF8047B704700BF9C05002044580020F6
S315080263D080B400AF034B1B681846BD465DF8047BC4
S315080263E0704700BF4458002080B485B000AF78607B
S315080263F07B6803F00703FB600C4BDB68BB60BA687B
S315080264004FF6FF031340BB60FB681A02BB681343CF
S3150802641043F0BF6343F40033BB60044ABB68D360EE
S3150802642000BF1437BD465DF8047B704700ED00E0F7
S3150802643080B400AF044BDB681B0A03F00703184657
S31508026440BD465DF8047B704700ED00E080B483B07A
S3150802645000AF0346FB80B7F90630002B0BDBFB883F
S3150802646003F01F020749B7F906305B09012000FA53
S3150802647002F241F8232000BF0C37BD465DF8047BC3
S31508026480704700BF00E100E080B483B000AF034666
S31508026490FB80B7F90630002B12DBFB8803F01F02DC
S315080264A00A49B7F906305B09012000FA02F22033DD
S315080264B041F82320BFF34F8F00BFBFF36F8F00BF92
S315080264C000BF0C37BD465DF8047B704700E100E06B
S315080264D080B483B000AF03463960FB80B7F9063053
S315080264E0002B0ADB3B68DAB20C49B7F9063012010F
S315080264F0D2B20B4483F800230AE03B68DAB20849B1
S31508026500FB8803F00F03043B1201D2B20B441A763E
S3150802651000BF0C37BD465DF8047B704700E100E01A
S3150802652000ED00E080B489B000AFF860B9607A6027
S31508026530FB6803F00703FB61FB69C3F10703042B3E
S3150802654028BF0423BB61FB690433062B02D9FB6906
S31508026550033B00E000237B614FF0FF32BB6902FA7E
S3150802656003F3DA43BB681A407B699A404FF0FF315E
S315080265707B6901FA03F3D9437B680B401343184638
S315080265802437BD465DF8047B704780B582B000AFFC
S3150802659078607868FFF728FF00BF0837BD4680BDD8
S315080265A080B586B000AF0346B9607A60FB81FFF713
S315080265B03FFF78617A68B9687869FFF7B3FF0246E0
S315080265C0B7F90E3011461846FFF782FF00BF183793
S315080265D0BD4680BD80B582B000AF0346FB80B7F9E1
S315080265E006301846FFF732FF00BF0837BD4680BDA2
S315080265F080B582B000AF0346FB80B7F9063018466D
S31508026600FFF742FF00BF0837BD4680BD80B584B09C
S3150802661000AF7860FFF7DCFEF8607B68002B01D1DB
S3150802662001236BE07B6893F85430DBB2022B08D067
S315080266307B6820229A657B68002283F84C20012316
S315080266405CE07B681B685A697B681B6842F0040237
S315080266505A617B68052283F8542020E0FFF7B8FECA
S315080266600246FB68D31A052B19D97B689B6D43F042
S3150802667010027B689A657B68032283F854207B683C
S315080266801B6D03F08003002B03D07B685B6F01222E
S315080266901A737B68002283F84C2001232EE07B685C
S315080266A01B681B6903F40053002BD7D07B681B6851
S315080266B05A697B681B6842F002025A617B680422A7
S315080266C083F854207B681B684FF4FE42DA607B68C5
S315080266D0012283F854207B681B6D03F08003002B8C
S315080266E007D07B685B6F01221A737B681B680022DE
S315080266F09A647B68002283F84C20002318461037D8
S31508026700BD4680BD80B483B000AF78607B68002B3D
S3150802671001D1012319E07B6893F85430DBB2022BCE
S3150802672004D07B6820229A6501230EE07B68042246
S3150802673083F854207B681B685B697A68126843F49D
S31508026740005343F004035361002318460C37BD4631
S315080267505DF8047B7047000080B584B000AF7860AE
S315080267607B68002B01D1012347E17B6893F85C30F3
S31508026770DBB2002B06D17B68002283F85D2078689D
S31508026780FEF772F97B681B689A697B681B6822F0B8
S3150802679010029A61FFF71CFEF86012E0FFF718FE76
S315080267A00246FB68D31A0A2B0BD97B681B6E43F089
S315080267B001027B681A667B68032283F85C20012340
S315080267C01BE17B681B689B6903F00803082BE5D06D
S315080267D07B681B689A697B681B6842F001029A61AA
S315080267E0FFF7F6FDF86012E0FFF7F2FD0246FB68D6
S315080267F0D31A0A2B0BD97B681B6E43F001027B68FE
S315080268001A667B68032283F85C200123F5E07B681D
S315080268101B689B6903F00103002BE5D07B681B68A4
S315080268209A697B681B6842F002029A617B681B6858
S31508026830744A934203D1744A7B685B6813607B6827
S315080268401B7C012B08D17B681B689A697B681B68CD
S3150802685022F040029A6107E07B681B689A697B68A6
S315080268601B6842F040029A617B685B7C012B08D167
S315080268707B681B689A697B681B6842F480429A6146
S3150802688007E07B681B689A697B681B6822F480426A
S315080268909A617B689B7C012B08D17B681B689A6985
S315080268A07B681B6822F480529A6107E07B681B6842
S315080268B09A697B681B6842F480529A617B681B68F6
S315080268C09B6923F440717B689A687B681B680A4354
S315080268D09A617B681B689A697B681B6822F0A40226
S315080268E09A617B681B681A697B681B6822F010022A
S315080268F01A617B68DB68012B08D17B681B689A6979
S315080269007B681B6842F004029A612CE07B68DB68AC
S31508026910002B28D07B68DB68022B1CD07B681B689F
S315080269209A697B681B6842F080029A617B681B68D9
S315080269301A697B681B6842F010021A617B68DB6879
S31508026940032B10D17B681B689A697B681B6842F027
S3150802695020029A6107E07B681B689A697B681B6854
S3150802696042F020029A617B689B69013B5A067B6862
S31508026970DB69013B1B021A437B681B6A013B42EA3D
S3150802698003017B685B69013B1A047B681B680A433F
S31508026990DA617B689B68B3F5407F15D17B689B6A91
S315080269A05A1E7B68DB6A013B1B021A437B681B6B18
S315080269B0013B1B0142EA03017B685B6A013B1A043D
S315080269C07B681B680A43DA607B681B68D3F8C010C9
S315080269D07B68DA6B7B681B680A43C3F8C020786851
S315080269E000F0C8FC7B6800229A657B6800221A665A
S315080269F07B68012283F85C20002318461037BD46BF
S31508026A0080BD00BF00A4004000A5004080B487B046
S31508026A1000AF786039607B6893F85C30FB75FB7D64
S31508026A20012B02D0FB7D022B3DD13B681B68002B54
S31508026A3019D13B689B689A073B68DB68DB061A43F1
S31508026A403B681B691B041A433B685B6913433B613A
S31508026A507B681A6C3B685B689B001344BB60BB6827
S31508026A603A691A601DE03B68DB685A073B681B698E
S31508026A7013433B613B689B689A073B685B69134310
S31508026A80FB607B685A6C3B685B68DB001344BB603F
S31508026A90BB683A691A60BB680433BB60BB68FA68AC
S31508026AA01A60002306E07B681B6E43F002027B68CD
S31508026AB01A66012318461C37BD465DF8047B7047E3
S31508026AC080B485B000AFF860B9607A603B60FB6855
S31508026AD093F85C30DBB2012B16D1FB681B68D3F83E
S31508026AE0803023F03F01BB681A017B689B001A437A
S31508026AF03B685B001A43BB691A43FB681B680A4377
S31508026B00C3F88020002306E0FB681B6E43F00402EC
S31508026B10FB681A66012318461437BD465DF8047BDE
S31508026B20704780B483B000AF78607B6893F85C30B6
S31508026B30DBB2012B10D17B68022283F85C207B68CA
S31508026B401B689A697B681B6822F001029A617B6856
S31508026B5000221A66002306E07B681B6E43F00402D5
S31508026B607B681A66012318460C37BD465DF8047B16
S31508026B70704780B586B000AFF860B9607A60FB6886
S31508026B8093F85C30DBB2022B2CD1FB681B68D3F876
S31508026B90C43003F40013002B07D0FB681B6E43F4C2
S31508026BA00072FB681A66012323E0FB681B68D3F8A8
S31508026BB0C4301B0C03F003037B617B697A68B968EE
S31508026BC0F86800F039FCFB681B6801217A6901FA4A
S31508026BD002F2C3F8CC2001227B699A40FB689A65C7
S31508026BE0002306E0FB681B6E43F00802FB681A6680
S31508026BF0012318461837BD4680BD80B483B000AF5E
S31508026C0078607B689B6D18460C37BD465DF8047B39
S31508026C107047000080B48BB000AFF860B9607A6044
S31508026C203B600023FB61FB6893F85C30FB76FB7ED6
S31508026C30022B40F0E880BB68402B37D1FB681B6803
S31508026C40D3F8903003F00F03002B07D1FB681B6EB5
S31508026C5043F48072FB681A660123DBE0FB681B6853
S31508026C60D3F890301B0E03F00103012B0AD1FB68FF
S31508026C701B68D3F880305B0A03F00103012B01D1AC
S31508026C800123FB61FB681B68D3F890301B0A03F0EB
S31508026C900303FA691344FB61FB68996CFA691346A4
S31508026CA0DB001344DB000B447B6236E0FB681B689F
S31508026CB0D3F8983003F00F03002B07D1FB681B6E3D
S31508026CC043F48072FB681A660123A3E0FB681B681B
S31508026CD0D3F898301B0E03F00103012B0AD1FB6887
S31508026CE01B68D3F880301B0A03F00103012B01D17C
S31508026CF00123FB61FB681B68D3F898301B0A03F073
S31508026D000303FA691344FB61FB68D96CFA691346F3
S31508026D10DB001344DB000B447B627B6A1B6803F0CF
S31508026D2080427B685A607B685B68002B07D17B6A66
S31508026D301B689B0CC3F30A027B681A6005E07B6A30
S31508026D401B6823F060427B681A607B6A1B6803F043
S31508026D5000527B689A607B6A1B6803F000427B6874
S31508026D601A617B6A04337B627B6A1B689AB27B6808
S31508026D70DA617B6A1B681B0C03F00F027B68DA6018
S31508026D807B6A1B6803F480127B685A617B6A1B68FC
S31508026D9003F400127B689A617B6A1B681B0E03F078
S31508026DA07F027B681A627B6A1B68DA0F7B685A6203
S31508026DB07B6A04337B627B6A7B6100233B620AE05F
S31508026DC07A693B6A1A4439683B6A0B4412781A7024
S31508026DD03B6A01333B627B68DB68114AD35C1A461D
S31508026DE03B6A9342ECD3BB68402B05D1FB681B6810
S31508026DF0FA69C3F8942004E0FB681B68FA69C3F8C9
S31508026E009C20002306E0FB681B6E43F00802FB6821
S31508026E101A66012318462C37BD465DF8047B70476F
S31508026E20F89E030880B483B000AF786039607B6847
S31508026E301B68D3F8C8203B681340002B01D10023F6
S31508026E4000E0012318460C37BD465DF8047B7047FF
S31508026E5080B485B000AF786039603B68402B07D1B3
S31508026E607B681B68D3F8903003F00F03FB6006E0DB
S31508026E707B681B68D3F8983003F00F03FB60FB6846
S31508026E8018461437BD465DF8047B704780B487B050
S31508026E9000AFF860B9607A60FB6893F85C30FB75FE
S31508026EA0FB7D012B03D0FB7D022B40F0C880FB68DB
S31508026EB01B689B6D3B61BB6803F00703002B04D07C
S31508026EC03B6903F00103002B3BD0BB6803F0380390
S31508026ED0002B04D03B6903F00203002B31D0BB68B8
S31508026EE003F4E073002B04D03B6903F00403002B80
S31508026EF027D0BB6803F4F053002B04D03B6903F098
S31508026F000803002B1DD0BB6803F46043002B04D092
S31508026F103B6903F01003002B13D0BB6803F440331C
S31508026F20002B04D03B6903F02003002B09D0BB6871
S31508026F3003F47C03002B0CD03B6903F04003002BBF
S31508026F4007D1FB681B68DA6DFB681B6842F0010211
S31508026F50DA65BB6803F00703002B04D03B6903F02C
S31508026F600103002B3BD1BB6803F03803002B04D086
S31508026F703B6903F00203002B31D1BB6803F4E073CB
S31508026F80002B04D03B6903F00403002B27D1BB680E
S31508026F9003F4F053002B04D03B6903F00803002BDB
S31508026FA01DD1BB6803F46043002B04D03B6903F090
S31508026FB01003002B13D1BB6803F44033002B04D013
S31508026FC03B6903F02003002B09D1BB6803F47C0359
S31508026FD0002B0CD03B6903F04003002B07D0FB685B
S31508026FE01B68DA6DFB681B6842F00202DA65BB6849
S31508026FF003F08003002B09D0FB681B68D3F8DC106A
S31508027000FB681B687A680A43C3F8DC20BB6803F48A
S315080270108073002B09D0FB681B68D3F8E010FB6865
S315080270201B687A680A43C3F8E020FB681B68596D37
S31508027030FB681B68BA680A435A65002306E0FB68C0
S315080270401B6E43F00202FB681A66012318461C37B8
S31508027050BD465DF8047B704780B58CB000AF78609A
S315080270607B681B681B6D03F4E053FB627B681B6835
S315080270705B6DFA6A1340FB627B681B681B6D03F043
S315080270800703BB627B681B685B6DBA6A1340BB6207
S315080270907B681B681B6D03F038037B627B681B6881
S315080270A05B6D7A6A13407B627B681B681B6D03F40F
S315080270B071033B627B681B685B6D3A6A13403B62ED
S315080270C07B681B681B6D03F46023FB617B681B6886
S315080270D05B6DFA691340FB617B681B685B6DBB617C
S315080270E07B681B681B6D7B617B6903F04003002B81
S315080270F00BD0BB6903F04003002B06D07B681B68E4
S3150802710040221A65786800F016F97B6903F48073E1
S31508027110002B19D0BB6903F48073002B14D07B684B
S315080271201B68D3F8D8303B617B681B68D3F8E0301C
S315080271303A6913403B617B681B684FF480721A6593
S315080271403969786800F0D8F8FB6A002B07D07B68A3
S315080271501B68FA6A1A65F96A786800F0A2F8BB6AC7
S31508027160002B07D07B681B68BA6A1A65B96A786801
S31508027170FDF7D0FA7B6A002B07D07B681B687A6A10
S315080271801A65796A786800F097F87B6903F40073E0
S31508027190002B0CD0BB6903F40073002B07D07B6865
S315080271A01B684FF400721A65786800F090F87B69DC
S315080271B003F08003002B18D0BB6903F08003002B71
S315080271C013D07B681B68D3F8D430FB607B681B68D6
S315080271D0D3F8DC30FA681340FB607B681B688022B0
S315080271E01A65F968786800F07CF87B6903F400533D
S315080271F0002B0CD0BB6903F40053002B07D07B6825
S315080272001B684FF400521A65786800F080F87B69AB
S3150802721003F40043002B0CD0BB6903F40043002B94
S3150802722007D07B681B684FF400421A65786800F03D
S3150802723078F87B6903F48043002B0FD0BB6903F40B
S315080272408043002B0AD07B681B684FF480421A657C
S315080272507B681B6E43F080027B681A66FB69002B0B
S3150802726007D07B681B68FA691A65F969786800F0BD
S3150802727076F83B6A002B09D07B681B683A6A1A655E
S315080272807B681A6E3B6A1A437B681A667B681B6EB2
S31508027290002B02D0786800F058F800BF3037BD4698
S315080272A080BD80B483B000AF7860396000BF0C3708
S315080272B0BD465DF8047B704780B483B000AF786042
S315080272C0396000BF0C37BD465DF8047B704780B451
S315080272D083B000AF786000BF0C37BD465DF8047B0B
S315080272E0704780B483B000AF7860396000BF0C374E
S315080272F0BD465DF8047B704780B483B000AF786002
S31508027300396000BF0C37BD465DF8047B704780B410
S3150802731083B000AF786000BF0C37BD465DF8047BCA
S31508027320704780B483B000AF786000BF0C37BD46A3
S315080273305DF8047B704780B483B000AF786000BF05
S315080273400C37BD465DF8047B704780B483B000AF46
S31508027350786000BF0C37BD465DF8047B704780B481
S3150802736083B000AF7860396000BF0C37BD465DF860
S31508027370047B704780B485B000AF78602C4BBB6045
S315080273807B681B682B4A934203D1BB6803F5547387
S31508027390BB607B68BA681A647B681B68D3F880305E
S315080273A023F4F8117B685B6B1A047B681B680A4333
S315080273B0C3F88020BB6803F170027B685A647B6855
S315080273C01B68D3F8803023F070617B689B6B1A06C2
S315080273D07B681B680A43C3F88020BB6803F1B002C6
S315080273E07B689A64BB6803F5C4727B68DA64BB6817
S315080273F003F518727B681A65BB6803F51E727B680B
S315080274005A65BB68FB6005E0FB6800221A60FB68E8
S315080274100433FB60BB6803F55473FA689A42F3D3E4
S3150802742000BF00BF1437BD465DF8047B704700BF36
S3150802743000AC004000A8004080B489B000AFF860F4
S31508027440B9607A603B60BB685B68002B0AD1BB688F
S315080274501A69BB689B681A43BB681B689B0413437B
S31508027460FB610AE0BB681A69BB689B681A43BB687A
S315080274701B68134343F08043FB61BB681B6A1A0609
S31508027480BB68DB691A43BB689B691A43BB685B69BD
S315080274901A43BB68DB681B0413433B61FB68596DDF
S315080274A03A681346DB001344DB000B44BB61BB6935
S315080274B0FA691A60BB690433BB61BB693A691A6027
S315080274C0BB690433BB6100237B6120E07B6903331C
S315080274D07A6813441B781A067B69023379680B4467
S315080274E01B781B041A437B69013379680B441B78A2
S315080274F01B02134379687A690A4412781A43BB69EC
S315080275001A60BB690433BB617B6904337B61BB6860
S31508027510DB68064AD35C1A467B699342D6D300BF18
S3150802752000BF2437BD465DF8047B7047F89E030802
S3150802753080B588B000AFF860B9607A60324B1B78C4
S31508027540012B01D102235AE02F4B01221A702E4B2E
S3150802755000225A604FF47A7000F0A4F80346FB77CB
S31508027560FB7F002B47D1284AFB689360274BBB61F8
S31508027570FB6823F00043022B04D17968B86800F04F
S31508027580DFF81BE0FB68224A934203D0FB68214AD4
S31508027590934204D17968B86800F00EF90EE0FB68E8
S315080275A023F000431C4A934204D17968B86800F074
S315080275B04FF903E07968B86800F04AF94FF47A702F
S315080275C000F070F80346FB77BB691A68FB6823F07C
S315080275D0304323F00403DB431A40BB691A60FB6895
S315080275E00C4A934207D10D4B7B617B691B6823F0DA
S315080275F004027B691A60044B00221A70FB7F184644
S315080276002037BD4680BD00BFA005002028200240C5
S31508027610020000100600001002000040402002404E
S3150802762080B483B000AF0023FB710D4B9B6A03F055
S315080276300103002B0DD00A4B0A4A5A60084B0A4A24
S315080276405A60074B9B6A03F00103002B01D0012302
S31508027650FB71FB7918460C37BD465DF8047B70470B
S315080276600020024023016745AB89EFCD80B483B081
S3150802767000AF0023FB710A4B9B6A094A43F00103D8
S315080276809362074B9B6A03F00103002B01D1012386
S31508027690FB71FB7918460C37BD465DF8047B7047CB
S315080276A00020024080B586B000AF7860FEF790FEF3
S315080276B07861204B3B6110E07B68B3F1FF3F0CD049
S315080276C0FEF786FE02467B69D31A7A689A4202D385
S315080276D07B68002B01D1032327E03B691B6803F073
S315080276E00B03002BE8D1144BFB603B691B6803F4C0
S315080276F07E03BB60BB68002B0CD0104B5A68BB6874
S3150802770013430E4A5360BB6803F47E02FB681A6091
S3150802771001230AE03B691B6803F48033002B03D07C
S31508027720FB684FF480321A60002318461837BD46A4
S3150802773080BD00BF2020024030200240A005002064
S3150802774080B48BB000AF78603960042387F827309D
S315080277507B683B623B68FB61164BBB61BB691B6876
S3150802776043F00202BB691A60EFF310833B613B697F
S315080277707B6172B600BFFB691A683B6A1A603B6A8C
S3150802778004333B62FB690433FB6197F82730013BFC
S3150802779087F8273097F82730002BECD17B69FB60F6
S315080277A0FB6883F3108800BF00BF2C37BD465DF81F
S315080277B0047B70472820024080B48BB000AF786003
S315080277C03960042387F827307B683B623B68FB6194
S315080277D01C4BBB611C4B7B61BB691B6843F00202F5
S315080277E0BB691A607B691A68184B9B6803F0040325
S315080277F01A437B691A60EFF31083FB60FB683B61EF
S3150802780072B600BFFB691A683B6A1A603B6A0433A0
S315080278103B62FB690433FB6197F82730013B87F823
S31508027820273097F82730002BECD13B69BB60BB6841
S3150802783083F3108800BF00BF2C37BD465DF8047B72
S31508027840704700BF2820024040200240A0050020C1
S3150802785080B485B000AF78603960094BFB60FB687D
S315080278601B6843F00202FB681A603A687B68128852
S3150802787092B21A8000BF1437BD465DF8047B704782
S315080278802820024080B586B000AF786039603A4B4E
S315080278901B78012B01D102236AE0374B01221A70A9
S315080278A0354B00225A604FF47A70FFF7FBFE034607
S315080278B0FB75FB7D002B57D17B681B682E4A9360AC
S315080278C02E4BFB607B681B6823F0004348F20802D4
S315080278D093420BD17B685B68184600F053F84FF465
S315080278E07A70FFF7DFFE0346FB7533E07B681B6899
S315080278F0234A934208D100F0B5F84FF47A70FFF79D
S31508027900D1FE0346FB7525E03B684FF0FF321A604D
S315080279107B689B683B6115E07B685B68194638693A
S3150802792000F068F84FF47A70FFF7BCFE0346FB7561
S31508027930FB7D002B03D03B683A691A600AE03B6973
S3150802794001333B617B68DA687B689B6813443A6952
S315080279509A42E1D3FB681A687B681B6823F00043E6
S31508027960DB431A40FB681A60034B00221A70FB7D40
S3150802797018461837BD4680BDA005002028200240BB
S315080279800800008080B485B000AF7860184BFB60B1
S315080279907B6803F00303032B08D1FB681B6843F4D7
S315080279A0004343F02003FA6813601BE07B6803F088
S315080279B00103002B09D0FB681B6823F0004323F060
S315080279C0280343F02802FB681A607B6803F0020367
S315080279D0002B07D0FB681B6843F0004343F02803DB
S315080279E0FA68136000BF1437BD465DF8047B70471A
S315080279F02820024080B485B000AF78603960184B01
S31508027A00FB603B6803F00103002B11D0FB681B687F
S31508027A1023F0004323F4FE53FA681360FB681A68DE
S31508027A207B689B01134343F02402FB681A6010E04B
S31508027A30FB681B6823F4FE52FB681A60FB681A6827
S31508027A407B689B01134343F0004343F02403FA681F
S31508027A50136000BF1437BD465DF8047B704700BF4C
S31508027A602820024080B483B000AF074B7B607B6856
S31508027A701B6843F008027B681A6000BF0C37BD46D4
S31508027A805DF8047B704700BF4020024080B487B08F
S31508027A9000AF7860396000233B6136E13B681A68BB
S31508027AA001213B6901FA03F31340FB60FB68002BD3
S31508027AB000F028813B685B68022B03D03B685B6851
S31508027AC0122B25D13B69DA087B68083253F8223033
S31508027AD07B613B6903F007039B000F2202FA03F35B
S31508027AE0DB437A6913407B613B681B6903F00F022B
S31508027AF03B6903F007039B0002FA03F37A6913430F
S31508027B007B613B69DA087B680832796943F8221097
S31508027B107B681B687B613B695B00032202FA03F3FD
S31508027B20DB437A6913407B613B685B6803F00302B7
S31508027B303B695B0002FA03F37A6913437B617B684C
S31508027B407A691A603B685B68012B0BD03B685B68F5
S31508027B50022B07D03B685B68112B03D03B685B6836
S31508027B60122B30D17B689B687B613B695B000322E1
S31508027B7002FA03F3DB437A6913407B613B68DA68EE
S31508027B803B695B0002FA03F37A6913437B617B68FC
S31508027B907A699A607B685B687B6101223B6902FAB3
S31508027BA003F3DB437A6913407B613B685B681B0915
S31508027BB003F001023B6902FA03F37A6913437B6114
S31508027BC07B687A695A603B685B68032B17D07B68C7
S31508027BD0DB687B613B695B00032202FA03F3DB4342
S31508027BE07A6913407B613B689A683B695B0002FAD3
S31508027BF003F37A6913437B617B687A69DA603B68C7
S31508027C005B6803F08053002B7CD0474A3B699B088C
S31508027C10183352F823307B613B6903F00303DB0018
S31508027C200F2202FA03F3DB437A6913407B617B680E
S31508027C309A0A3E4B13403A6902F00302D200934075
S31508027C407A6913437B6138493B699B0818337A6919
S31508027C5041F82320344B1B687B61FB68DB437A6956
S31508027C6013407B613B685B6803F48013002B03D0E7
S31508027C707A69FB6813437B612B4A7B6913602A4B3B
S31508027C805B687B61FB68DB437A6913407B613B680F
S31508027C905B6803F40013002B03D07A69FB6813436D
S31508027CA07B61214A7B6953601F4BD3F884307B6121
S31508027CB0FB68DB437A6913407B613B685B6803F4C4
S31508027CC00033002B03D07A69FB6813437B61164A9B
S31508027CD07B69C2F88430144BD3F880307B61FB6829
S31508027CE0DB437A6913407B613B685B6803F4803344
S31508027CF0002B03D07A69FB6813437B610A4A7B69C6
S31508027D00C2F880303B6901333B613B681A683B69BC
S31508027D1022FA03F3002B7FF4C1AE00BF00BF1C3763
S31508027D20BD465DF8047B7047002002447F7F2F0022
S31508027D3080B487B000AF7860396000237B61A0E029
S31508027D4001227B6902FA03F33A6813403B613B69F5
S31508027D50002B00F09380524A7B699B08183352F82D
S31508027D602330FB607B6903F00303DB000F2202FA70
S31508027D7003F3FA681340FB607B689A0A494B13407F
S31508027D807A6902F00302D2009340FA689A4236D11F
S31508027D90434BD3F880203B69DB4341491340C1F882
S31508027DA080303F4BD3F884203B69DB433C49134080
S31508027DB0C1F884303A4B1A683B69DB4338491340A9
S31508027DC00B60374B5A683B69DB43354913404B60B6
S31508027DD07B6903F00303DB000F2202FA03F3FB605D
S31508027DE02F4A7B699B08183352F82310FB68DA433B
S31508027DF02B487B699B080A40183340F823207B6886
S31508027E001A687B695B00032101FA03F31A437B684C
S31508027E101A607B69DA087B68083253F822107B6994
S31508027E2003F007039B000F2202FA03F3DB437A6986
S31508027E30D20819407B68083243F822107B689A6890
S31508027E407B695B00032101FA03F3DB431A407B6873
S31508027E509A607B685A6801217B6901FA03F3DB435E
S31508027E601A407B685A607B68DA687B695B00032183
S31508027E7001FA03F3DB431A407B68DA607B69013354
S31508027E807B613A687B6922FA03F3002B7FF458AFC9
S31508027E9000BF00BF1C37BD465DF8047B704700BFB4
S31508027EA0002002447F7F2F0080B485B000AF78603F
S31508027EB00B467B807B681A697B881340002B02D0AD
S31508027EC00123FB7301E00023FB73FB7B184614377F
S31508027ED0BD465DF8047B704780B483B000AF786016
S31508027EE00B467B8013467B707B78002B03D07A88FF
S31508027EF07B689A6102E07A887B689A6200BF0C37CF
S31508027F00BD465DF8047B704780B485B000AF7860E3
S31508027F100B467B807B685B69FB607A88FB6813404B
S31508027F201A04FB68D9437B880B401A437B689A611B
S31508027F3000BF1437BD465DF8047B704780B584B030
S31508027F4000AF78607B68002B01D1012370E0786866
S31508027F5000F072F87B681B684CF6CC421A607B68A4
S31508027F601B6845F255521A607B681B687A68526824
S31508027F705A607B681B687A6892689A60FEF728FAE4
S31508027F80F8600FE0FEF724FA0246FB68D31A212BA3
S31508027F9008D97B681B68DB6803F00203002B01D053
S31508027FA0032345E07B681B68DB6803F00203002BAA
S31508027FB0E8D17B681B69002B05D17B681B684FF4E7
S31508027FC080425A6106E07B681A697B681B6842F43C
S31508027FD040425A61FEF7FCF9F8600FE0FEF7F8F93D
S31508027FE00246FB68D31A212B08D97B681B68DB6813
S31508027FF003F00F03002B01D0032319E07B681B68EB
S31508028000DB6803F00F03002BE8D17B681B681A694B
S315080280107B68DB689A4205D07B681B687A68D268F7
S315080280201A6104E07B681B684AF6AA221A600023D2
S3150802803018461037BD4680BD80B483B000AF78605D
S3150802804000BF0C37BD465DF8047B704780B483B029
S3150802805000AF78607B681B684AF6AA221A6000237A
S3150802806018460C37BD465DF8047B704780B588B064
S3150802807000AF78607B68002B02D1012300F028BC90
S31508028080944BDB6903F01803FB61924B9B6A03F07E
S315080280900303BB617B681B6803F01003002B5BD0EC
S315080280A0FB69082B05D0FB69182B14D1BB69022B77
S315080280B011D17B68DB69002B02D1012300F008BCD1
S315080280C0844B9B6923F47C127B681B6A1B048149D7
S315080280D013438B6140E07B68DB69002B23D07D4B21
S315080280E01B687C4A43F480731360FEF771F9786162
S315080280F008E0FEF76DF902467B69D31A022B01D90D
S315080281000323E5E3734B1B6803F40073002BF0D0DB
S31508028110704B9B6923F47C127B681B6A1B046D49AE
S3150802812013438B6118E06B4B1B686A4A23F480730E
S315080281301360FEF74DF9786108E0FEF749F9024641
S315080281407B69D31A022B01D90323C1E3614B1B684E
S3150802815003F40073002BF0D17B681B6803F001035C
S31508028160002B00F0A080FB69102B05D0FB69182BA9
S3150802817009D1BB69032B06D17B685B68002B40F0EB
S3150802818092800123A4E37B685B68B3F5803F06D13E
S31508028190504B1B684F4A43F48033136058E07B68A0
S315080281A05B68002B12D14B4B1B684A4A23F4803377
S315080281B01360484B1B68474A23F480131360454BE8
S315080281C01B68444A23F48023136041E07B685B689A
S315080281D0B3F5A02F12D13F4B1B683E4A43F48023C6
S315080281E013603C4B1B683B4A23F480131360394BDC
S315080281F01B68384A43F48033136029E07B685B685E
S31508028200B3F5A81F12D1334B1B68324A43F48023B5
S315080282101360304B1B682F4A43F4801313602D4BAF
S315080282201B682C4A43F48033136011E0294B1B6800
S31508028230284A23F480331360264B1B68254A23F405
S3150802824080231360234B1B68224A23F4801313608E
S315080282507B685B68002B13D0FEF7BAF8786108E0F2
S31508028260FEF7B6F802467B69D31A642B01D90323B3
S315080282702EE3184B1B6803F40033002BF0D012E0F0
S31508028280FEF7A6F8786108E0FEF7A2F802467B69CF
S31508028290D31A642B01D903231AE30E4B1B6803F482
S315080282A00033002BF0D17B681B6803F00203002B16
S315080282B000F09A80FB69002B05D0FB69182B49D17F
S315080282C0BB69012B46D17B68DB68002B04D10123ED
S315080282D0FEE200BF000C0244FB69002B1CD19A4B3C
S315080282E01B6803F018027B681B699A4214D0964BE6
S315080282F01B6823F018027B681B69934913430B60BA
S3150802830000F0D0FD914B1B681846FCF725FD034685
S31508028310002B01D00123DBE2FEF75AF8786108E068
S31508028320FEF756F802467B69D31A022B01D90323B4
S31508028330CEE2854B1B6803F00203002BF0D0824B7A
S315080283401B6923F4FE027B685B691B047E4913439F
S315080283500B6149E07B68DB68002B2CD07A4B1B68E3
S3150802836023F018027B681B69774913430B60764B27
S315080283701B68754A43F001031360FEF729F8786112
S3150802838008E0FEF725F802467B69D31A022B01D9C3
S3150802839003239DE26C4B1B6803F00203002BF0D00B
S315080283A0694B1B6923F4FE027B685B691B046649F9
S315080283B013430B6118E0644B1B68634A23F00103FD
S315080283C01360FEF705F8786108E0FEF701F8024641
S315080283D07B69D31A022B01D9032379E25A4B1B680C
S315080283E003F00203002BF0D17B681B6803F0080335
S315080283F0002B3CD07B689B69002B1CD0524BD3F8D0
S31508028400F030514A43F08063C2F8F030FDF7E0FFDE
S31508028410786108E0FDF7DCFF02467B69D31A022B76
S3150802842001D9032354E2484BD3F8F03003F0006332
S31508028430002BEFD01BE0444BD3F8F030424A23F02E
S315080284408063C2F8F030FDF7C3FF786108E0FDF7F4
S31508028450BFFF02467B69D31A022B01D9032337E2EF
S31508028460394BD3F8F03003F00063002BEFD17B6869
S315080284701B6803F00403002B00F0D280344B5B6ABE
S3150802848003F00103002B18D1314B5B6A304A43F0E3
S3150802849001035362FDF79CFF786108E0FDF798FF38
S315080284A002467B69D31A022B01D9032310E2284B11
S315080284B05B6A03F00103002BF0D07B689B68012BF3
S315080284C008D1214BD3F8F0301F4A43F00103C2F812
S315080284D0F03074E07B689B68002B18D11A4BD3F8EE
S315080284E0F030194A23F00103C2F8F030164BD3F8DC
S315080284F0F030154A23F08003C2F8F030124BD3F855
S31508028500F030114A23F00403C2F8F03057E07B68D2
S315080285109B68052B1ED10C4BD3F8F0300A4A43F060
S315080285200403C2F8F030084BD3F8F030064A23F0B9
S315080285308003C2F8F030044BD3F8F030024A43F015
S315080285400103C2F8F0303AE0000C02449805002014
S31508028550000802447B689B68852B18D1A24BD3F886
S31508028560F030A14A43F00403C2F8F0309E4BD3F828
S31508028570F0309D4A43F08003C2F8F0309A4BD3F8A4
S31508028580F030994A43F00103C2F8F03017E0964BEF
S31508028590D3F8F030944A23F00103C2F8F030924B34
S315080285A0D3F8F030904A23F00403C2F8F0308E4B29
S315080285B0D3F8F0308C4A23F08003C2F8F0307B6897
S315080285C09B68002B16D0FDF703FF78610AE0FDF7DA
S315080285D0FFFE02467B69D31A41F28832934201D9D9
S315080285E0032375E1804BD3F8F03003F00203002B26
S315080285F0EDD015E0FDF7ECFE78610AE0FDF7E8FE3E
S3150802860002467B69D31A41F28832934201D903237F
S315080286105EE1754BD3F8F03003F00203002BEDD17F
S315080286207B681B6803F02003002B36D07B685B6AE5
S31508028630002B19D06C4B1B686B4A43F480531360AA
S31508028640FDF7C6FE786108E0FDF7C2FE02467B69C1
S31508028650D31A022B01D903233AE1634B1B6803F4AD
S315080286600053002BF0D018E05F4B1B685E4A23F4D8
S3150802867080531360FDF7ACFE786108E0FDF7A8FEAB
S3150802868002467B69D31A022B01D9032320E1564BF2
S315080286901B6803F40053002BF0D17B689B6A002BFE
S315080286A000F01581FB69182B00F0AF807B689B6A86
S315080286B0022B40F086804C4B1B684B4A23F0807392
S315080286C01360FDF785FE786108E0FDF781FE024634
S315080286D07B69D31A022B01D90323F9E0424B1B68A3
S315080286E003F00073002BF0D13F4B9B6A23F47C53B3
S315080286F023F003037A68D16A7A68126B12020A4374
S31508028700394913438B627B685B6B013BC3F30802EF
S315080287107B689B6B013B5B029BB21A437B68DB6BF4
S31508028720013B1B0403F4FE031A437B681B6C013BE3
S315080287301B0603F0FE432C4913434B632A4B9B6AE1
S31508028740294A23F0100393627B68DB6C264ADB0016
S315080287509363254B9B6A244A43F010039362224B88
S315080287609B6A23F00C027B685B6C1F4913438B627E
S315080287701D4B9B6A23F020027B689B6C1A491343A4
S315080287808B62194B9B6A184A43F480339362164BE1
S315080287901B68154A43F080731360FDF719FE78616A
S315080287A008E0FDF715FE02467B69D31A022B01D9AA
S315080287B003238DE00C4B1B6803F00073002BF0D0EB
S315080287C085E0094B1B68084A23F080731360FDF79E
S315080287D0FFFD78610AE0FDF7FBFD02467B69D31AC5
S315080287E0022B03D9032373E0000C02443A4B1B689D
S315080287F003F00073002BEED1374B9B6A364A23F4FB
S31508028800E02323F00303936261E0334B9B6A3B61E7
S31508028810314B5B6BFB607B689B6A012B31D03B69F2
S3150802882003F003027B68DB6A9A422AD13B691B0A78
S3150802883003F03F027B681B6B9A4222D1FB68C3F3A3
S3150802884008027B685B6B013B9A421AD1FB685B0A9A
S3150802885003F07F027B689B6B013B9A4211D1FB684E
S315080288601B0C03F07F027B68DB6B013B9A4208D143
S31508028870FB681B0E03F07F027B681B6C013B9A4266
S3150802888001D0012324E0144B9B6BDB08C3F30C02D3
S315080288907B68DB6C9A421AD00F4B9B6A0E4A23F00E
S315080288A010039362FDF794FD786100BFFDF790FD12
S315080288B002467B699342F9D07B68DB6C064ADB0089
S315080288C09363054B9B6A044A43F0100393620023A1
S315080288D018462037BD4680BD000C024480B584B0D8
S315080288E000AF786039607B68002B01D101239EE1D5
S315080288F0834B1B6803F00F033A689A4210D9804BE0
S315080289001B6823F00F027E493B6813430B607C4BBE
S315080289101B6803F00F033A689A4201D0012386E1E5
S315080289207B681B6803F01003002B12D07B685A6918
S31508028930744B1B6A1B0A03F070039A4209D9714BDE
S315080289401B6A23F4E0427B685B691B026D49134389
S315080289500B627B681B6803F00803002B12D07B6846
S315080289601A69684B1B6A1B0903F070039A4209D9F4
S31508028970644B1B6A23F4E0627B681B691B0161492D
S3150802898013430B627B681B6803F00403002B10D0A9
S315080289907B68DA685B4B1B6A03F070039A4208D954
S315080289A0584B1B6A23F070027B68DB6855491343F0
S315080289B00B627B681B6803F00203002B10D07B68EE
S315080289C09A68504B1B6A03F00F039A4208D94D4B1B
S315080289D01B6A23F00F027B689B684A4913430B62A2
S315080289E07B681B6803F00103002B00F093807B6809
S315080289F05B68032B07D1434B1B6803F00073002BFC
S31508028A0021D1012313E17B685B68022B07D13D4B19
S31508028A101B6803F40033002B15D1012307E17B6899
S31508028A205B68012B07D1374B1B6803F40073002BD5
S31508028A3009D10123FBE0334B1B6803F00203002B29
S31508028A4001D10123F3E02F4BDB6923F003027B6894
S31508028A505B682C491343CB61FDF7BAFCF8607B6867
S31508028A605B68032B12D10AE0FDF7B2FC0246FB68EB
S31508028A70D31A41F28832934201D90323D7E0214B14
S31508028A80DB6903F01803182BEED143E07B685B68B9
S31508028A90022B12D10AE0FDF79BFC0246FB68D31AA9
S31508028AA041F28832934201D90323C0E0154BDB69B0
S31508028AB003F01803102BEED12CE07B685B68012BC0
S31508028AC022D10AE0FDF784FC0246FB68D31A41F27A
S31508028AD08832934201D90323A9E00A4BDB6903F0E2
S31508028AE01803082BEED115E0FDF772FC0246FB6867
S31508028AF0D31A41F28832934206D9032397E000BF7C
S31508028B0000200240000C02444B4BDB6903F01803B9
S31508028B10002BE9D17B681B6803F00203002B10D0F7
S31508028B207B689A68444B1B6A03F00F039A4208D281
S31508028B30414B1B6A23F00F027B689B683E4913432D
S31508028B400B623E4B1B6803F00F033A689A4210D237
S31508028B503A4B1B6823F00F0238493B6813430B60F4
S31508028B60364B1B6803F00F033A689A4201D0012379
S31508028B705DE07B681B6803F00403002B10D07B685A
S31508028B80DA682D4B1B6A03F070039A4208D22A4B05
S31508028B901B6A23F070027B68DB68274913430B6262
S31508028BA07B681B6803F00803002B12D07B681A69DE
S31508028BB0214B1B6A1B0903F070039A4209D21E4B0A
S31508028BC01B6A23F4E0627B681B691B011A4913437B
S31508028BD00B627B681B6803F01003002B12D07B68BC
S31508028BE05A69154B1B6A1B0A03F070039A4209D28B
S31508028BF0114B1B6A23F4E0427B685B691B020E4930
S31508028C0013430B6200F022F802460B4B1B6A03F071
S31508028C100F030B49CB5C22FA03F30A4A13600A4B89
S31508028C201B681846FCF798F80346FB72FB7A184647
S31508028C301037BD4680BD00BF000C0244002002402A
S31508028C40E09E0308940500209805002080B489B0A8
S31508028C5000AF8C4BDB6903F01803082B02D18A4B51
S31508028C60FB6107E1874BDB6903F01803002B12D17E
S31508028C70844B1B6803F02003002B09D0814B1B6829
S31508028C80DB0803F00303814A22FA03F3FB61F1E0EE
S31508028C907E4BFB61EEE07B4BDB6903F01803102B7E
S31508028CA002D17B4BFB61E5E0764BDB6903F01803E7
S31508028CB0182B40F0DD80734B9B6A03F003037B613C
S31508028CC0704B9B6A1B0A03F03F033B616D4B9B6A21
S31508028CD01B0903F00103FB606A4B9B6BDB08C3F3BA
S31508028CE00C03FA6802FB03F307EE903AF8EE677A8A
S31508028CF0C7ED027A3B69002B00F0B7807B69012B2E
S31508028D0003D07B69032B56D077E05E4B1B6803F0D2
S31508028D102003002B2DD05B4B1B68DB0803F00303F3
S31508028D205A4A22FA03F37B607B6807EE903AF8EE1A
S31508028D30676A3B6907EE903AF8EE677A86EEA77A93
S31508028D40504B5B6BC3F3080307EE903AF8EE676A7B
S31508028D5097ED026ADFED4F5AC6EE257A76EEA77AC6
S31508028D60F7EE006A77EEA67A67EE277AC7ED067AF5
S31508028D7065E03B6907EE903AF8EE677ADFED466AF8
S31508028D8086EEA77A3F4B5B6BC3F3080307EE903A6E
S31508028D90F8EE676A97ED026ADFED3E5AC6EE257A65
S31508028DA076EEA77AF7EE006A77EEA67A67EE277A64
S31508028DB0C7ED067A43E03B6907EE903AF8EE677A22
S31508028DC0DFED366A86EEA77A2E4B5B6BC3F3080392
S31508028DD007EE903AF8EE676A97ED026ADFED2D5ACA
S31508028DE0C6EE257A76EEA77AF7EE006A77EEA67AC7
S31508028DF067EE277AC7ED067A21E03B6907EE903AD5
S31508028E00F8EE677ADFED266A86EEA77A1D4B5B6B6C
S31508028E10C3F3080307EE903AF8EE676A97ED026A1B
S31508028E20DFED1C5AC6EE257A76EEA77AF7EE006AC9
S31508028E3077EEA67A67EE277AC7ED067A00BF114B58
S31508028E405B6B5B0A03F07F0301333B603B6807EE0B
S31508028E50903AB8EE677AD7ED066AC6EE877AFCEEDE
S31508028E60E77A17EE903AFB6104E00023FB6101E022
S31508028E70064BFB61FB6918462437BD465DF8047B41
S31508028E80704700BF000C024400093D000090D00361
S31508028E90001BB700000000460024744C001B374B29
S31508028EA00024744A80B500AFFFF7D0FE0246084B8D
S31508028EB01B6A03F00F030749CB5C03F01F0322FA70
S31508028EC003F3054A1360044B1B68184680BD00BFAE
S31508028ED0000C0244E09E03089405002080B500AF0A
S31508028EE0FFF7E0FF0246064B1B6A1B0903F007035E
S31508028EF00449CB5C03F01F0322FA03F3184680BD2C
S31508028F00000C0244F09E030880B500AFFFF7CAFFC3
S31508028F100246064B1B6A1B0A03F007030449CB5C8D
S31508028F2003F01F0322FA03F3184680BD000C02441D
S31508028F30F09E030880B500AFFFF7B4FF0246064B62
S31508028F401B6A1B0B03F007030449CB5C03F01F03E0
S31508028F5022FA03F3184680BD000C0244F09E030869
S31508028F6080B485B000AF786039607B681F221A60CA
S31508028F70154BDB6903F003027B685A60124B1B6AC6
S31508028F80FB60FB6803F00F027B689A60FB6803F0DC
S31508028F9070027B68DA60FB681B0903F070027B6863
S31508028FA01A61FB681B0A03F070027B685A61074B59
S31508028FB01B6803F00F023B681A6000BF1437BD46F0
S31508028FC05DF8047B704700BF000C02440020024093
S31508028FD02DE9B04FD8B000AFC7F84C01002387F887
S31508028FE05B31002387F85A31D7F84C31D3E900238D
S31508028FF002F08074002554EA05030BD0CD4BD3F852
S31508029000E83023F04041D7F84C319B6DC94A0B43EF
S31508029010C2F8E830D7F84C31D3E9002302F0010848
S315080290204FF0000958EA090342D0D7F84C31DB6DF4
S31508029030052B23D801A252F823F000BF8590020817
S3150802904055900208699002088590020885900208E0
S3150802905085900208D7F84C310833184604F0DAFE30
S31508029060034687F85B310EE0D7F84C3130331846A1
S3150802907004F068FF034687F85B3104E0012387F8AA
S315080290805B3100E000BF97F85B31002B0CD1A94B8E
S31508029090D3F8D83023F00701D7F84C31DB6DA54A4F
S315080290A00B43C2F8D83003E097F85B3187F85A3198
S315080290B0D7F84C31D3E9002302F0020A4FF0000B2D
S315080290C05AEA0B0300F08880D7F84C311B6E282B1E
S315080290D068D801A252F823F0AD910208A5910208B8
S315080290E0A5910208A5910208A5910208A591020870
S315080290F0A5910208A59102087D910208A591020888
S31508029100A5910208A5910208A5910208A59102084F
S31508029110A5910208A591020891910208A591020853
S31508029120A5910208A5910208A5910208A59102082F
S31508029130A5910208A5910208AD910208A591020817
S31508029140A5910208A5910208A5910208A59102080F
S31508029150A5910208A5910208AD910208A5910208F7
S31508029160A5910208A5910208A5910208A5910208EF
S31508029170A5910208A5910208AD910208D7F84C31CB
S315080291800833184604F046FE034687F85B310EE0BC
S31508029190D7F84C313033184604F0D4FE034687F824
S315080291A05B3104E0012387F85B3100E000BF97F8E2
S315080291B05B31002B0CD15F4BD3F8D83023F0380142
S315080291C0D7F84C311B6E5B4A0B43C2F8D83003E022
S315080291D097F85B3187F85A31D7F84C31D3E900232F
S315080291E002F00403C7F840310023C7F84431D7E92F
S315080291F050120B4613434ED0D7F84C315B6EB3F57B
S31508029200A07F2CD0B3F5A07F25D8B3F5807F28D0D0
S31508029210B3F5807F1FD8C02B25D0C02B1BD8802B37
S315080292200FD0802B17D8002B1FD0402B13D1D7F87D
S315080292304C310833184604F0EDFD034687F85B31D6
S3150802924014E0D7F84C313033184604F07BFE034657
S3150802925087F85B310AE0012387F85B3106E000BF35
S3150802926004E000BF02E000BF00E000BF97F85B31F0
S31508029270002B0CD12F4BD3F8D83023F4E071D7F852
S315080292804C315B6E2B4A0B43C2F8D83003E097F891
S315080292905B3187F85A31D7F84C31D3E9002302F00B
S315080292A00803C7F838310023C7F83C31D7E94E120C
S315080292B00B46134356D0D7F84C319B6EB3F5206F45
S315080292C031D0B3F5206F2AD8B3F5006F2DD0B3F598
S315080292D0006F24D8B3F5C06F29D0B3F5C06F1ED876
S315080292E0B3F5806F11D0B3F5806F18D8002B23D051
S315080292F0B3F5007F13D1D7F84C310833184604F07A
S3150802930089FD034687F85B3117E0D7F84C313033CD
S31508029310184604F017FE034687F85B310DE0012371
S3150802932087F85B3109E000BF07E000BF05E000BF30
S3150802933003E000BF000C024400BF97F85B31002B24
S315080293400CD1BB4BD3F8D83023F46061D7F84C3133
S315080293509B6EB74A0B43C2F8D83003E097F85B31E5
S3150802936087F85A31D7F84C31D3E9002302F01003B3
S31508029370C7F830310023C7F83431D7E94C120B4607
S31508029380134353D0D7F84C31DB6EB3F5A04F31D027
S31508029390B3F5A04F2AD8B3F5804F2DD0B3F5804F39
S315080293A024D8B3F5405F29D0B3F5405F1ED8B3F58C
S315080293B0005F11D0B3F5005F18D8002B20D0B3F5A3
S315080293C0805F13D1D7F84C310833184604F022FDD2
S315080293D0034687F85B3114E0D7F84C313033184628
S315080293E004F0B0FD034687F85B310AE0012387F8EB
S315080293F05B3106E000BF04E000BF02E000BF00E008
S3150802940000BF97F85B31002B0CD1894BD3F8D830C3
S3150802941023F4E041D7F84C31DB6E854A0B43C2F898
S31508029420D83003E097F85B3187F85A31D7F84C31D0
S31508029430D3E9002302F02003C7F828310023C7F82E
S315080294402C31D7E94A120B46134353D0D7F84C317D
S315080294501B6FB3F5203F31D0B3F5203F2AD8B3F5B9
S31508029460003F2DD0B3F5003F24D8B3F5C03F29D02D
S31508029470B3F5C03F1ED8B3F5803F11D0B3F5803F90
S3150802948018D8002B20D0B3F5004F13D1D7F84C319A
S315080294900833184604F0BEFC034687F85B3114E02D
S315080294A0D7F84C313033184604F04CFD034687F89A
S315080294B05B310AE0012387F85B3106E000BF04E06E
S315080294C000BF02E000BF00E000BF97F85B31002B47
S315080294D00CD1574BD3F8D83023F46031D7F84C3136
S315080294E01B6F534A0B43C2F8D83003E097F85B3137
S315080294F087F85A31D7F84C31D3E9002302F04003F2
S31508029500C7F820310023C7F82431D7E948120B4699
S31508029510134353D0D7F84C315B6FB3F5A01F31D044
S31508029520B3F5A01F2AD8B3F5801F2DD0B3F5801F37
S3150802953024D8B3F5402F29D0B3F5402F1ED8B3F55A
S31508029540002F11D0B3F5002F18D8002B20D0B3F571
S31508029550802F13D1D7F84C310833184604F05AFC39
S31508029560034687F85B3114E0D7F84C313033184696
S3150802957004F0E8FC034687F85B310AE0012387F822
S315080295805B3106E000BF04E000BF02E000BF00E076
S3150802959000BF97F85B31002B0CD1254BD3F8D83096
S315080295A023F4E011D7F84C315B6F214A0B43C2F81A
S315080295B0D83003E097F85B3187F85A31D7F84C313F
S315080295C0D3E9002302F08003C7F818310023C7F84D
S315080295D01C31D7E946120B46134355D0D7F84C31FE
S315080295E09B6FB3F5200F33D0B3F5200F2CD8B3F504
S315080295F0000F2FD0B3F5000F26D8B3F5C00F2BD026
S31508029600B3F5C00F20D8B3F5800F13D0B3F5800F8A
S315080296101AD8002B22D0B3F5001F15D1D7F84C3132
S315080296200833184604F0F6FB034687F85B3116E062
S31508029630000C0244D7F84C313033184604F082FC49
S31508029640034687F85B310AE0012387F85B3106E0B7
S3150802965000BF04E000BF02E000BF00E000BF97F8C9
S315080296605B31002B0CD1BB4BD3F8D83023F4600105
S31508029670D7F84C319B6FB74A0B43C2F8D83003E090
S3150802968097F85B3187F85A31D7F84C31D3E900237A
S3150802969002F48073C7F810310023C7F81431D7E9EA
S315080296A044120B46134353D0D7F84C31DB6FB3F150
S315080296B0A06F31D0B3F1A06F2AD8B3F1806F2DD045
S315080296C0B3F1806F24D8B3F1407F29D0B3F1407F3C
S315080296D01ED8B3F1007F11D0B3F1007F18D8002B42
S315080296E020D0B3F1807F13D1D7F84C31083318460E
S315080296F004F090FB034687F85B3114E0D7F84C3147
S315080297003033184604F01EFC034687F85B310AE03C
S31508029710012387F85B3106E000BF04E000BF02E0E0
S3150802972000BF00E000BF97F85B31002B0CD1894BD4
S31508029730D3F8D83023F0E061D7F84C31DB6F854A8D
S315080297400B43C2F8D83003E097F85B3187F85A31F1
S31508029750D7F84C31D3E9002302F40073C7F808316D
S315080297600023C7F80C31D7E942120B46134355D0EA
S31508029770D7F84C31D3F88030B3F1205F31D0B3F14A
S31508029780205F2AD8B3F1005F2DD0B3F1005F24D849
S31508029790B3F1C05F29D0B3F1C05F1ED8B3F1805FC1
S315080297A011D0B3F1805F18D8002B20D0B3F1006F27
S315080297B013D1D7F84C310833184604F02BFB03466D
S315080297C087F85B3114E0D7F84C313033184604F089
S315080297D0B9FB034687F85B310AE0012387F85B3158
S315080297E006E000BF04E000BF02E000BF00E000BFE1
S315080297F097F85B31002B0DD1564BD3F8D83023F0AE
S315080298006051D7F84C31D3F88030524A0B43C2F82C
S31508029810D83003E097F85B3187F85A31D7F84C31DC
S31508029820D3E9002302F48063C7F800310023C7F89E
S315080298300431D7E940120B46134344D0D7F84C31CA
S31508029840D3F88430052B23D801A252F823F000BF9F
S3150802985099980208699802087D9802089998020858
S315080298609998020899980208D7F84C31083318468D
S3150802987004F0D0FA034687F85B310EE0D7F84C318C
S315080298803033184604F05EFB034687F85B3104E082
S31508029890012387F85B3100E000BF97F85B31002BA4
S315080298A00DD12C4BD3F8DC3023F00701D7F84C3115
S315080298B0D3F88430274A0B43C2F8DC3003E097F822
S315080298C05B3187F85A31D7F84C31D3E9002302F4D1
S315080298D00063C7F8F8300023C7F8FC30D7E93E1210
S315080298E00B4613434FD0D7F84C31D3F88830502B58
S315080298F029D0502B23D8402B27D0402B1FD8302BCA
S3150802990025D0302B1BD8202B0FD0202B17D8002B75
S3150802991022D0102B13D1D7F84C310833184604F04D
S3150802992079FA034687F85B3117E0D7F84C313033BA
S31508029930184604F007FB034687F85B310DE001235E
S3150802994087F85B3109E000BF07E000BF05E000BF0A
S3150802995003E000BF000C024400BF97F85B31002BFE
S315080299600DD1AF4BD3F8DC3023F07001D7F84C3168
S31508029970D3F88830AA4A0B43C2F8DC3003E097F8DA
S315080299805B3187F85A31D7F84C31D3E9002302F410
S315080299908053C7F8F0300023C7F8F430D7E93C12F1
S315080299A00B46134355D0D7F84C31D3F88C30B3F164
S315080299B0A06F31D0B3F1A06F2AD8B3F1806F2DD042
S315080299C0B3F1806F24D8B3F1407F29D0B3F1407F39
S315080299D01ED8B3F1007F11D0B3F1007F18D8002B3F
S315080299E020D0B3F1807F13D1D7F84C31083318460B
S315080299F004F010FA034687F85B3114E0D7F84C31C5
S31508029A003033184604F09EFA034687F85B310AE0BB
S31508029A10012387F85B3106E000BF04E000BF02E0DD
S31508029A2000BF00E000BF97F85B31002B0DD17C4BDD
S31508029A30D3F8E03023F0E061D7F84C31D3F88C3014
S31508029A40774A0B43C2F8E03003E097F85B3187F8B0
S31508029A505A31D7F84C31D3E9002302F40053C7F838
S31508029A60E8300023C7F8EC30D7E93A120B4613431D
S31508029A703DD0D7F84C31D3F89030B3F5403F1BD0E0
S31508029A80B3F5403F14D8B3F5003F17D0B3F5003FFE
S31508029A900ED8002B14D0B3F5803F09D1D7F84C3134
S31508029AA03033184604F04EFA034687F85B3108E06D
S31508029AB0012387F85B3104E000BF02E000BF00E043
S31508029AC000BF97F85B31002B0DD1554BD3F8E43024
S31508029AD023F44031D7F84C31D3F89030504A0B432F
S31508029AE0C2F8E43003E097F85B3187F85A31D7F8C1
S31508029AF04C31D3E9002302F48043C7F8E03000234F
S31508029B00C7F8E430D7E938120B4613433DD0D7F8E5
S31508029B104C31D3F89430B3F5402F1BD0B3F5402F10
S31508029B2014D8B3F5002F17D0B3F5002F0ED8002B93
S31508029B3014D0B3F5802F09D1D7F84C3130331846F3
S31508029B4004F000FA034687F85B3108E0012387F838
S31508029B505B3104E000BF02E000BF00E000BF97F8F7
S31508029B605B31002B0DD12E4BD3F8E43023F4402180
S31508029B70D7F84C31D3F89430294A0B43C2F8E4306B
S31508029B8003E097F85B3187F85A31D7F84C31D3E9B5
S31508029B90002302F40043C7F8D8300023C7F8DC30A4
S31508029BA0D7E936120B46134340D0D7F84C31D3F8CF
S31508029BB09830B3F5401F1BD0B3F5401F14D8B3F540
S31508029BC0001F17D0B3F5001F0ED8002B14D0B3F51B
S31508029BD0801F09D1D7F84C313033184604F0B2F950
S31508029BE0034687F85B3108E0012387F85B3104E016
S31508029BF000BF02E000BF00E000BF97F85B31002B10
S31508029C0010D1074BD3F8E43023F44011D7F84C317E
S31508029C10D3F89830024A0B43C2F8E43006E000BF94
S31508029C20000C024497F85B3187F85A31D7F84C3161
S31508029C30D3E900230021C7F8D01003F48063C7F8DC
S31508029C40D430D7E934120B4613433DD0D7F84C31FA
S31508029C50D3F89C30B3F5400F1BD0B3F5400F14D898
S31508029C60B3F5000F17D0B3F5000F0ED8002B14D09A
S31508029C70B3F5800F09D1D7F84C313033184604F0C2
S31508029C8061F9034687F85B3108E0012387F85B31FF
S31508029C9004E000BF02E000BF00E000BF97F85B31B6
S31508029CA0002B0DD1BE4BD3F8E43023F44001D7F88C
S31508029CB04C31D3F89C30BA4A0B43C2F8E43003E07D
S31508029CC097F85B3187F85A31D7F84C31D3E9002334
S31508029CD002F48033C7F8C8300023C7F8CC30D7E976
S31508029CE032120B46134335D0D7F84C31D3F8A0308D
S31508029CF0B3F1007F15D0B3F1007F0ED8002B12D036
S31508029D00B3F1807F09D1D7F84C313033184604F0C5
S31508029D1019F9034687F85B3106E0012387F85B31B8
S31508029D2002E000BF00E000BF97F85B31002B0DD1BF
S31508029D309B4BD3F8E43023F04071D7F84C31D3F873
S31508029D40A030974A0B43C2F8E43003E097F85B3138
S31508029D5087F85A31D7F84C31D3E900230021C7F8DE
S31508029D60C01003F40063C7F8C430D7E930120B46B3
S31508029D7013430ED08A4BDB69894A23F40043D36125
S31508029D80874BD969D7F84C31D3F80431844A0B4347
S31508029D90D361D7F84C31D3E9002302F40033C7F86C
S31508029DA0B8300023C7F8BC30D7E92E120B46134346
S31508029DB055D0D7F84C31D3F8A430B3F5A06F31D0CB
S31508029DC0B3F5A06F2AD8B3F5806F2DD0B3F5806F9F
S31508029DD024D8B3F5407F29D0B3F5407F1ED8B3F512
S31508029DE0007F11D0B3F5007F18D8002B20D0B3F529
S31508029DF0807F13D1D7F84C310833184604F00AF895
S31508029E00034687F85B3114E0D7F84C3130331846ED
S31508029E1004F098F8034687F85B310AE0012387F8CD
S31508029E205B3106E000BF04E000BF02E000BF00E0CD
S31508029E3000BF97F85B31002B0DD1594BD3F8DC30B4
S31508029E4023F4E061D7F84C31D3F8A430544A0B43D3
S31508029E50C2F8DC3003E097F85B3187F85A31D7F855
S31508029E604C31D3E9002302F48023C7F8B03000232B
S31508029E70C7F8B430D7E92C120B46134355D0D7F896
S31508029E804C31D3F8A830B3F5A04F31D0B3F5A04F73
S31508029E902AD8B3F5804F2DD0B3F5804F24D8B3F521
S31508029EA0405F29D0B3F5405F1ED8B3F5005F11D0E5
S31508029EB0B3F5005F18D8002B20D0B3F5805F13D115
S31508029EC0D7F84C310833184603F0A4FF034687F83F
S31508029ED05B3114E0D7F84C313033184604F032F8C7
S31508029EE0034687F85B310AE0012387F85B3106E00F
S31508029EF000BF04E000BF02E000BF00E000BF97F821
S31508029F005B31002B0DD1264BD3F8DC3023F4E0412C
S31508029F10D7F84C31D3F8A830214A0B43C2F8DC30C3
S31508029F2003E097F85B3187F85A31D7F84C31D3E911
S31508029F3000230021C7F8A81003F02003C7F8AC30A5
S31508029F40D7E92A120B46134357D0D7F84C31D3F820
S31508029F50AC30B3F5A02F33D0B3F5A02F2CD8B3F578
S31508029F60802F2FD0B3F5802F26D8B3F5403F2BD0BC
S31508029F70B3F5403F20D8B3F5003F13D0B3F5003F01
S31508029F801AD8002B22D0B3F5803F15D1D7F84C3119
S31508029F900833184603F03EFF034687F85B3116E09E
S31508029FA0000C0244D7F84C313033184603F0CAFF86
S31508029FB0034687F85B310AE0012387F85B3106E03E
S31508029FC000BF04E000BF02E000BF00E000BF97F850
S31508029FD05B31002B0DD1BB4BD3F8DC3023F4E021E7
S31508029FE0D7F84C31D3F8AC30B64A0B43C2F8DC305A
S31508029FF003E097F85B3187F85A31D7F84C31D3E941
S3150802A00000230021C7F8A01003F04003C7F8A430C4
S3150802A010D7E928120B46134355D0D7F84C31D3F853
S3150802A020B030B3F5A00F31D0B3F5A00F2AD8B3F5E7
S3150802A030800F2DD0B3F5800F24D8B3F5401F29D051
S3150802A040B3F5401F1ED8B3F5001F11D0B3F5001F94
S3150802A05018D8002B20D0B3F5801F13D1D7F84C316E
S3150802A0600833184603F0D6FE034687F85B3114E038
S3150802A070D7F84C313033184603F064FF034687F8A5
S3150802A0805B310AE0012387F85B3106E000BF04E092
S3150802A09000BF02E000BF00E000BF97F85B31002B6B
S3150802A0A00DD1884BD3F8DC3023F4E001D7F84C31D4
S3150802A0B0D3F8B030834A0B43C2F8DC3003E097F892
S3150802A0C05B3187F85A31D7F84C31D3E9002300219E
S3150802A0D0C7F8981003F08003C7F89C30D7E9261210
S3150802A0E00B46134355D0D7F84C31D3F8B430B3F1F5
S3150802A0F0A06F31D0B3F1A06F2AD8B3F1806F2DD0FB
S3150802A100B3F1806F24D8B3F1407F29D0B3F1407FF1
S3150802A1101ED8B3F1007F11D0B3F1007F18D8002BF7
S3150802A12020D0B3F1807F13D1D7F84C3108331846C3
S3150802A13003F070FE034687F85B3114E0D7F84C311A
S3150802A1403033184603F0FEFE034687F85B310AE011
S3150802A150012387F85B3106E000BF04E000BF02E096
S3150802A16000BF00E000BF97F85B31002B0DD1554BBD
S3150802A170D3F8DC3023F0E061D7F84C31D3F8B430A9
S3150802A180504A0B43C2F8DC3003E097F85B3187F894
S3150802A1905A31D7F84C31D3E900230021C7F8901079
S3150802A1A003F48073C7F89430D7E924120B46134395
S3150802A1B055D0D7F84C31D3F8B830B3F1A04F31D0D7
S3150802A1C0B3F1A04F2AD8B3F1804F2DD0B3F1804F07
S3150802A1D024D8B3F1405F29D0B3F1405F1ED8B3F15A
S3150802A1E0005F11D0B3F1005F18D8002B20D0B3F16D
S3150802A1F0805F13D1D7F84C310833184603F00AFEAC
S3150802A200034687F85B3114E0D7F84C3130331846E9
S3150802A21003F098FE034687F85B310AE0012387F8C4
S3150802A2205B3106E000BF04E000BF02E000BF00E0C9
S3150802A23000BF97F85B31002B0DD1224BD3F8DC30E7
S3150802A24023F0E041D7F84C31D3F8B8301D4A0B4316
S3150802A250C2F8DC3003E097F85B3187F85A31D7F851
S3150802A2604C31D3E9002302F40023C7F888300023CF
S3150802A270C7F88C30D7E922120B46134355D0D7F8C4
S3150802A2804C31D3F8C030B3F5802F35D0B3F5802FD3
S3150802A2902ED8B3F5403F31D0B3F5403F28D8B3F5B1
S3150802A2A0003F1BD0B3F5003F22D8002B03D0B3F5ED
S3150802A2B0803F09D01CE0034B9B6A024A43F40033F1
S3150802A2C093621CE0000C0244D7F84C310833184656
S3150802A2D003F0A0FD034687F85B3110E0D7F84C314E
S3150802A2E03033184603F02EFE034687F85B3106E044
S3150802A2F0012387F85B3102E000BF00E000BF97F850
S3150802A3005B31002B0DD1C34BD3F8E83023F4E0219F
S3150802A310D7F84C31D3F8C030BE4A0B43C2F8E830FE
S3150802A32003E097F85B3187F85A31D7F84C31D3E90D
S3150802A330002302F48013C7F880300023C7F884305C
S3150802A340D7E920120B46134351D0D7F84C31D3F82C
S3150802A350C430B3F5001F33D0B3F5001F2CD8B3F5BC
S3150802A360C01F2DD0B3F5C01F26D8B3F5801F19D04C
S3150802A370B3F5801F20D8002B03D0B3F5002F07D0E2
S3150802A3801AE0A44B9B6AA34A43F40033936218E08B
S3150802A390D7F84C310833184603F03CFD034687F8D4
S3150802A3A05B310EE0D7F84C313033184603F0CAFD5C
S3150802A3B0034687F85B3104E0012387F85B3100E046
S3150802A3C000BF97F85B31002B0DD1924BD3F8E830DA
S3150802A3D023F46011D7F84C31D3F8C4308D4A0B43B5
S3150802A3E0C2F8E83003E097F85B3187F85A31D7F8B4
S3150802A3F04C31D3E9002302F40013BB670023FB6741
S3150802A400D7E91E120B46134332D0D7F84C31D3F88C
S3150802A410D430052B0FD8032B11D2012B11D9022BBD
S3150802A42009D1D7F84C310833184603F0F3FC034632
S3150802A43087F85B3106E0012387F85B3102E000BF4B
S3150802A44000E000BF97F85B31002B0DD1714BD3F8B2
S3150802A450E83023F00701D7F84C31D3F8D4306D4AE7
S3150802A4600B43C2F8E83003E097F85B3187F85A31B4
S3150802A470D7F84C31D3E900230021396703F4007376
S3150802A4807B67D7E91C120B46134324D0D7F84C3105
S3150802A490D3F8D830002B05D0082B05D0012387F82E
S3150802A4A05B3102E000BF00E000BF97F85B31002B8A
S3150802A4B00DD1584BD3F8E83023F00801D7F84C31C0
S3150802A4C0D3F8D830534A0B43C2F8E83003E097F87A
S3150802A4D05B3187F85A31D7F84C31D3E9002302F0B9
S3150802A4E00073BB660023FB66D7E91A120B461343B1
S3150802A4F000F0B980484B5B6A474A43F0010353624E
S3150802A500FBF766FFC7F854010BE0FBF761FF02464B
S3150802A510D7F85431D31A022B03D9032387F85B31B0
S3150802A52005E03D4B5B6A03F00103002BEDD097F87B
S3150802A5305B31002B40F09380364BD3F8F03003F4AE
S3150802A5404073C7F85C31D7F85C31002B23D0D7F8B3
S3150802A5504C31D3F8F820D7F85C3193421BD02D4BF7
S3150802A560D3F8F03023F44073C7F85C31294BD3F89B
S3150802A570F030284A43F48033C2F8F030254BD3F83A
S3150802A580F030244A23F48033C2F8F030214AD7F84F
S3150802A5905C31C2F8F030D7F85C3103F00103002BC6
S3150802A5A019D0FBF715FFC7F854010DE0FBF710FFAA
S3150802A5B00246D7F85431D21A41F288339A4203D95D
S3150802A5C0032387F85B3106E0124BD3F8F03003F029
S3150802A5D00203002BEAD097F85B31002B3AD1D7F861
S3150802A5E04C31D3F8F83003F44073B3F5407F15D1F4
S3150802A5F0084BDB6923F47C51D7F84C31D3F8F83091
S3150802A6001B0923F07F4323F03003024A0B43D3612D
S3150802A6100AE000BF000C0244000802449F4BDB69B3
S3150802A6209E4A23F47C53D3619C4BD3F8F0309B4A61
S3150802A63023F44073C2F8F030984BD3F8F010D7F8E9
S3150802A6404C31D3F8F830C3F30B03944A0B43C2F8E0
S3150802A650F03008E097F85B3187F85A3103E097F84B
S3150802A6605B3187F85A31D7F84C31D3E9002302F027
S3150802A67080633B6600237B66D7E918120B461343B1
S3150802A68035D0D7F84C31D3F8C830302B14D0302B0C
S3150802A6900ED8202B12D0202B0AD8002B10D0102B24
S3150802A6A006D17E4B9B6A7D4A43F40033936208E0E7
S3150802A6B0012387F85B3104E000BF02E000BF00E037
S3150802A6C000BF97F85B31002B0DD1744BD3F8E830F5
S3150802A6D023F03001D7F84C31D3F8C8306F4A0B4310
S3150802A6E0C2F8E83003E097F85B3187F85A31D7F8B1
S3150802A6F04C31D3E9002302F48003BB650023FB65D2
S3150802A700D7E916120B46134333D0D7F84C31D3F890
S3150802A710CC30002B02D0402B07D010E05F4B9B6A4F
S3150802A7205E4A43F4003393620DE0D7F84C3108339E
S3150802A730184603F06FFB034687F85B3103E00123F3
S3150802A74087F85B3100BF97F85B31002B0DD1534B6D
S3150802A750D3F8E43023F04001D7F84C31D3F8CC30A3
S3150802A7604E4A0B43C2F8E43003E097F85B3187F8A8
S3150802A7705A31D7F84C31D3E9002302F400033B657A
S3150802A78000237B65D7E914120B46134333D0D7F857
S3150802A7904C31D3F8D030002B02D0802B07D010E0F2
S3150802A7A03E4B9B6A3D4A43F4003393620DE0D7F869
S3150802A7B04C310833184603F02DFB034687F85B3104
S3150802A7C003E0012387F85B3100BF97F85B31002B62
S3150802A7D00DD1324BD3F8E43023F08001D7F84C314F
S3150802A7E0D3F8D0302D4A0B43C2F8E43003E097F889
S3150802A7F05B3187F85A31D7F84C31D3E9002302F096
S3150802A8000063BB640023FB64D7E912120B461343A9
S3150802A8104AD0D7F84C31D3F8E030042B27D801A216
S3150802A82052F823F039A8020847A802085BA80208CA
S3150802A83077A8020877A80208184B9B6A174A43F4B6
S3150802A8400033936218E0D7F84C310833184603F000
S3150802A850E1FA034687F85B310EE0D7F84C3130331C
S3150802A860184603F06FFB034687F85B3104E00123C1
S3150802A87087F85B3100E000BF97F85B31002B0FD1F8
S3150802A880064BD3F8E03023F00701D7F84C31D3F85A
S3150802A890E030024A0B43C2F8E03005E0000C0244FD
S3150802A8A097F85B3187F85A31D7F84C31D3E9002348
S3150802A8B002F080533B6400237B64D7E910120B46EF
S3150802A8C0134300F08180D7F84C31D3F8E430202BBB
S3150802A8D05FD801A252F823F05DA9020893A90208DB
S3150802A8E093A9020893A9020893A9020893A9020840
S3150802A8F093A9020893A902086BA9020893A9020858
S3150802A90093A9020893A9020893A9020893A902081F
S3150802A91093A9020893A902087FA9020893A9020823
S3150802A92093A9020893A9020893A9020893A90208FF
S3150802A93093A9020893A902089BA9020893A90208E7
S3150802A94093A9020893A9020893A9020893A90208DF
S3150802A95093A9020893A902089BA90208AB4B9B6A12
S3150802A960AA4A43F40033936218E0D7F84C31083305
S3150802A970184603F04FFA034687F85B310EE0D7F81C
S3150802A9804C313033184603F0DDFA034687F85B315B
S3150802A99004E0012387F85B3100E000BF97F85B31DA
S3150802A9A0002B0DD1994BD3F8E03023F03801D7F8B4
S3150802A9B04C31D3F8E430954A0B43C2F8E03003E051
S3150802A9C097F85B3187F85A31D7F84C31D3E9002327
S3150802A9D002F00053BB630023FB63D7E90E120B4652
S3150802A9E013434ED0D7F84C31D3F8E830B3F5807F0D
S3150802A9F02ED0B3F5807F27D8C02B2BD0C02B23D8D7
S3150802AA00802B17D0802B1FD8002B02D0402B07D0C3
S3150802AA101AE07E4B9B6A7D4A43F4003393621AE03E
S3150802AA20D7F84C310833184603F0F4F9034687F889
S3150802AA305B3110E0D7F84C313033184603F082FA0E
S3150802AA40034687F85B3106E0012387F85B3102E0AB
S3150802AA5000BF00E000BF97F85B31002B0DD16B4BAE
S3150802AA60D3F8E03023F4E071D7F84C31D3F8E83064
S3150802AA70664A0B43C2F8E03003E097F85B3187F881
S3150802AA805A31D7F84C31D3E9002302F080433B63AD
S3150802AA9000237B63D7E90C120B46134355D0D7F82C
S3150802AAA04C31D3F8EC30B3F5206F31D0B3F5206FC3
S3150802AAB02AD8B3F5006F2DD0B3F5006F24D8B3F5B5
S3150802AAC0C06F29D0B3F5C06F1ED8B3F5806F11D009
S3150802AAD0B3F5806F18D8002B20D0B3F5007F13D1B9
S3150802AAE0D7F84C310833184603F094F9034687F829
S3150802AAF05B3114E0D7F84C313033184603F022FAAA
S3150802AB00034687F85B310AE0012387F85B3106E0E2
S3150802AB1000BF04E000BF02E000BF00E000BF97F8F4
S3150802AB205B31002B0DD1394BD3F8E03023F4606149
S3150802AB30D7F84C31D3F8EC30344A0B43C2F8E0303C
S3150802AB4003E097F85B3187F85A31D7F84C31D3E9E5
S3150802AB50002302F00043BB620023FB62D7E90A1214
S3150802AB600B46134358D0D7F84C31D3F8F030B3F527
S3150802AB70A04F31D0B3F5A04F2AD8B3F5804F2DD0C8
S3150802AB80B3F5804F24D8B3F5405F29D0B3F5405FBB
S3150802AB901ED8B3F5005F11D0B3F5005F18D8002BA5
S3150802ABA020D0B3F5805F13D1D7F84C310833184655
S3150802ABB003F030F9034687F85B3114E0D7F84C31D5
S3150802ABC03033184603F0BEF9034687F85B310AE0CC
S3150802ABD0012387F85B3106E000BF04E000BF02E00C
S3150802ABE000BF00E000BF97F85B31002B10D1074B7E
S3150802ABF0D3F8E03023F4E042D7F84C31D3F8F030FA
S3150802AC0002491343C1F8E03006E000BF000C0244D3
S3150802AC1097F85B3187F85A31D7F84C31D3E90023D4
S3150802AC200021396203F001037B62D7E908120B4659
S3150802AC30134355D0D7F84C31D3F8F430B3F5203F47
S3150802AC4031D0B3F5203F2AD8B3F5003F2DD0B3F55E
S3150802AC50003F24D8B3F5C03F29D0B3F5C03F1ED86C
S3150802AC60B3F5803F11D0B3F5803F18D8002B20D01A
S3150802AC70B3F5004F13D1D7F84C310833184603F011
S3150802AC80C9F8034687F85B3114E0D7F84C313033FC
S3150802AC90184603F057F9034687F85B310AE00123A1
S3150802ACA087F85B3106E000BF04E000BF02E000BFA0
S3150802ACB000E000BF97F85B31002B0DD1884BD3F823
S3150802ACC0E03023F46032D7F84C31D3F8F4308449B3
S3150802ACD01343C1F8E03003E097F85B3187F85A313D
S3150802ACE0D7F84C31D3E900230021B96103F00203F6
S3150802ACF0FB61D7E906120B4613433DD0D7F84C3110
S3150802AD00D3F8DC30032B1CD801A252F823F000BF7B
S3150802AD104BAD020821AD02082FAD02084BAD020861
S3150802AD206F4B9B6A6E4A43F4003393620EE0D7F880
S3150802AD304C310833184603F06DF8034687F85B3141
S3150802AD4004E0012387F85B3100E000BF97F85B3126
S3150802AD50002B0DD1624BD3F8E43023F00302D7F867
S3150802AD604C31D3F8DC305E491343C1F8E43003E0D2
S3150802AD7097F85B3187F85A31D7F84C31D3E9002373
S3150802AD800021396103F004037B61D7E904120B46FB
S3150802AD9013433AD0D7F84C31D3F8BC30B3F5007F19
S3150802ADA00ED0B3F5007F15D8002B17D0B3F5807FE8
S3150802ADB010D14B4B9B6A4A4A43F4003393620EE026
S3150802ADC0D7F84C310833184603F024F8034687F8B7
S3150802ADD05B3104E0012387F85B3100E000BF97F896
S3150802ADE05B31002B0DD13E4BD3F8E83023F4407289
S3150802ADF0D7F84C31D3F8BC3039491343C1F8E83097
S3150802AE0003E097F85B3187F85A31D7F84C31D3E922
S3150802AE1000230021B96003F01003FB60D7E9021290
S3150802AE200B46134338D0D7F84C31D3F80031302BC0
S3150802AE301BD0302B15D8102B02D0202B07D010E0B0
S3150802AE40274B9B6A264A43F4003393620EE0D7F8EF
S3150802AE504C313033184603F075F8034687F85B31F0
S3150802AE6004E0012387F85B3100E000BF97F85B3105
S3150802AE70002B0DD11A4BD3F8E43023F03002D7F861
S3150802AE804C31D3F8003116491343C1F8E43003E0D4
S3150802AE9097F85B3187F85A31D7F84C31D3E9002352
S3150802AEA00021396003F008037B60D7E900120B46DC
S3150802AEB013430CD00A4BD3F8E83023F0C002D7F874
S3150802AEC04C31D3F8FC3006491343C1F8E83097F8F9
S3150802AED05A31184607F5B077BD46BDE8B08F00BFB0
S3150802AEE0000C024480B48BB000AF7860AD4B5B6B4C
S3150802AEF0C3F308033B62AB4B9B6A03F00303FB6194
S3150802AF00A84B9B6A1B0A03F03F03BB61A54B9B6ACE
S3150802AF1003F010037B61A34B9B6BDB08C3F30C03A3
S3150802AF207A6902FB03F307EE903AF8EE677AC7ED01
S3150802AF30047ABB69002B00F02681FB69032B53D0E8
S3150802AF40FB69032B6FD8FB69012B03D0FB69022B24
S3150802AF502BD068E0934B1B68DB0803F00303924A85
S3150802AF6022FA03F3FB60FB6807EE903AF8EE676A8B
S3150802AF70BB6907EE903AF8EE677A86EEA77A3B6ADD
S3150802AF8007EE903AF8EE676A97ED046ADFED875A9C
S3150802AF90C6EE257A76EEA77AF7EE006A77EEA67AF5
S3150802AFA067EE277AC7ED097A68E0BB6907EE903A39
S3150802AFB0F8EE677ADFED7E6A86EEA77A3B6A07EED7
S3150802AFC0903AF8EE676A97ED046ADFED785AC6EEAC
S3150802AFD0257A76EEA77AF7EE006A77EEA67A67EE14
S3150802AFE0277AC7ED097A49E0BB6907EE903AF8EE87
S3150802AFF0677ADFED706A86EEA77A3B6A07EE903AC1
S3150802B000F8EE676A97ED046ADFED685AC6EE257AA6
S3150802B01076EEA77AF7EE006A77EEA67A67EE277AD1
S3150802B020C7ED097A2AE05F4B1B68DB0803F00303C6
S3150802B0305D4A22FA03F3FB60FB6807EE903AF8EEE4
S3150802B040676ABB6907EE903AF8EE677A86EEA77AE0
S3150802B0503B6A07EE903AF8EE676A97ED046ADFED07
S3150802B060535AC6EE257A76EEA77AF7EE006A77EE97
S3150802B070A67A67EE277AC7ED097A00BF494B1B689D
S3150802B08003F00073B3F1007F21D1464B9B6A03F4A8
S3150802B0908033002B17D0434B5B6B5B0A03F07F03AD
S3150802B0A007EE903AF8EE677AB7EE007A37EE877AC5
S3150802B0B0D7ED096AC6EE877AFCEEE77A17EE902A8A
S3150802B0C07B681A6006E07B6800221A6002E07B68E9
S3150802B0D000221A60334B1B6803F00073B3F1007F3A
S3150802B0E021D1304B9B6A03F40033002B17D02D4B2A
S3150802B0F05B6B1B0C03F07F0307EE903AF8EE677A58
S3150802B100B7EE007A37EE877AD7ED096AC6EE877AFE
S3150802B110FCEEE77A17EE902A7B685A6006E07B68AF
S3150802B12000225A6002E07B6800225A601D4B1B68A7
S3150802B13003F00073B3F1007F21D11A4B9B6A03F423
S3150802B1408023002B17D0174B5B6B1B0E03F07F0374
S3150802B15007EE903AF8EE677AB7EE007A37EE877A14
S3150802B160D7ED096AC6EE877AFCEEE77A17EE902AD9
S3150802B1707B689A6010E07B6800229A600CE07B6824
S3150802B18000229A6008E07B6800221A607B68002227
S3150802B1905A607B6800229A6000BF2C37BD465DF86C
S3150802B1A0047B7047000C02440090D003000000465E
S3150802B1B00024744A001B374B80B48BB000AF78600A
S3150802B1C0AD4BDB6BC3F308033B62AB4BDB6A03F0A5
S3150802B1D00303FB61A84BDB6A1B0A03F03F03BB614F
S3150802B1E0A54BDB6A03F010037B61A34B1B6CDB08E0
S3150802B1F0C3F30C037A6902FB03F307EE903AF8EEFF
S3150802B200677AC7ED047ABB69002B00F02681FB69D1
S3150802B210032B53D0FB69032B6FD8FB69012B03D091
S3150802B220FB69022B2BD068E0934B1B68DB0803F003
S3150802B2300303924A22FA03F3FB60FB6807EE903A8D
S3150802B240F8EE676ABB6907EE903AF8EE677A86EE19
S3150802B250A77A3B6A07EE903AF8EE676A97ED046AB0
S3150802B260DFED875AC6EE257A76EEA77AF7EE006AFA
S3150802B27077EEA67A67EE277AC7ED097A68E0BB69A0
S3150802B28007EE903AF8EE677ADFED7E6A86EEA77ADF
S3150802B2903B6A07EE903AF8EE676A97ED046ADFEDC5
S3150802B2A0785AC6EE257A76EEA77AF7EE006A77EE30
S3150802B2B0A67A67EE277AC7ED097A49E0BB6907EEEF
S3150802B2C0903AF8EE677ADFED706A86EEA77A3B6AFD
S3150802B2D007EE903AF8EE676A97ED046ADFED685A68
S3150802B2E0C6EE257A76EEA77AF7EE006A77EEA67AA2
S3150802B2F067EE277AC7ED097A2AE05F4B1B68DB08F7
S3150802B30003F003035D4A22FA03F3FB60FB6807EEC8
S3150802B310903AF8EE676ABB6907EE903AF8EE677AF2
S3150802B32086EEA77A3B6A07EE903AF8EE676A97EDD9
S3150802B330046ADFED535AC6EE257A76EEA77AF7EE59
S3150802B340006A77EEA67A67EE277AC7ED097A00BF12
S3150802B350494B1B6803F00063B3F1006F21D1464BDA
S3150802B360DB6A03F48033002B17D0434BDB6B5B0A93
S3150802B37003F07F0307EE903AF8EE677AB7EE007AA3
S3150802B38037EE877AD7ED096AC6EE877AFCEEE77A50
S3150802B39017EE902A7B681A6006E07B6800221A601C
S3150802B3A002E07B6800221A60334B1B6803F00063D5
S3150802B3B0B3F1006F21D1304BDB6A03F40033002B63
S3150802B3C017D02D4BDB6B1B0C03F07F0307EE903A6D
S3150802B3D0F8EE677AB7EE007A37EE877AD7ED096A1A
S3150802B3E0C6EE877AFCEEE77A17EE902A7B685A60F1
S3150802B3F006E07B6800225A6002E07B6800225A60F7
S3150802B4001D4B1B6803F00063B3F1006F21D11A4B81
S3150802B410DB6A03F48023002B17D0174BDB6B1B0E5A
S3150802B42003F07F0307EE903AF8EE677AB7EE007AF2
S3150802B43037EE877AD7ED096AC6EE877AFCEEE77A9F
S3150802B44017EE902A7B689A6010E07B6800229A6061
S3150802B4500CE07B6800229A6008E07B6800221A608A
S3150802B4607B6800225A607B6800229A6000BF2C37EC
S3150802B470BD465DF8047B7047000C02440090D00379
S3150802B480000000460024744A001B374B80B48BB078
S3150802B49000AF7860AD4B5B6CC3F308033B62AB4B02
S3150802B4A01B6B03F00303FB61A84B1B6B1B0A03F020
S3150802B4B03F03BB61A54B1B6B03F010037B61A34BD8
S3150802B4C09B6CDB08C3F30C037A6902FB03F307EEF2
S3150802B4D0903AF8EE677AC7ED047ABB69002B00F05A
S3150802B4E02681FB69032B53D0FB69032B6FD8FB69B3
S3150802B4F0012B03D0FB69022B2BD068E0934B1B6808
S3150802B500DB0803F00303924A22FA03F3FB60FB68A3
S3150802B51007EE903AF8EE676ABB6907EE903AF8EEDC
S3150802B520677A86EEA77A3B6A07EE903AF8EE676A7A
S3150802B53097ED046ADFED875AC6EE257A76EEA77A84
S3150802B540F7EE006A77EEA67A67EE277AC7ED097AEA
S3150802B55068E0BB6907EE903AF8EE677ADFED7E6A35
S3150802B56086EEA77A3B6A07EE903AF8EE676A97ED97
S3150802B570046ADFED785AC6EE257A76EEA77AF7EEF2
S3150802B580006A77EEA67A67EE277AC7ED097A49E066
S3150802B590BB6907EE903AF8EE677ADFED706A86EED7
S3150802B5A0A77A3B6A07EE903AF8EE676A97ED046A5D
S3150802B5B0DFED685AC6EE257A76EEA77AF7EE006AC6
S3150802B5C077EEA67A67EE277AC7ED097A2AE05F4B05
S3150802B5D01B68DB0803F003035D4A22FA03F3FB60E8
S3150802B5E0FB6807EE903AF8EE676ABB6907EE903A8F
S3150802B5F0F8EE677A86EEA77A3B6A07EE903AF8EE95
S3150802B600676A97ED046ADFED535AC6EE257A76EE37
S3150802B610A77AF7EE006A77EEA67A67EE277AC7ED7B
S3150802B620097A00BF494B1B6803F00053B3F1005F68
S3150802B63021D1464B1B6B03F48033002B17D0434BA7
S3150802B6405B6C5B0A03F07F0307EE903AF8EE677AC3
S3150802B650B7EE007A37EE877AD7ED096AC6EE877AA9
S3150802B660FCEEE77A17EE902A7B681A6006E07B689A
S3150802B67000221A6002E07B6800221A60334B1B68BC
S3150802B68003F00053B3F1005F21D1304B1B6B03F477
S3150802B6900033002B17D02D4B5B6C1B0C03F07F037A
S3150802B6A007EE903AF8EE677AB7EE007A37EE877ABF
S3150802B6B0D7ED096AC6EE877AFCEEE77A17EE902A84
S3150802B6C07B685A6006E07B6800225A6002E07B6863
S3150802B6D000225A601D4B1B6803F00053B3F1005F4A
S3150802B6E021D11A4B1B6B03F48023002B17D0174B5F
S3150802B6F05B6C1B0E03F07F0307EE903AF8EE677A4F
S3150802B700B7EE007A37EE877AD7ED096AC6EE877AF8
S3150802B710FCEEE77A17EE902A7B689A6010E07B685F
S3150802B72000229A600CE07B6800229A6008E07B6837
S3150802B73000221A607B6800225A607B6800229A609F
S3150802B74000BF2C37BD465DF8047B7047000C0244E7
S3150802B7500090D003000000460024744A001B374BB1
S3150802B76090B58FB000AFC7E90001D7E9000100F133
S3150802B7707E44214350D1264BD3F8F03003F440736C
S3150802B7803B63234BD3F8F03003F00203022B08D1B4
S3150802B7903B6BB3F5807F04D14FF400437B6302F021
S3150802B7A02ABB1B4BD3F8F03003F00063B3F1006FEA
S3150802B7B008D13B6BB3F5007F04D14FF4FA437B63A0
S3150802B7C002F019BB124B1B6803F40033B3F5003FB2
S3150802B7D019D13B6BB3F5407F15D10D4BDB6903F4E9
S3150802B7E07C53B3F5007F0AD3094BDB691B0A03F0C6
S3150802B7F03F03084AB2FBF3F37B6302F0FCBA002369
S3150802B8007B6302F0F8BA00237B6302F0F4BA00BF46
S3150802B810000C0244001BB700D7E90001A1F58064B9
S3150802B82050EA040101F07582D7E90001012871F591
S3150802B830806182F0DD82D7E90001A1F5007450EA41
S3150802B840040101F06C81D7E90001012871F5007144
S3150802B85082F0CE82D7E90001A1F5807450EA04018C
S3150802B86001F00286D7E90001012871F5807182F09C
S3150802B870BF82D7E90001A1F1800450EA040101F070
S3150802B8804C85D7E90001012871F1800182F0B08266
S3150802B890D7E90001A1F1400450EA040101F09E84AF
S3150802B8A0D7E90001012871F1400182F0A182D7E9A6
S3150802B8B00001A1F1200450EA040101F0E883D7E966
S3150802B8C00001012871F1200182F09282D7E9000174
S3150802B8D0A1F1100450EA040102F05682D7E90001E8
S3150802B8E0012871F1100182F08382D7E90001A1F1E2
S3150802B8F0080450EA040102F0CC81D7E900010128C4
S3150802B90071F1080182F07482D7E900010C1F50EA2E
S3150802B910040101F04886D7E90001012871F1040102
S3150802B92082F06682D7E900018C1E50EA040102F011
S3150802B9304381D7E90001012871F1020182F0588298
S3150802B940D7E900014C1E50EA040102F0CE80D7E97D
S3150802B9500001012871F1010182F04A82D7E900014A
S3150802B96000F10044214302F05980D7E90001D94C7D
S3150802B970A04271F1000182F03B82D7E9000100F191
S3150802B9804044214301F0D987D7E90001D24CA042AD
S3150802B99071F1000182F02C82D7E9000100F16044BE
S3150802B9A0214301F05187D7E90001CC4CA04271F13D
S3150802B9B0000182F01D82D7E9000100F1704421439B
S3150802B9C001F09A86D7E90001C54CA04271F100013F
S3150802B9D082F00E82D7E9000100F17844214301F092
S3150802B9E01286D7E90001BF4CA04271F1000182F02C
S3150802B9F0FF81D7E9000100F17C44214302F07E81F0
S3150802BA00D7E90001B84CA04271F1000182F0F08139
S3150802BA10D7E90001A0F50004214300F09E82D7E988
S3150802BA200001B24CA04271F1000182F0E181D7E92E
S3150802BA300001A0F58004214300F06D82D7E90001D8
S3150802BA40AB4CA04271F1000182F0D281D7E9000124
S3150802BA50A0F50014214301F00D80D7E90001A54C99
S3150802BA60A04271F1000182F0C381D7E90001A0F575
S3150802BA708014214300F0D081D7E900019E4CA042F0
S3150802BA8071F1000182F0B481D7E90001A0F5002422
S3150802BA90214300F04281D7E90001984CA04271F196
S3150802BAA0000182F0A581D7E90001A0F5802421438F
S3150802BAB001F04E82D7E90001914CA04271F10001D2
S3150802BAC082F09681D7E90001A0F50034214301F0FE
S3150802BAD09781D7E900018B4CA04271F1000182F0EF
S3150802BAE08781D7E90001A0F58034214301F054810A
S3150802BAF0D7E90001B0F1011F71F1000182F07881E6
S3150802BB00D7E90001A0F50044214301F0B780D7E93F
S3150802BB10000148F20104A04271F1000182F0688135
S3150802BB20D7E90001A0F58044214301F06480D7E9F2
S3150802BB30000144F20104A04271F1000182F0588129
S3150802BB40D7E90001A0F50054214301F01180D7E995
S3150802BB50000142F20104A04271F1000182F048811B
S3150802BB60D7E90001A0F58054214300F01E87D7E9E2
S3150802BB70000141F20104A04271F1000182F038810C
S3150802BB80D7E90001A0F50064214300F0A886D7E9A9
S3150802BB90000140F60104A04271F1000182F02881F9
S3150802BBA0D7E90001A0F58064214300F03286D7E97F
S3150802BBB0000140F20144A04271F1000182F01881AD
S3150802BBC0D7E90001A0F50074214300F0B085D7E952
S3150802BBD0000140F20124A04271F1000182F00881BD
S3150802BBE0D7E90001A0F58074214300F03585D7E92D
S3150802BBF0000140F20114A04271F1000182F0F880BE
S3150802BC00D7E90001A0F18004214300F0BA84D7E9FC
S3150802BC100001812871F1000182F0EA80D7E900016A
S3150802BC20212871F100016FD2D7E90001014302F020
S3150802BC30DF80D7E90001421E41F1FF33202A73F162
S3150802BC40000182F0D5801F2A02F2D28001A151F8A2
S3150802BC5022F000BFB5BF020881C00208F1DD020862
S3150802BC6041C10208F1DD0208F1DD0208F1DD020830
S3150802BC7011C20208F1DD0208F1DD0208F1DD02084F
S3150802BC80F1DD0208F1DD0208F1DD0208F1DD020844
S3150802BC90F3C20208F1DD0208F1DD0208F1DD02084D
S3150802BCA0F1DD0208F1DD0208F1DD0208F1DD020824
S3150802BCB0F1DD0208F1DD0208F1DD0208F1DD020814
S3150802BCC0F1DD0208F1DD0208F1DD0208F1DD020804
S3150802BCD0C9C30208010000800100004001000020DB
S3150802BCE001000010010000080100000401008000A4
S3150802BCF001004000010020000100100001000800B8
S3150802BD000100040001000200D7E90023A2F1400164
S3150802BD100B4300F0C48302F06BB8A14BD3F8E830AA
S3150802BD2003F4E0233B633B6BB3F5802F36D03B6BC2
S3150802BD30B3F5802F6BD83B6BB3F5403F2BD03B6BEB
S3150802BD40B3F5403F63D83B6BB3F5003F1BD03B6B63
S3150802BD50B3F5003F5BD83B6B002B04D03B6BB3F5C6
S3150802BD60803F08D053E007F120031846FFF7BAF8D8
S3150802BD707B6A7B634EE007F114031846FFF71CFA49
S3150802BD807B697B6346E007F108031846FFF77EFBEB
S3150802BD90BB687B633EE0834B7B633BE0804BD3F817
S3150802BDA0E83003F04043FB627D4B1B6803F0020355
S3150802BDB0022B0CD1FB6A002B09D1794B1B68DB08D5
S3150802BDC003F00303784A22FA03F37B631EE0744BFB
S3150802BDD01B6803F40073B3F5007F06D1FB6AB3F15F
S3150802BDE0804F02D1714B7B6310E06D4B1B6803F4E5
S3150802BDF00033B3F5003F06D1FB6AB3F1004F02D117
S3150802BE006B4B7B6302E000237B6303E002E00023C3
S3150802BE107B6300BF01F0EFBF614BD3F8E83003F450
S3150802BE2060133B633B6BB3F5001F36D03B6BB3F530
S3150802BE30001F6BD83B6BB3F5C01F2BD03B6BB3F51A
S3150802BE40C01F63D83B6BB3F5801F1BD03B6BB3F5A2
S3150802BE50801F5BD83B6B002B04D03B6BB3F5002FDE
S3150802BE6008D053E007F120031846FFF73BF87B6A30
S3150802BE707B634EE007F114031846FFF79DF97B69C9
S3150802BE807B6346E007F108031846FFF7FFFABB682B
S3150802BE907B633EE0434B7B633BE0414BD3F8E830A0
S3150802BEA003F04043FB623E4B1B6803F00203022B7E
S3150802BEB00CD1FB6A002B09D1394B1B68DB0803F04E
S3150802BEC00303394A22FA03F37B631EE0344B1B68E9
S3150802BED003F40073B3F5007F06D1FB6AB3F1804F12
S3150802BEE002D1324B7B6310E02D4B1B6803F40033FF
S3150802BEF0B3F5003F06D1FB6AB3F1004F02D12C4BD2
S3150802BF007B6302E000237B6303E002E000237B639A
S3150802BF1000BF01F070BF224BD3F8E43003F04003B0
S3150802BF203B633B6B002B08D107F120031846FEF74B
S3150802BF30D9FF7B6A7B6301F05EBF3B6B402B08D15E
S3150802BF4007F114031846FFF737F9FB697B6301F01B
S3150802BF5052BF00237B6301F04EBF114BD3F8E43086
S3150802BF6003F080033B633B6B002B08D107F12003E8
S3150802BF701846FEF7B7FF7B6A7B6301F03CBF3B6B53
S3150802BF80802B08D107F114031846FFF715F9FB6948
S3150802BF907B6301F030BF00237B6301F02CBF00BF37
S3150802BFA0000C02440080BB000090D00300093D004B
S3150802BFB0001BB7009D4BD3F8D83003F007033B6349
S3150802BFC03B6B002B04D1FCF79FFF786301F013BF8C
S3150802BFD0964B1B6803F00063B3F1006F0AD13B6B03
S3150802BFE0012B07D107F114031846FFF7E5F8BB69D9
S3150802BFF07B6343E08D4B1B6803F00053B3F1005F8C
S3150802C0000AD13B6B022B07D107F108031846FFF743
S3150802C0103DFAFB687B6331E0844B1B6803F002033D
S3150802C020022B0CD13B6B032B09D1804B1B68DB0817
S3150802C03003F003037E4A22FA03F37B631EE07B4B7B
S3150802C0401B6803F40073B3F5007F05D13B6B042B21
S3150802C05002D1784B7B6311E0744BD3F8F03003F0CE
S3150802C0600203022B06D13B6B052B03D14FF4004387
S3150802C0707B6303E000237B6301F0BDBE01F0BBBE18
S3150802C0806A4BD3F8D83003F038033B633B6B002B7B
S3150802C09004D1FCF723FF786301F0ADBE634B1B683E
S3150802C0A003F00063B3F1006F0AD13B6B082B07D18B
S3150802C0B007F114031846FFF77FF8BB697B633DE077
S3150802C0C03B6B102B08D107F108031846FFF7DEF978
S3150802C0D0FB687B6301F08FBE544B1B6803F00203B7
S3150802C0E0022B0CD13B6B182B09D1504B1B68DB0872
S3150802C0F003F003034E4A22FA03F37B631EE04B4B1B
S3150802C1001B6803F40073B3F5007F05D13B6B202B44
S3150802C11002D1484B7B6311E0444BD3F8F03003F06D
S3150802C1200203022B06D13B6B282B03D14FF40043A3
S3150802C1307B6303E000237B6301F05DBE01F05BBE17
S3150802C1403A4BD3F8D83003F4E0733B633B6B002BCE
S3150802C15004D1FCF7C3FE786301F04DBE334B1B686E
S3150802C16003F00063B3F1006F0AD13B6B402B07D192
S3150802C17007F114031846FFF71FF8BB697B6345E00E
S3150802C1802A4B1B6803F00053B3F1005F0AD13B6BDD
S3150802C190802B07D107F108031846FFF777F9FB68E2
S3150802C1A07B6333E0214B1B6803F00203022B0CD19D
S3150802C1B03B6BC02B09D11D4B1B68DB0803F003033D
S3150802C1C01B4A22FA03F37B6320E0184B1B6803F42D
S3150802C1D00073B3F5007F06D13B6BB3F5807F02D1BE
S3150802C1E0144B7B6312E0114BD3F8F03003F00203D1
S3150802C1F0022B07D13B6BB3F5A07F03D14FF4004363
S3150802C2007B6303E000237B6301F0F5BD01F0F3BD18
S3150802C210064BD3F8D83003F460633B633B6B002BC1
S3150802C2200AD1FCF75BFE786301F0E5BD000C024417
S3150802C2300090D00300093D00A04B1B6803F0006381
S3150802C240B3F1006F0BD13B6BB3F5007F07D107F152
S3150802C25014031846FEF7B0FFBB697B6347E0974BAA
S3150802C2601B6803F00053B3F1005F0BD13B6BB3F5C8
S3150802C270806F07D107F108031846FFF707F9FB682D
S3150802C2807B6334E08D4B1B6803F00203022B0DD14E
S3150802C2903B6BB3F5C06F09D1884B1B68DB0803F00B
S3150802C2A00303874A22FA03F37B6320E0834B1B6866
S3150802C2B003F40073B3F5007F06D13B6BB3F5006F49
S3150802C2C002D1804B7B6312E07C4BD3F8F03003F04B
S3150802C2D00203022B07D13B6BB3F5206F03D14FF450
S3150802C2E000437B6303E000237B6301F084BD01F016
S3150802C2F082BD724BD3F8D83003F4E0433B633B6B01
S3150802C300002B04D1FCF7EAFD786301F074BD6B4B90
S3150802C3101B6803F00063B3F1006F0BD13B6BB3F5F7
S3150802C320805F07D107F114031846FEF745FFBB697C
S3150802C3307B6347E0614B1B6803F00053B3F1005F70
S3150802C3400BD13B6BB3F5005F07D107F1080318461B
S3150802C350FFF79CF8FB687B6334E0584B1B6803F0D5
S3150802C3600203022B0DD13B6BB3F5405F09D1534B48
S3150802C3701B68DB0803F00303514A22FA03F37B63C3
S3150802C38020E04E4B1B6803F40073B3F5007F06D119
S3150802C3903B6BB3F5804F02D14A4B7B6312E0474BA6
S3150802C3A0D3F8F03003F00203022B07D13B6BB3F547
S3150802C3B0A04F03D14FF400437B6303E000237B6362
S3150802C3C001F019BD01F017BD3C4BD3F8D83003F480
S3150802C3D060333B633B6B002B04D1FCF77FFD78632C
S3150802C3E001F009BD354B1B6803F00063B3F1006F1A
S3150802C3F00BD13B6BB3F5004F07D107F1140318466F
S3150802C400FEF7DAFEBB697B6347E02C4B1B6803F039
S3150802C4100053B3F1005F0BD13B6BB3F5803F07D1F5
S3150802C42007F108031846FFF731F8FB687B6334E027
S3150802C430224B1B6803F00203022B0DD13B6BB3F5AB
S3150802C440C03F09D11D4B1B68DB0803F003031C4AD6
S3150802C45022FA03F37B6320E0184B1B6803F400738C
S3150802C460B3F5007F06D13B6BB3F5003F02D1154BFE
S3150802C4707B6312E0114BD3F8F03003F00203022B70
S3150802C48007D13B6BB3F5203F03D14FF400437B63DF
S3150802C49003E000237B6301F0AEBC01F0ACBC074BA2
S3150802C4A0D3F8D83003F4E0133B633B6B002B0BD174
S3150802C4B0FCF714FD786301F09EBC00BF000C024431
S3150802C4C00090D00300093D00A04B1B6803F00063EF
S3150802C4D0B3F1006F0BD13B6BB3F5802F07D107F190
S3150802C4E014031846FEF768FEBB697B6347E0974B61
S3150802C4F01B6803F00053B3F1005F0BD13B6BB3F536
S3150802C500002F07D107F108031846FEF7BFFFFB689D
S3150802C5107B6334E08D4B1B6803F00203022B0DD1BB
S3150802C5203B6BB3F5402F09D1884B1B68DB0803F038
S3150802C5300303874A22FA03F37B6320E0834B1B68D3
S3150802C54003F40073B3F5007F06D13B6BB3F5801F86
S3150802C55002D1804B7B6312E07C4BD3F8F03003F0B8
S3150802C5600203022B07D13B6BB3F5A01F03D14FF48D
S3150802C57000437B6303E000237B6301F03CBC01F0CC
S3150802C5803ABC724BD3F8D83003F460033B633B6B77
S3150802C590002B04D1FCF7A2FC786301F02CBC6B4B90
S3150802C5A01B6803F00063B3F1006F0BD13B6BB3F565
S3150802C5B0001F07D107F114031846FEF7FDFDBB69F4
S3150802C5C07B6347E0614B1B6803F00053B3F1005FDE
S3150802C5D00BD13B6BB3F5800F07D107F10803184659
S3150802C5E0FEF754FFFB687B6334E0584B1B6803F085
S3150802C5F00203022B0DD13B6BB3F5C00F09D1534B86
S3150802C6001B68DB0803F00303514A22FA03F37B6330
S3150802C61020E04E4B1B6803F40073B3F5007F06D186
S3150802C6203B6BB3F5000F02D14A4B7B6312E0474BD3
S3150802C630D3F8F03003F00203022B07D13B6BB3F5B4
S3150802C640200F03D14FF400437B6303E000237B638F
S3150802C65001F0D1BB01F0CFBB3C4BD3F8D83003F085
S3150802C660E0633B633B6B002B04D1FCF737FC786332
S3150802C67001F0C1BB354B1B6803F00063B3F1006FD1
S3150802C6800BD13B6BB3F1807F07D107F11403184630
S3150802C690FEF792FDBB697B6347E02C4B1B6803F0F0
S3150802C6A00053B3F1005F0BD13B6BB3F1007F07D1A7
S3150802C6B007F108031846FEF7E9FEFB687B6334E0D8
S3150802C6C0224B1B6803F00203022B0DD13B6BB3F11D
S3150802C6D0407F09D11D4B1B68DB0803F003031C4A84
S3150802C6E022FA03F37B6320E0184B1B6803F40073FA
S3150802C6F0B3F5007F06D13B6BB3F1806F02D1154BC0
S3150802C7007B6312E0114BD3F8F03003F00203022BDD
S3150802C71007D13B6BB3F1A06F03D14FF400437B63A0
S3150802C72003E000237B6301F066BB01F064BB074BA1
S3150802C730D3F8D83003F060533B633B6B002B0BD125
S3150802C740FCF7CCFB786301F056BB00BF000C024431
S3150802C7500090D00300093D00A14B1B6803F000635B
S3150802C760B3F1006F0BD13B6BB3F1006F07D107F141
S3150802C77014031846FEF720FDBB697B6347E0984B16
S3150802C7801B6803F00053B3F1005F0BD13B6BB3F1A7
S3150802C790805F07D107F108031846FEF777FEFB68A4
S3150802C7A07B6334E08E4B1B6803F00203022B0DD128
S3150802C7B03B6BB3F1C05F09D1894B1B68DB0803F0F9
S3150802C7C00303884A22FA03F37B6320E0844B1B683F
S3150802C7D003F40073B3F5007F06D13B6BB3F1005F38
S3150802C7E002D1814B7B6312E07D4BD3F8F03003F024
S3150802C7F00203022B07D13B6BB3F1205F03D14FF43F
S3150802C80000437B6303E000237B6301F0F4BA01F083
S3150802C810F2BA734BD3F8DC3003F007033B633B6B86
S3150802C820002B04D1FCF75AFB786301F0E4BA6C4B8F
S3150802C8301B6803F00063B3F1006F0AD13B6B012B4F
S3150802C84007D107F114031846FEF7B6FCBB697B63EA
S3150802C85043E0634B1B6803F00053B3F1005F0AD150
S3150802C8603B6B022B07D107F108031846FEF70EFEAB
S3150802C870FB687B6331E05A4B1B6803F00203022B09
S3150802C8800CD13B6B032B09D1554B1B68DB0803F014
S3150802C8900303544A22FA03F37B631EE0504B1B68D8
S3150802C8A003F40073B3F5007F05D13B6B042B02D169
S3150802C8B04D4B7B6311E04A4BD3F8F03003F0020389
S3150802C8C0022B06D13B6B052B03D14FF400437B6346
S3150802C8D003E000237B6301F08EBA01F08CBA404B69
S3150802C8E0D3F8DC3003F070033B633B6B002B04D1B7
S3150802C8F0FCF7F4FA786301F07EBA394B1B6803F049
S3150802C9000063B3F1006F0AD13B6B102B07D107F115
S3150802C91014031846FEF750FCBB697B6343E0304BB1
S3150802C9201B6803F00053B3F1005F0AD13B6B202B5F
S3150802C93007D107F108031846FEF7A8FDFB687B63D3
S3150802C94031E0274B1B6803F00203022B0CD13B6B29
S3150802C950302B09D1224B1B68DB0803F00303214A5B
S3150802C96022FA03F37B631EE01D4B1B6803F4007374
S3150802C970B3F5007F05D13B6B402B02D11A4B7B6383
S3150802C98011E0174BD3F8F03003F00203022B06D15D
S3150802C9903B6B502B03D14FF400437B6303E0002328
S3150802C9A07B6301F028BA01F026BA0D4BD3F8E030C2
S3150802C9B003F0E0633B633B6B002B04D1FCF7BAFA46
S3150802C9C0786301F018BA3B6BB3F1807F0ED107F199
S3150802C9D014031846FEF7F0FBBB697B6301F00BBA3A
S3150802C9E0000C02440090D00300093D003B6BB3F1F2
S3150802C9F0007F08D107F108031846FEF747FDFB68D2
S3150802CA007B6301F0F8B9A44B1B6803F00203022BFF
S3150802CA100DD13B6BB3F1407F09D19F4B1B68DB08F5
S3150802CA2003F003039D4A22FA03F37B6320E09A4B41
S3150802CA301B6803F40073B3F5007F06D13B6BB3F1B1
S3150802CA40806F02D1964B7B6312E0934BD3F8F0309A
S3150802CA5003F00203022B07D13B6BB3F1A06F03D19C
S3150802CA604FF400437B6303E000237B6301F0C3B901
S3150802CA7001F0C1B9884BD3F8E83003F007033B63EA
S3150802CA803B6B002B04D1FCF70DFA786301F0B3B9BE
S3150802CA903B6B012B04D1FCF7D9F8786301F0ABB9EB
S3150802CAA03B6B022B08D107F114031846FEF784FBE9
S3150802CAB0FB697B6301F09FB9774B1B6803F400336C
S3150802CAC0B3F5003F05D13B6B032B02D1754B7B6354
S3150802CAD023E0714B1B6803F00203022B0CD13B6B5C
S3150802CAE0042B09D16C4B1B68DB0803F003036B4A62
S3150802CAF022FA03F37B6310E0674B1B6803F40073A7
S3150802CB00B3F5007F05D13B6B052B02D1644B7B63E2
S3150802CB1003E000237B6301F06EB901F06CB95E4B4A
S3150802CB20D3F8E83003F008033B635B4BD3F8F030E5
S3150802CB3003F00203022B06D13B6B002B03D14FF401
S3150802CB4000437B6312E0544BD3F8F03003F00063E2
S3150802CB50B3F1006F06D13B6B082B03D14FF4FA43AE
S3150802CB607B6303E000237B6301F045B901F043B917
S3150802CB70494BD3F8E43003F440333B633B6B002B59
S3150802CB8004D1FCF7ABF9786301F035B93B6BB3F521
S3150802CB90803F08D107F108031846FEF777FC3B6980
S3150802CBA07B6301F028B93C4B1B6803F00203022B96
S3150802CBB00DD13B6BB3F5003F09D1374B1B68DB0838
S3150802CBC003F00303354A22FA03F37B6311E0324B7F
S3150802CBD01B6803F40073B3F5007F06D13B6BB3F50C
S3150802CBE0403F02D12E4B7B6303E000237B6301F0B7
S3150802CBF002B901F000B9284BD3F8E43003F4402314
S3150802CC003B633B6B002B04D1FCF768F9786301F0B0
S3150802CC10F2B83B6BB3F5802F08D107F10803184623
S3150802CC20FEF734FC3B697B6301F0E5B81A4B1B68D7
S3150802CC3003F00203022B0DD13B6BB3F5002F09D18A
S3150802CC40154B1B68DB0803F00303144A22FA03F3A5
S3150802CC507B6311E0104B1B6803F40073B3F5007F86
S3150802CC6006D13B6BB3F5402F02D10D4B7B6303E034
S3150802CC7000237B6301F0BFB801F0BDB8064BD3F8B9
S3150802CC80E43003F440133B633B6B002B0CD1FCF7F7
S3150802CC9051F9786301F0AFB8000C02440090D00352
S3150802CCA000093D00001BB7003B6BB3F5801F08D196
S3150802CCB007F108031846FEF7E9FB3B697B6301F0B7
S3150802CCC09AB89F4B1B6803F00203022B0DD13B6BEC
S3150802CCD0B3F5001F09D19A4B1B68DB0803F003035F
S3150802CCE0984A22FA03F37B6311E0954B1B6803F417
S3150802CCF00073B3F5007F06D13B6BB3F5401F02D133
S3150802CD00914B7B6303E000237B6301F074B801F067
S3150802CD1072B88B4BD3F8E43003F440033B633B6BA6
S3150802CD20002B04D1FCF706F9786301F064B83B6B73
S3150802CD30B3F5800F08D107F108031846FEF7A6FBDC
S3150802CD403B697B6301F057B87D4B1B6803F002030E
S3150802CD50022B0DD13B6BB3F5000F09D1784B1B683B
S3150802CD60DB0803F00303774A22FA03F37B6311E035
S3150802CD70734B1B6803F40073B3F5007F06D13B6B54
S3150802CD80B3F5400F02D1704B7B6303E000237B634C
S3150802CD9001F031B801F02FB8694BD3F8E43003F04B
S3150802CDA040733B633B6B002B04D1FCF797F878631F
S3150802CDB001F021B83B6BB3F1807F08D107F1080374
S3150802CDC01846FEF763FB3B697B6301F014B85C4BBC
S3150802CDD01B6803F00203022B0ED13B6BB3F1007FF3
S3150802CDE00AD1574B1B68DB0803F00303554A22FA9C
S3150802CDF003F37B6300F0FFBF00237B6300F0FBBFF6
S3150802CE004F4BD3F8DC3003F4E0633B633B6BB3F57B
S3150802CE10A06F56D03B6BB3F5A06F00F28B803B6BCD
S3150802CE20B3F5806F3ED03B6BB3F5806F00F282801C
S3150802CE303B6BB3F5407F27D03B6BB3F5407F79D880
S3150802CE403B6BB3F5007F17D03B6BB3F5007F71D808
S3150802CE503B6B002B04D03B6BB3F5807F04D069E0B3
S3150802CE60FCF768F8786368E007F114031846FEF7DA
S3150802CE70A3F97B697B6360E007F108031846FEF7AE
S3150802CE8005FB3B697B6358E02D4BD3F8F03003F082
S3150802CE900203022B03D14FF400437B634DE00023C8
S3150802CEA07B634AE0264BD3F8F03003F00063B3F114
S3150802CEB0006F03D14FF4FA437B633EE000237B63A2
S3150802CEC03BE01F4BD3F8E83003F04043FB621C4BB0
S3150802CED01B6803F00203022B0CD1FB6A002B09D153
S3150802CEE0174B1B68DB0803F00303164A22FA03F3FF
S3150802CEF07B631EE0124B1B6803F40073B3F5007FD5
S3150802CF0006D1FB6AB3F1804F02D10F4B7B6310E067
S3150802CF100B4B1B6803F40033B3F5003F06D1FB6ADB
S3150802CF20B3F1004F02D1094B7B6302E000237B6316
S3150802CF3003E002E000237B6300BF00F05CBF00BF92
S3150802CF40000C02440090D00300093D00001BB70004
S3150802CF509E4BD3F8DC3003F4E0433B633B6BB3F5FB
S3150802CF60A04F56D03B6BB3F5A04F00F28B803B6BBC
S3150802CF70B3F5804F3ED03B6BB3F5804F00F282800B
S3150802CF803B6BB3F5405F27D03B6BB3F5405F79D86F
S3150802CF903B6BB3F5005F17D03B6BB3F5005F71D8F7
S3150802CFA03B6B002B04D03B6BB3F5805F04D069E082
S3150802CFB0FBF794FF786368E007F114031846FEF757
S3150802CFC0FBF87B697B6360E007F108031846FEF706
S3150802CFD05DFA3B697B6358E07C4BD3F8F03003F08B
S3150802CFE00203022B03D14FF400437B634DE0002377
S3150802CFF07B634AE0754BD3F8F03003F00063B3F174
S3150802D000006F03D14FF4FA437B633EE000237B6350
S3150802D0103BE06E4BD3F8E83003F04043FB626B4BC0
S3150802D0201B6803F00203022B0CD1FB6A002B09D101
S3150802D030664B1B68DB0803F00303654A22FA03F30F
S3150802D0407B631EE0614B1B6803F40073B3F5007F34
S3150802D05006D1FB6AB3F1804F02D15E4B7B6310E0C7
S3150802D0605A4B1B6803F40033B3F5003F06D1FB6A3B
S3150802D070B3F1004F02D1584B7B6302E000237B6376
S3150802D08003E002E000237B6300BF00F0B4BE4F4B0F
S3150802D090D3F8DC3003F4E0233B633B6BB3F5A02FF4
S3150802D0A056D03B6BB3F5A02F00F28B803B6BB3F5E2
S3150802D0B0802F3ED03B6BB3F5802F00F282803B6B0C
S3150802D0C0B3F5403F27D03B6BB3F5403F79D83B6B6E
S3150802D0D0B3F5003F17D03B6BB3F5003F71D83B6BF6
S3150802D0E0002B04D03B6BB3F5803F04D069E0FBF715
S3150802D0F021FF786368E007F114031846FEF75CF827
S3150802D1007B697B6360E007F108031846FEF7BEF900
S3150802D1103B697B6358E02D4BD3F8F03003F00203EA
S3150802D120022B03D14FF400437B634DE000237B635C
S3150802D1304AE0264BD3F8F03003F00063B3F1006FF0
S3150802D14003D14FF4FA437B633EE000237B633BE063
S3150802D1501E4BD3F8E83003F04043FB621B4B1B68B7
S3150802D16003F00203022B0CD1FB6A002B09D1174BE1
S3150802D1701B68DB0803F00303154A22FA03F37B63F1
S3150802D1801EE0124B1B6803F40073B3F5007F06D149
S3150802D190FB6AB3F1804F02D10E4B7B6310E00B4B57
S3150802D1A01B6803F40033B3F5003F06D1FB6AB3F1FB
S3150802D1B0004F02D1084B7B6302E000237B6303E046
S3150802D1C002E000237B6300BF00F015BE000C024498
S3150802D1D00090D00300093D00001BB7009E4BD3F810
S3150802D1E0DC3003F4E0033B633B6BB3F5A00F56D088
S3150802D1F03B6BB3F5A00F00F28B803B6BB3F5800F48
S3150802D2003ED03B6BB3F5800F00F282803B6BB3F5E1
S3150802D210401F27D03B6BB3F5401F79D83B6BB3F55C
S3150802D220001F17D03B6BB3F5001F71D83B6B002B61
S3150802D23004D03B6BB3F5801F04D069E0FBF77AFE96
S3150802D240786368E007F114031846FDF7B5FF7B69B2
S3150802D2507B6360E007F108031846FEF717F93B6996
S3150802D2607B6358E07C4BD3F8F03003F00203022BC1
S3150802D27003D14FF400437B634DE000237B634AE00E
S3150802D280754BD3F8F03003F00063B3F1006F03D1A6
S3150802D2904FF4FA437B633EE000237B633BE06E4B2D
S3150802D2A0D3F8E83003F04043FB626B4B1B6803F08C
S3150802D2B00203022B0CD1FB6A002B09D1664B1B68B1
S3150802D2C0DB0803F00303654A22FA03F37B631EE0D5
S3150802D2D0614B1B6803F40073B3F5007F06D1FB6A42
S3150802D2E0B3F1804F02D15E4B7B6310E05A4B1B6849
S3150802D2F003F40033B3F5003F06D1FB6AB3F1004FDE
S3150802D30002D1584B7B6302E000237B6303E002E011
S3150802D31000237B6300BF00F06EBD4F4BD3F8DC30B1
S3150802D32003F0E0633B633B6BB3F1A06F56D03B6BF4
S3150802D330B3F1A06F00F28B803B6BB3F1806F3ED0E6
S3150802D3403B6BB3F1806F00F282803B6BB3F1407F97
S3150802D35027D03B6BB3F1407F79D83B6BB3F1007FA3
S3150802D36017D03B6BB3F1007F71D83B6B002B04D00F
S3150802D3703B6BB3F1807F04D069E0FBF7DBFD786392
S3150802D38068E007F114031846FDF716FF7B697B630D
S3150802D39060E007F108031846FEF778F83B697B63F5
S3150802D3A058E02D4BD3F8F03003F00203022B03D1D9
S3150802D3B04FF400437B634DE000237B634AE0264B30
S3150802D3C0D3F8F03003F00063B3F1006F03D14FF4E2
S3150802D3D0FA437B633EE000237B633BE01E4BD3F8B4
S3150802D3E0E83003F04043FB621B4B1B6803F0020361
S3150802D3F0022B0CD1FB6A002B09D1174B1B68DB08E1
S3150802D40003F00303154A22FA03F37B631EE0124B69
S3150802D4101B6803F40073B3F5007F06D1FB6AB3F108
S3150802D420804F02D10E4B7B6310E00B4B1B6803F453
S3150802D4300033B3F5003F06D1FB6AB3F1004F02D1C0
S3150802D440084B7B6302E000237B6303E002E00023D0
S3150802D4507B6300BF00F0CFBC000C02440090D003EF
S3150802D46000093D00001BB7009E4BD3F8DC3003F0E1
S3150802D470E0433B633B6BB3F1A04F56D03B6BB3F132
S3150802D480A04F00F28B803B6BB3F1804F3ED03B6BD3
S3150802D490B3F1804F00F282803B6BB3F1405F27D035
S3150802D4A03B6BB3F1405F79D83B6BB3F1005F17D0A2
S3150802D4B03B6BB3F1005F71D83B6B002B04D03B6B1F
S3150802D4C0B3F1805F04D069E0FBF734FD786368E066
S3150802D4D007F114031846FDF76FFE7B697B6360E06C
S3150802D4E007F108031846FDF7D1FF3B697B6358E04D
S3150802D4F07C4BD3F8F03003F00203022B03D14FF42E
S3150802D50000437B634DE000237B634AE0754BD3F807
S3150802D510F03003F00063B3F1006F03D14FF4FA431E
S3150802D5207B633EE000237B633BE06E4BD3F8E83037
S3150802D53003F04043FB626B4B1B6803F00203022BAA
S3150802D5400CD1FB6A002B09D1664B1B68DB0803F07A
S3150802D5500303654A22FA03F37B631EE0614B1B68E9
S3150802D56003F40073B3F5007F06D1FB6AB3F1804F6B
S3150802D57002D15E4B7B6310E05A4B1B6803F40033FF
S3150802D580B3F5003F06D1FB6AB3F1004F02D1584BFF
S3150802D5907B6302E000237B6303E002E000237B63F4
S3150802D5A000BF00F028BC4F4BD3F8E83003F44073B1
S3150802D5B03B634C4B1B6803F40033B3F5003F06D1BB
S3150802D5C03B6B002B03D14A4B7B6300F014BC3B6BCD
S3150802D5D0B3F5807F08D107F120031846FDF782FCD0
S3150802D5E07B6A7B6300F007BC3B6BB3F5007F07D110
S3150802D5F007F114031846FDF7DFFDBB697B63FAE3FF
S3150802D60000237B63F7E3374BD3F8E03003F00703D5
S3150802D6103B633B6B042B61D801A252F823F000BF8F
S3150802D62035D6020845D6020855D6020865D6020836
S3150802D6306BD6020807F120031846FDF753FC7B6AEE
S3150802D6407B634EE007F114031846FDF7B5FD7B69C7
S3150802D6507B6346E007F108031846FDF717FFBB6828
S3150802D6607B633EE0234B7B633BE01E4BD3F8E830FB
S3150802D67003F04043FB621B4B1B6803F00203022BB9
S3150802D6800CD1FB6A002B09D1164B1B68DB0803F089
S3150802D6900303154A22FA03F37B631EE0114B1B6848
S3150802D6A003F40073B3F5007F06D1FB6AB3F1804F2A
S3150802D6B002D10E4B7B6310E00A4B1B6803F400335E
S3150802D6C0B3F5003F06D1FB6AB3F1004F02D1084B0E
S3150802D6D07B6302E000237B6303E002E000237B63B3
S3150802D6E000BF88E3000C02440090D00300093D0005
S3150802D6F0001BB7000080BB00A94BD3F8E03003F04B
S3150802D70038033B633B6B202B00F29A8001A252F846
S3150802D71023F000BF99D7020841D8020841D8020867
S3150802D72041D8020841D8020841D8020841D802085D
S3150802D73041D80208A9D7020841D8020841D80208E6
S3150802D74041D8020841D8020841D8020841D802083D
S3150802D75041D80208B9D7020841D8020841D80208B6
S3150802D76041D8020841D8020841D8020841D802081D
S3150802D77041D80208C9D7020841D8020841D8020886
S3150802D78041D8020841D8020841D8020841D80208FD
S3150802D79041D80208CFD7020807F120031846FDF739
S3150802D7A0A1FB7B6A7B634EE007F114031846FDF77B
S3150802D7B003FD7B697B6346E007F108031846FDF71C
S3150802D7C065FEBB687B633EE0764B7B633BE0744B4E
S3150802D7D0D3F8E83003F04043FB62714B1B6803F051
S3150802D7E00203022B0CD1FB6A002B09D16C4B1B6876
S3150802D7F0DB0803F003036C4A22FA03F37B631EE099
S3150802D800674B1B6803F40073B3F5007F06D1FB6A06
S3150802D810B3F1804F02D1654B7B6310E0604B1B6806
S3150802D82003F40033B3F5003F06D1FB6AB3F1004FA8
S3150802D83002D15F4B7B6302E000237B6303E002E0D5
S3150802D84000237B6300BFD6E2554BD3F8E03003F4DE
S3150802D850E0733B633B6BB3F5807F31D03B6BB3F52B
S3150802D860807F66D83B6BC02B27D03B6BC02B60D81A
S3150802D8703B6B802B19D03B6B802B5AD83B6B002B0A
S3150802D88003D03B6B402B08D053E007F12003184620
S3150802D890FDF728FB7B6A7B634EE007F11403184603
S3150802D8A0FDF78AFC7B697B6346E007F108031846A5
S3150802D8B0FDF7ECFDBB687B633EE03A4B7B633BE0DE
S3150802D8C0374BD3F8E83003F04043FB62344B1B680E
S3150802D8D003F00203022B0CD1FB6A002B09D1304B51
S3150802D8E01B68DB0803F003032F4A22FA03F37B6360
S3150802D8F01EE02B4B1B6803F40073B3F5007F06D1B9
S3150802D900FB6AB3F1804F02D1284B7B6310E0244BAC
S3150802D9101B6803F40033B3F5003F06D1FB6AB3F183
S3150802D920004F02D1224B7B6302E000237B6303E0B4
S3150802D93002E000237B6300BF5DE2194BD3F8E030B7
S3150802D94003F460633B633B6B002B03D1FBF7DCFA02
S3150802D950786350E2124B1B6803F00063B3F1006F61
S3150802D9600BD13B6BB3F5007F07D107F114031846B9
S3150802D970FDF722FCBB697B634FE0094B1B6803F08A
S3150802D9800053B3F1005F15D13B6BB3F5806F11D12C
S3150802D99007F108031846FDF779FDFB687B633CE04F
S3150802D9A0000C02440080BB000090D00300093D0031
S3150802D9B0001BB700944B1B6803F00203022B0DD120
S3150802D9C03B6BB3F5C06F09D18F4B1B68DB0803F0BD
S3150802D9D003038E4A22FA03F37B631EE08A4B1B6813
S3150802D9E003F40073B3F5007F06D13B6BB3F5006F02
S3150802D9F002D1874B7B6310E0834B1B6803F4003329
S3150802DA00B3F5003F06D13B6BB3F5206F02D1814BCC
S3150802DA107B6302E000237B63EDE1ECE17A4BD3F80A
S3150802DA20E03003F4E0433B633B6B002B03D1FBF787
S3150802DA3081FA7863DFE1744B1B6803F00063B3F184
S3150802DA40006F0BD13B6BB3F5805F07D107F1140367
S3150802DA501846FDF7B1FBBB697B6345E06A4B1B6859
S3150802DA6003F00053B3F1005F0BD13B6BB3F5005FD4
S3150802DA7007D107F108031846FDF708FDFB687B6323
S3150802DA8032E0614B1B6803F00203022B0DD13B6B9C
S3150802DA90B3F5405F09D15C4B1B68DB0803F003034F
S3150802DAA05A4A22FA03F37B631EE0574B1B6803F4B8
S3150802DAB00073B3F5007F06D13B6BB3F5804F02D1F5
S3150802DAC0534B7B6310E0504B1B6803F40033B3F5EA
S3150802DAD0003F06D13B6BB3F5A04F02D14D4B7B639A
S3150802DAE002E000237B6386E185E1474BD3F8E03009
S3150802DAF003F460333B633B6B002B03D1FBF704FA59
S3150802DB00786378E1404B1B6803F00063B3F1006F5A
S3150802DB100BD13B6BB3F5004F07D107F11403184637
S3150802DB20FDF74AFBBB697B6345E0374B1B6803F08D
S3150802DB300053B3F1005F0BD13B6BB3F5803F07D1BE
S3150802DB4007F108031846FDF7A1FCFB687B6332E080
S3150802DB502D4B1B6803F00203022B0DD13B6BB3F569
S3150802DB60C03F09D1284B1B68DB0803F00303274A89
S3150802DB7022FA03F37B631EE0234B1B6803F400734C
S3150802DB80B3F5007F06D13B6BB3F5003F02D1204BBC
S3150802DB907B6310E01C4B1B6803F40033B3F5003FAC
S3150802DBA006D13B6BB3F5203F02D11A4B7B6302E0E9
S3150802DBB000237B631FE11EE1134BD3F8E43003F025
S3150802DBC003033B633B6B032B5FD801A252F823F096
S3150802DBD0E1DB0208E9DB0208F9DB020819DC0208C4
S3150802DBE0FBF760F9786353E007F120031846FDF75F
S3150802DBF079F97B6A7B634BE007F114031846FDF754
S3150802DC00DBFAFB697B6343E0000C02440090D00315
S3150802DC1000093D00001BB700794BD3F8E83003F042
S3150802DC204043FB62764B1B6803F00203022B0CD1BE
S3150802DC30FB6A002B09D1724B1B68DB0803F003034E
S3150802DC40704A22FA03F37B631EE06D4B1B6803F4EA
S3150802DC500073B3F5007F06D1FB6AB3F1804F02D198
S3150802DC60694B7B6310E0664B1B6803F40033B3F51C
S3150802DC70003F06D1FB6AB3F1004F02D1634B7B63C7
S3150802DC8002E000237B6303E002E000237B6300BF1C
S3150802DC90B1E05B4BD3F8E83003F0C0033B63584B63
S3150802DCA0D3F8F03003F00203022B06D13B6B002BAC
S3150802DCB003D14FF400437B631FE0514BD3F8F03096
S3150802DCC003F00063B3F1006F06D13B6B402B03D11F
S3150802DCD04FF4FA437B6310E0494B1B6803F4007365
S3150802DCE0B3F5007F06D13B6B802B03D148F21203B2
S3150802DCF07B6302E000237B637DE07CE0404BD3F844
S3150802DD00E83003F030033B633D4B1B6803F40053D2
S3150802DD10B3F5005F05D13B6B002B02D13C4B7B630D
S3150802DD2031E0374B1B6803F00073B3F1007F0AD169
S3150802DD303B6B102B07D107F120031846FDF7D2F8E3
S3150802DD407B6A7B631FE02E4BD3F8F03003F00203A5
S3150802DD50022B06D13B6B202B03D14FF400437B6386
S3150802DD6011E0274BD3F8F03003F00063B3F1006FEC
S3150802DD7006D13B6B302B03D14FF4FA437B6302E0A7
S3150802DD8000237B6337E036E01D4BD3F8E43003F01B
S3150802DD9030033B633B6B102B07D107F12003184670
S3150802DDA0FDF7A0F87B6A7B6325E0154B1B6803F039
S3150802DDB00053B3F1005F0AD13B6B202B07D107F161
S3150802DDC008031846FDF762FBFB687B630FE00C4B02
S3150802DDD01B6803F40053B3F5005F05D13B6B302B88
S3150802DDE002D10B4B7B6302E000237B6303E002E074
S3150802DDF000237B6300BF7B6B18463C37BD4690BD4C
S3150802DE00000C02440090D00300093D00001BB70035
S3150802DE10006CDC0280B584B000AF7860484B1B68A2
S3150802DE20474A23F080631360F8F7D2FAF86008E0ED
S3150802DE30F8F7CEFA0246FB68D31A022B01D9032356
S3150802DE407AE03F4B1B6803F00063002BF0D13C4B92
S3150802DE50DB6A23F47C5323F003037A6811687A6831
S3150802DE60526812020A4336491343CB627B689B689F
S3150802DE70013BC3F308027B68DB68013B5B029BB28A
S3150802DE801A437B681B69013B1B0403F4FE031A430E
S3150802DE907B685B69013B1B0603F0FE432849134373
S3150802DEA0CB63274BDB6A23F00C027B689B69244908
S3150802DEB01343CB62224BDB6A23F020027B68DB69C1
S3150802DEC01F491343CB621E4BDA6A7B685B6A1C499D
S3150802DED01343CB621A4BDB6A194A23F01003D36247
S3150802DEE0174B1B6C23F47F4323F0F8037A68126AF4
S3150802DEF0D200134913430B64114BDB6A104A43F0F1
S3150802DF001003D3620E4B1B680D4A43F080631360FD
S3150802DF10F8F75EFAF86008E0F8F75AFA0246FB687C
S3150802DF20D31A022B01D9032306E0054B1B6803F01B
S3150802DF300063002BF0D0002318461037BD4680BD7B
S3150802DF40000C024480B584B000AF7860484B1B6869
S3150802DF50474A23F080531360F8F73AFAF86008E064
S3150802DF60F8F736FA0246FB68D31A022B01D90323BD
S3150802DF707AE03F4B1B6803F00053002BF0D13C4B71
S3150802DF801B6B23F47C5323F003037A6811687A68BF
S3150802DF90526812020A43364913430B637B689B682D
S3150802DFA0013BC3F308027B68DB68013B5B029BB259
S3150802DFB01A437B681B69013B1B0403F4FE031A43DD
S3150802DFC07B685B69013B1B0603F0FE432849134342
S3150802DFD04B64274B1B6B23F00C027B689B69244915
S3150802DFE013430B63224B1B6B23F020027B68DB690E
S3150802DFF01F4913430B631E4B1A6B7B685B6A1C49EA
S3150802E00013430B631A4B1B6B194A23F01003136352
S3150802E010174B9B6C23F47F4323F0F8037A68126A42
S3150802E020D200134913438B64114B1B6B104A43F0FE
S3150802E030100313630E4B1B680D4A43F0805313609B
S3150802E040F8F7C6F9F86008E0F8F7C2F90246FB687D
S3150802E050D31A022B01D9032306E0054B1B6803F0EA
S3150802E0600053002BF0D0002318461037BD4680BD5A
S3150802E070000C024480B582B000AF78607B68002B42
S3150802E08001D1012349E07B6893F83D30DBB2002BCE
S3150802E09006D17B68002283F83C207868F6F77CFD77
S3150802E0A07B68022283F83D207B681A687B68043302
S3150802E0B01946104600F074FB7B68012283F8482053
S3150802E0C07B68012283F83E207B68012283F83F2081
S3150802E0D07B68012283F840207B68012283F841206D
S3150802E0E07B68012283F842207B68012283F8432059
S3150802E0F07B68012283F844207B68012283F8452045
S3150802E1007B68012283F846207B68012283F8472030
S3150802E1107B68012283F83D20002318460837BD464E
S3150802E12080BD000080B485B000AF78607B6893F844
S3150802E1303D30DBB2012B01D001237CE07B68022251
S3150802E14083F83D207B681B68DA687B681B6842F0A7
S3150802E1500102DA607B681B683A4A93424AD07B68B6
S3150802E1601B68394A934245D07B681B68B3F1804FD6
S3150802E17040D07B681B68B3F1A04F3BD07B681B6815
S3150802E180324A934236D07B681B68314A934231D071
S3150802E1907B681B682F4A93422CD07B681B682E4AE1
S3150802E1A0934227D07B681B682C4A934222D07B680D
S3150802E1B01B682B4A93421DD07B681B68294A9342E7
S3150802E1C018D07B681B68284A934213D07B681B6861
S3150802E1D0264A93420ED07B681B68254A934209D089
S3150802E1E07B681B68234A934204D07B681B68224AD1
S3150802E1F0934215D17B681B689A68204B1340FB60D3
S3150802E200FB68062B15D0FB68B3F5803F11D07B68F7
S3150802E2101B681A687B681B6842F001021A6008E0EC
S3150802E2207B681B681A687B681B6842F001021A60E1
S3150802E23000E000BF002318461437BD465DF8047B8C
S3150802E240704700BF002C0140002C0150000400401A
S3150802E250000400500008004000080050000C00406E
S3150802E260000C0050003401400034015000180040F0
S3150802E270001800500040014000400150070001000C
S3150802E28080B584B000AF78607B681B68DB68FB608A
S3150802E2907B681B681B69BB60BB6803F00203002B23
S3150802E2A020D0FB6803F00203002B1BD07B681B6897
S3150802E2B06FF002021A617B6801221A777B681B6873
S3150802E2C09B6903F00303002B03D0786800F04AFA2F
S3150802E2D005E0786800F03CFA786800F04DFA7B6849
S3150802E2E000221A77BB6803F00403002B20D0FB68D0
S3150802E2F003F00403002B1BD07B681B686FF0040233
S3150802E3001A617B6802221A777B681B689B6903F489
S3150802E3104073002B03D0786800F024FA05E0786889
S3150802E32000F016FA786800F027FA7B6800221A7756
S3150802E330BB6803F00803002B20D0FB6803F0080330
S3150802E340002B1BD07B681B686FF008021A617B687A
S3150802E35004221A777B681B68DB6903F00303002B28
S3150802E36003D0786800F0FEF905E0786800F0F0F965
S3150802E370786800F001FA7B6800221A77BB6803F016
S3150802E3801003002B20D0FB6803F01003002B1BD0D0
S3150802E3907B681B686FF010021A617B6808221A777D
S3150802E3A07B681B68DB6903F44073002B03D078682B
S3150802E3B000F0D8F905E0786800F0CAF9786800F044
S3150802E3C0DBF97B6800221A77BB6803F00103002B8E
S3150802E3D00CD0FB6803F00103002B07D07B681B688F
S3150802E3E06FF001021A617868F6F776F9BB6803F0EE
S3150802E3F08003002B0CD0FB6803F08003002B07D0A8
S3150802E4007B681B686FF080021A61786800F05CFC12
S3150802E410BB6803F48073002B0CD0FB6803F08003FF
S3150802E420002B07D07B681B686FF480721A617868C4
S3150802E43000F054FCBB6803F04003002B0CD0FB68C9
S3150802E44003F04003002B07D07B681B686FF040027D
S3150802E4501A61786800F09AF9BB6803F02003002B6A
S3150802E4600CD0FB6803F02003002B07D07B681B68DF
S3150802E4706FF020021A61786800F01CFCBB6803F48E
S3150802E4808013002B0CD0FB6803F48013002B07D0F3
S3150802E4907B681B686FF480121A61786800F028FCA2
S3150802E4A0BB6803F40013002B0CD0FB6803F40013BB
S3150802E4B0002B07D07B681B686FF400121A61786814
S3150802E4C000F020FCBB6803F48003002B0CD0FB6829
S3150802E4D003F48003002B07D07B681B686FF4800265
S3150802E4E01A61786800F018FCBB6803F40003002B75
S3150802E4F00CD0FB6803F40003002B07D07B681B686B
S3150802E5006FF400021A61786800F010FC00BF103739
S3150802E510BD4680BD80B584B000AF786039600023FF
S3150802E520FB737B6893F83C30012B01D10223FEE092
S3150802E5307B68012283F83C207B68022283F83D200F
S3150802E5407B681B689B68BB60BB6823F4441323F093
S3150802E5507703BB60BB6823F47F43BB607B681B6899
S3150802E560BA689A603B681B68B3F5001F00F0C98059
S3150802E570B3F5001F00F2CE806F4A934200F0C180C5
S3150802E5806D4A934200F2C6806C4A934200F0B98003
S3150802E5906A4A934200F2BE80694A934200F0B18009
S3150802E5A0674A934200F2B680664A934200F0A9800F
S3150802E5B0644A934200F2AE80634A934200F0A18015
S3150802E5C0614A934200F2A680604A934200F099801B
S3150802E5D05E4A934200F29E80B3F1101F00F09180CA
S3150802E5E0B3F1101F00F29680B3F5801F00F0898000
S3150802E5F0B3F5801F00F28E80B3F5005F3ED0B3F507
S3150802E600005F00F28780B3F5805F00F08680B3F57D
S3150802E610805F7FD8702B1AD0702B7BD8602B50D096
S3150802E620602B77D8502B3CD0502B73D8402B58D020
S3150802E630402B6FD8302B64D0302B6BD8202B60D070
S3150802E640202B67D8002B5CD0102B5AD062E07B684F
S3150802E65018683B6899683B685A683B68DB6800F04B
S3150802E66039FA7B681B689B68BB60BB6843F0770313
S3150802E670BB607B681B68BA689A604FE07B6818685B
S3150802E6803B6899683B685A683B68DB6800F022FA7F
S3150802E6907B681B689A687B681B6842F480429A60AA
S3150802E6A03CE07B6818683B6859683B68DB681A4631
S3150802E6B000F094F97B681B685021184600F0EDF9C2
S3150802E6C02CE07B6818683B6859683B68DB681A4621
S3150802E6D000F0B3F97B681B686021184600F0DDF983
S3150802E6E01CE07B6818683B6859683B68DB681A4611
S3150802E6F000F074F97B681B684021184600F0CDF9D2
S3150802E7000CE07B681A683B681B681946104600F0DD
S3150802E710C4F903E00123FB7300E000BF7B68012212
S3150802E72083F83D207B68002283F83C20FB7B184651
S3150802E7301037BD4680BD00BF700010006000100093
S3150802E7405000100040001000300010002000100099
S3150802E75080B483B000AF786000BF0C37BD465DF861
S3150802E760047B704780B483B000AF786000BF0C3773
S3150802E770BD465DF8047B704780B483B000AF78600D
S3150802E78000BF0C37BD465DF8047B704780B483B082
S3150802E79000AF786000BF0C37BD465DF8047B704752
S3150802E7A080B485B000AF786039607B681B68FB600F
S3150802E7B07B68744A93422BD07B68734A934227D06C
S3150802E7C07B68B3F1804F23D07B68B3F1A04F1FD08B
S3150802E7D07B686E4A93421BD07B686D4A934217D078
S3150802E7E07B686C4A934213D07B686B4A93420FD07C
S3150802E7F07B686A4A93420BD07B68694A934207D080
S3150802E8007B68684A934203D07B68674A934208D179
S3150802E810FB6823F07003FB603B685B68FA68134386
S3150802E820FB607B68574A93425BD07B68564A9342A1
S3150802E83057D07B68B3F1804F53D07B68B3F1A04FB2
S3150802E8404FD07B68514A93424BD07B68504A9342D9
S3150802E85047D07B684F4A934243D07B684E4A9342DD
S3150802E8603FD07B684D4A93423BD07B684C4A9342E1
S3150802E87037D07B684B4A934233D07B684A4A9342E5
S3150802E8802FD07B68494A93422BD07B68484A9342E9
S3150802E89027D07B68474A934223D07B68464A9342ED
S3150802E8A01FD07B68454A93421BD07B68444A9342F1
S3150802E8B017D07B68434A934213D07B68424A9342F5
S3150802E8C00FD07B68414A93420BD07B68404A9342F9
S3150802E8D007D07B683F4A934203D07B683E4A9342FD
S3150802E8E008D1FB6823F44073FB603B68DB68FA686F
S3150802E8F01343FB60FB6823F080023B685B691343A2
S3150802E900FB607B68FA681A603B689A687B68DA6219
S3150802E9103B681A687B689A627B681A4A934223D0D4
S3150802E9207B68194A93421FD07B681E4A93421BD0C2
S3150802E9307B681D4A934217D07B68224A934213D0BA
S3150802E9407B68214A93420FD07B68204A93420BD0B8
S3150802E9507B681F4A934207D07B681E4A934203D0BC
S3150802E9607B681D4A934203D13B681A697B681A631E
S3150802E9707B6801225A6100BF1437BD465DF8047BE5
S3150802E980704700BF002C0140002C015000040040D3
S3150802E990000400500008004000080050000C004027
S3150802E9A0000C0050003401400034015000180040A9
S3150802E9B000180050001C0040001C005000200040B7
S3150802E9C00020005000400140004001500044014030
S3150802E9D000440150004801400048015080B487B005
S3150802E9E000AFF860B9607A60FB681B6A7B61FB68F6
S3150802E9F01B6A23F00102FB681A62FB689B693B618A
S3150802EA003B6923F0F0033B617B681B013A691343B8
S3150802EA103B617B6923F00A037B617A69BB6813430E
S3150802EA207B61FB683A699A61FB687A691A6200BF78
S3150802EA301C37BD465DF8047B704780B487B000AFCB
S3150802EA40F860B9607A60FB681B6A7B61FB681B6ABF
S3150802EA5023F01002FB681A62FB689B693B613B69FB
S3150802EA6023F470433B617B681B033A6913433B619A
S3150802EA707B6923F0A0037B61BB681B017A69134398
S3150802EA807B61FB683A699A61FB687A691A6200BF18
S3150802EA901C37BD465DF8047B704780B485B000AF6D
S3150802EAA0786039607B689B68FB60FB6823F44013D7
S3150802EAB023F07003FB603A68FB68134343F00703CD
S3150802EAC0FB607B68FA689A6000BF1437BD465DF83A
S3150802EAD0047B704780B487B000AFF860B9607A608B
S3150802EAE03B60FB689B687B617B6923F47F437B61A0
S3150802EAF03B681A027B681A43BB6813437A69134355
S3150802EB007B61FB687A699A6000BF1C37BD465DF86F
S3150802EB10047B704780B485B000AF786039607B6843
S3150802EB2093F83C30012B01D10223A1E07B68012234
S3150802EB3083F83C207B68022283F83D207B681B68A9
S3150802EB405B68FB607B681B689B68BB607B681B68AD
S3150802EB504A4A93420ED07B681B68494A934209D0B7
S3150802EB607B681B68474A934204D07B681B68464AFF
S3150802EB70934208D1FB6823F47003FB603B685B6829
S3150802EB80FA681343FB60FB6823F0007323F07003F3
S3150802EB90FB603B681B68FA681343FB607B681B686B
S3150802EBA0FA685A607B681B68344A93424AD07B6883
S3150802EBB01B68334A934245D07B681B68B3F1804F82
S3150802EBC040D07B681B68B3F1A04F3BD07B681B68BB
S3150802EBD02E4A934236D07B681B682D4A934231D01F
S3150802EBE07B681B682B4A93422CD07B681B682A4A8F
S3150802EBF0934227D07B681B68284A934222D07B68B7
S3150802EC001B68274A93421DD07B681B681D4A93429C
S3150802EC1018D07B681B681C4A934213D07B681B6812
S3150802EC20204A93420ED07B681B681F4A934209D03A
S3150802EC307B681B681D4A934204D07B681B681C4A82
S3150802EC4093420CD1BB6823F08003BB603B689B6888
S3150802EC50BA681343BB607B681B68BA689A607B68AC
S3150802EC60012283F83D207B68002283F83C2000239A
S3150802EC7018461437BD465DF8047B7047002C0140E0
S3150802EC80002C0150003401400034015000040040B9
S3150802EC90000400500008004000080050000C004024
S3150802ECA0000C0050001800400018005000400140B7
S3150802ECB00040015080B483B000AF786000BF0C37C3
S3150802ECC0BD465DF8047B704780B483B000AF7860B8
S3150802ECD000BF0C37BD465DF8047B704780B483B02D
S3150802ECE000AF786000BF0C37BD465DF8047B7047FD
S3150802ECF080B483B000AF786000BF0C37BD465DF8BC
S3150802ED00047B704780B483B000AF786000BF0C37CD
S3150802ED10BD465DF8047B704780B483B000AF786067
S3150802ED2000BF0C37BD465DF8047B704780B483B0DC
S3150802ED3000AF786000BF0C37BD465DF8047B7047AC
S3150802ED4080B582B000AF78607B68002B01D10123C1
S3150802ED5042E07B68D3F88830002B06D17B68002214
S3150802ED6083F884207868F5F73DFF7B682422C3F888
S3150802ED7088207B681B681A687B681B6822F0010278
S3150802ED801A607B689B6A002B02D0786800F020FF25
S3150802ED90786800F02FFD0346012B01D101231BE001
S3150802EDA07B681B685A687B681B6822F490425A6023
S3150802EDB07B681B689A687B681B6822F02A029A603D
S3150802EDC07B681B681A687B681B6842F001021A6036
S3150802EDD0786800F09FFF034618460837BD4680BD8F
S3150802EDE080B582B000AF78607B68002B01D1012321
S3150802EDF031E07B682422C3F888207B681B681A687E
S3150802EE007B681B6822F001021A607B681B68002275
S3150802EE101A607B681B6800225A607B681B6800229E
S3150802EE209A607868F5F774FF7B680022C3F8902029
S3150802EE307B680022C3F888207B680022C3F88C20EE
S3150802EE407B680022DA667B6800221A677B680022E2
S3150802EE5083F88420002318460837BD4680BD80B54E
S3150802EE608AB002AFF860B9603B601346FB80FB6864
S3150802EE70D3F88830202B40F08B80BB68002B02D059
S3150802EE80FB88002B01D1012383E0FB681B689B6882
S3150802EE9003F08003802B07D1FB681B689A68FB681E
S3150802EEA01B6822F080029A60FB680022C3F8902051
S3150802EEB0FB682122C3F88820F7F78AFA7861FB688B
S3150802EEC0FA88A3F85420FB68FA88A3F85620FB6848
S3150802EED09B68B3F5805F08D1FB681B69002B04D1D8
S3150802EEE00023FB61BB68BB6103E0BB68FB610023CF
S3150802EEF0BB6130E03B6800937B6900228021F86899
S3150802EF0000F0B2FF0346002B05D0FB682022C3F8A7
S3150802EF10882003233DE0FB69002B0BD1BB691B88C4
S3150802EF201A46FB681B68C2F308029A62BB69023377
S3150802EF30BB6107E0FB691A78FB681B689A62FB6982
S3150802EF400133FB61FB68B3F856309BB2013B9AB2B8
S3150802EF50FB68A3F85620FB68B3F856309BB2002B21
S3150802EF60C8D13B6800937B6900224021F86800F00B
S3150802EF707BFF0346002B05D0FB682022C3F88820B6
S3150802EF80032306E0FB682022C3F88820002300E05A
S3150802EF90022318462037BD4680BD000080B58AB0D8
S3150802EFA000AFF860B9601346FB80FB68D3F88C3073
S3150802EFB0202B4BD1BB68002B02D0FB88002B01D13A
S3150802EFC0012344E0FB680022DA66FB681B689B683B
S3150802EFD003F04003402B07D1FB681B689A68FB685D
S3150802EFE01B6822F040029A60FB681B681A4A934221
S3150802EFF024D0FB681B68194A93421FD0FB681B681A
S3150802F0005B6803F40003002B18D0FB681B687B615E
S3150802F0107B6953E8003F3B613B6943F080637B624F
S3150802F020FB681B681A467B6A3B62FA61F9693A6AA7
S3150802F03041E80023BB61BB69002BE6D1FB881A466F
S3150802F040B968F86800F078FF034600E0022318461C
S3150802F0502837BD4680BD00BF002400440024005462
S3150802F06080B594B000AF78607B681B687B637B6B66
S3150802F07053E8003F3B633B6B23F49073FB647B6866
S3150802F0801B681A46FB6C3B64FA63F96B3A6C41E8F7
S3150802F0900023BB63BB6B002BE6D17B681B68083376
S3150802F0A03B623B6A53E8003FFB61FB6923F08053EE
S3150802F0B023F00103BB647B681B680833BA6CFA62E7
S3150802F0C0BB62B96AFA6A41E800237B627B6A002B53
S3150802F0D0E3D17B68DB6E012B18D17B681B68FB606A
S3150802F0E0FB6853E8003FBB60BB6823F010037B64F0
S3150802F0F07B681B681A467B6CBB617A617969BA6957
S3150802F10041E800233B613B69002BE6D17B681B681B
S3150802F1109B6803F04003402B3AD17B68D3F88030D2
S3150802F120002B17D07B68D3F88030264ADA667B68CC
S3150802F130D3F880301846F7F7E5FA0346002B3CD099
S3150802F1407B68D3F88030DB6E7A68D2F88020104666
S3150802F150984732E07B680022A3F85E207B6800228B
S3150802F1609A657B681B680F221A627B681B689A6914
S3150802F1707B681B6842F008029A617B682022C3F802
S3150802F1808C207B680022DA66786800F0FBFA14E0C5
S3150802F1907B680022A3F85E207B6800229A657B685A
S3150802F1A01B680F221A627B682022C3F88C207B68B0
S3150802F1B00022DA66786800F0E5FA00231846503726
S3150802F1C0BD4680BD7502030880B5AEB000AF786053
S3150802F1D07B681B68DB69C7F8B4307B681B681B68E9
S3150802F1E0C7F8B0307B681B689B68C7F8AC30D7F89D
S3150802F1F0B42040F60F031340C7F8A830D7F8A83052
S3150802F200002B1BD1D7F8B43003F02003002B15D0FE
S3150802F210D7F8B03003F02003002B05D1D7F8AC306D
S3150802F22003F08053002B09D07B685B6F002B00F03C
S3150802F23093827B685B6F786898478DE2D7F8A83027
S3150802F240002B00F0FD80D7F8AC207A4B1340002B38
S3150802F25006D1D7F8B020784B1340002B00F0F08087
S3150802F260D7F8B43003F00103002B11D0D7F8B03029
S3150802F27003F48073002B0BD07B681B6801221A6289
S3150802F2807B68D3F8903043F001027B68C3F890207C
S3150802F290D7F8B43003F00203002B11D0D7F8AC30FC
S3150802F2A003F00103002B0BD07B681B6802221A624B
S3150802F2B07B68D3F8903043F004027B68C3F8902049
S3150802F2C0D7F8B43003F00403002B11D0D7F8AC30CA
S3150802F2D003F00103002B0BD07B681B6804221A6219
S3150802F2E07B68D3F8903043F002027B68C3F890201B
S3150802F2F0D7F8B43003F00803002B17D0D7F8B0308C
S3150802F30003F02003002B05D1D7F8AC20494B134054
S3150802F310002B0BD07B681B6808221A627B68D3F81D
S3150802F320903043F008027B68C3F89020D7F8B430CF
S3150802F33003F40063002B12D0D7F8B03003F08063D1
S3150802F340002B0CD07B681B684FF400621A627B683C
S3150802F350D3F8903043F020027B68C3F890207B688C
S3150802F360D3F89030002B00F0F981D7F8B43003F0C7
S3150802F3702003002B13D0D7F8B03003F02003002B5C
S3150802F38005D1D7F8AC3003F08053002B07D07B6841
S3150802F3905B6F002B03D07B685B6F786898477B6846
S3150802F3A0D3F89030C7F8A4307B681B689B6803F0D3
S3150802F3B04003402B05D0D7F8A43003F02803002BCE
S3150802F3C02ED0786800F0DAFE7B681B689B6803F02B
S3150802F3D04003402B20D17B68D3F88030002B17D00E
S3150802F3E07B68D3F88030154ADA667B68D3F88030B2
S3150802F3F01846F7F787F90346002B19D07B68D3F826
S3150802F4008030DB6E7A68D2F88020104698470FE083
S3150802F4107868F6F75DFF0BE07868F6F759FF07E0BC
S3150802F4207868F6F755FF7B680022C3F8902095E1C5
S3150802F43000BF93E1010000102001000449020308FD
S3150802F4407B68DB6E012B40F02981D7F8B43003F0D4
S3150802F4501003002B00F02281D7F8B03003F0100316
S3150802F460002B00F01B817B681B6810221A627B68DE
S3150802F4701B689B6803F04003402B40F091807B6831
S3150802F480D3F880301B689B6CA7F89230B7F8923095
S3150802F490002B00F065817B68B3F85C30B7F89220E0
S3150802F4A09A4280F05D817B68B7F89220A3F85E20C5
S3150802F4B07B68D3F880301B6D812B60D07B681B6814
S3150802F4C07B677B6F53E8003F3B673B6F23F4807390
S3150802F4D0C7F88C307B681B681A46D7F88C30C7F891
S3150802F4E08030FA67F96FD7F8802041E80023BB67B6
S3150802F4F0BB6F002BE2D17B681B6808333B663B6E09
S3150802F50053E8003FFB65FB6D23F00103C7F888301B
S3150802F5107B681B680833D7F88820FA66BB66B96E1B
S3150802F520FA6E41E800237B667B6E002BE3D17B688B
S3150802F5302022C3F88C207B680022DA667B681B6867
S3150802F540FB64FB6C53E8003FBB64BB6C23F01003FF
S3150802F550C7F884307B681B681A46D7F88430BB65BF
S3150802F5607A65796DBA6D41E800233B653B6D002BE0
S3150802F570E4D17B68D3F880301846F7F747F87B68FA
S3150802F58002221A677B68B3F85C207B68B3F85E30A0
S3150802F5909BB2D31A9BB21946786800F0FDF8DFE0F1
S3150802F5A07B68B3F85C207B68B3F85E309BB2D31AEB
S3150802F5B0A7F8A2307B68B3F85E309BB2002B00F046
S3150802F5C0D180B7F8A230002B00F0CC807B681B688C
S3150802F5D0BB63BB6B53E8003F7B637B6B23F490737F
S3150802F5E0C7F89C307B681B681A46D7F89C307B6440
S3150802F5F03A64396C7A6C41E80023FB63FB6B002B97
S3150802F600E4D17B681B6808337B627B6A53E8003F58
S3150802F6103B623B6A23F0805323F00103C7F8983014
S3150802F6207B681B680833D7F898203A63FB62F96A45
S3150802F6303A6B41E80023BB62BB6A002BE1D17B68C7
S3150802F6402022C3F88C207B680022DA667B680022B7
S3150802F6505A677B681B683B613B6953E8003FFB605E
S3150802F660FB6823F01003C7F894307B681B681A46B8
S3150802F670D7F89430FB61BA61B969FA6941E800239F
S3150802F6807B617B69002BE4D17B6802221A67B7F893
S3150802F690A2301946786800F07FF863E0D7F8B430EC
S3150802F6A003F48013002B0ED0D7F8AC3003F4800392
S3150802F6B0002B08D07B681B684FF480121A627868A0
S3150802F6C001F060FB51E0D7F8B43003F08003002B59
S3150802F6D014D0D7F8B03003F08003002B05D1D7F841
S3150802F6E0AC3003F40003002B08D07B689B6F002B19
S3150802F6F03AD07B689B6F7868984735E0D7F8B4307C
S3150802F70003F04003002B09D0D7F8B03003F04003CA
S3150802F710002B03D0786800F0D2FD26E0D7F8B43083
S3150802F72003F40003002B09D0D7F8B03003F0804366
S3150802F730002B03D0786801F039FB16E0D7F8B4300D
S3150802F74003F08073002B10D0D7F8B030002B0CDAF8
S3150802F750786801F021FB08E000BF06E000BF04E07C
S3150802F76000BF02E000BF00E000BFB837BD4680BD5B
S3150802F77080B483B000AF786000BF0C37BD465DF831
S3150802F780047B704780B483B000AF786000BF0C3743
S3150802F790BD465DF8047B704780B483B000AF7860DD
S3150802F7A00B467B8000BF0C37BD465DF8047B70476D
S3150802F7B080B485B000AF78607B68D3F88830FB6088
S3150802F7C07B68D3F88C30BB60FA68BB68134318466B
S3150802F7D01437BD465DF8047B704780B483B000AF2A
S3150802F7E078607B68D3F8903018460C37BD465DF8CA
S3150802F7F0047B70472DE9B04F94B000AFF86200233E
S3150802F80087F84730FB6A1A68784B9A42FB6A9A6805
S3150802F810FB6A1B691A43FB6A5B691A43FB6ADB6963
S3150802F8201343FB64FB6A1B681B6871491940FB6A30
S3150802F8301A68FB6C0B431360FB6A1B685B6823F44C
S3150802F8404050FB6AD968FB6A1A6840EA01035360AA
S3150802F850FB6A9B69FB64FB6A1A68644B9A4209D085
S3150802F860FB6A1A68634B9A4204D0FB6A1A6AFB6CF3
S3150802F8701343FB64FB6A1B689B6823F06E4121F401
S3150802F8803061FB6A1A68FB6C0B439360FB6A1B6860
S3150802F890DB6A23F00F00FB6A596AFB6A1A6840EAB8
S3150802F8A00103D362FB6A1A68534B9A4202D10123B7
S3150802F8B0BB6466E0FB6A1A68504B9A4202D102237D
S3150802F8C0BB645EE0FB6A1A684D4B9A4202D1042376
S3150802F8D0BB6456E0FB6A1A684A4B9A4202D108236D
S3150802F8E0BB644EE0FB6A1A68474B9A4202D1102360
S3150802F8F0BB6446E0FB6A1A68444B9A4202D120234B
S3150802F900BB643EE0FB6A1A68414B9A4202D1402325
S3150802F910BB6436E0FB6A1A683E4B9A4202D18023E0
S3150802F920BB642EE0FB6A1A683B4B9A4203D14FF43A
S3150802F9308073BB6425E0FB6A1A68384B9A4203D186
S3150802F9404FF40073BB641CE0FB6A1A68344B9A4294
S3150802F95003D14FF48063BB6413E0FB6A1A68314B28
S3150802F9609A4203D14FF40063BB640AE0FB6A1A6841
S3150802F9701E4B9A4203D14FF48053BB6401E0002325
S3150802F980BB64FB6A1A68194B9A4205D0FB6A1A6865
S3150802F990184B9A4240F09480BB6C00223B627A6212
S3150802F9A0D7E90801FBF7DCFE38643B6C002B00F054
S3150802F9B0F780FB6A5B6A1C4A32F813301A463B6CBC
S3150802F9C0B3FBF2F37B63FB6A5A6813465B00134484
S3150802F9D07A6B9A4205D3FB6A5B681B037A6B9A4277
S3150802F9E024D9012387F8473069E000BF0024004480
S3150802F9F0F369FFCF00240054003801400044004058
S3150802FA0000480040004C004000500040006400409E
S3150802FA1000780040007C00400080004000680040FA
S3150802FA20006C004000840040089F03083B6C0022DB
S3150802FA30BB61FA61FB6A5B6A644A32F813309BB2AD
S3150802FA4000223B617A61D7E90423D7E90601F1F777
S3150802FA502BF902460B46104619464FF000024FF0A4
S3150802FA6000030B0243EA10630202F96A496849086D
S3150802FA7000200C46054612EB040843EB0509FB6A0F
S3150802FA805B680022BB60FA60D7E902234046494612
S3150802FA90F1F70AF902460B461346FB63FB6BB3F50D
S3150802FAA0407F08D3FB6BB3F5801F04D2FB6A1B6841
S3150802FAB0FA6BDA6003E0012387F8473070E06FE0FB
S3150802FAC0FB6ADB69B3F5004F3CD1BB6C00223B6095
S3150802FAD07A60D7E90001FBF743FE38643B6C002BDA
S3150802FAE05ED0FB6A5B6A394A32F813301A463B6CB7
S3150802FAF0B3FBF2F35A00FB6A5B685B081A44FB6ABB
S3150802FB005B68B2FBF3F3FB63FB6B0F2B16D9FB6B3C
S3150802FB10B3F5803F12D2FB6B9BB223F00F037B87B0
S3150802FB20FB6B5B089BB203F007039AB27B8F134306
S3150802FB307B87FB6A1B687A8FDA6031E0012387F8D4
S3150802FB4047302DE0BB6C00229A46934650465946EA
S3150802FB50FBF706FE38643B6C002B21D0FB6A5B6A16
S3150802FB601A4A32F813301A463B6CB3FBF2F2FB6AB6
S3150802FB705B685B081A44FB6A5B68B2FBF3F3FB63D8
S3150802FB80FB6B0F2B09D9FB6BB3F5803F05D2FB6BD9
S3150802FB909AB2FB6A1B68DA6002E0012387F84730EB
S3150802FBA0FB6A0122A3F86A20FB6A0122A3F86820ED
S3150802FBB0FB6A00225A67FB6A00229A6797F847305F
S3150802FBC018465037BD46BDE8B08F00BF089F0308E8
S3150802FBD080B483B000AF78607B689B6A03F0080341
S3150802FBE0002B0AD07B681B685B6823F400417B689C
S3150802FBF09A6B7B681B680A435A607B689B6A03F0A8
S3150802FC000103002B0AD07B681B685B6823F400316A
S3150802FC107B68DA6A7B681B680A435A607B689B6A58
S3150802FC2003F00203002B0AD07B681B685B6823F487
S3150802FC3080317B681A6B7B681B680A435A607B684B
S3150802FC409B6A03F00403002B0AD07B681B685B6877
S3150802FC5023F480217B685A6B7B681B680A435A60C7
S3150802FC607B689B6A03F01003002B0AD07B681B682B
S3150802FC709B6823F480517B68DA6B7B681B680A43AE
S3150802FC809A607B689B6A03F02003002B0AD07B6884
S3150802FC901B689B6823F400517B681A6C7B681B6897
S3150802FCA00A439A607B689B6A03F04003002B1AD0CA
S3150802FCB07B681B685B6823F480117B685A6C7B68D7
S3150802FCC01B680A435A607B685B6CB3F5801F0AD1CE
S3150802FCD07B681B685B6823F4C0017B689A6C7B6847
S3150802FCE01B680A435A607B689B6A03F08003002BF1
S3150802FCF00AD07B681B685B6823F400217B68DA6C90
S3150802FD007B681B680A435A6000BF0C37BD465DF81C
S3150802FD10047B704780B598B002AF78607B68002292
S3150802FD20C3F89020F6F754FB78657B681B681B6856
S3150802FD3003F00803082B2FD16FF07E4300937B6DE7
S3150802FD4000224FF40011786800F08EF80346002B63
S3150802FD5022D07B681B68BB63BB6B53E8003F7B639F
S3150802FD607B6B23F080033B657B681B681A463B6DF9
S3150802FD707B643A64396C7A6C41E80023FB63FB6B5B
S3150802FD80002BE6D17B682022C3F888207B680022F4
S3150802FD9083F88420032363E07B681B681B6803F0EF
S3150802FDA00403042B49D16FF07E4300937B6D002236
S3150802FDB04FF48001786800F057F80346002B3CD0D0
S3150802FDC07B681B687B627B6A53E8003F3B623B6A3F
S3150802FDD023F49073FB647B681B681A46FB6C3B63CF
S3150802FDE0FA62F96A3A6B41E80023BB62BB6A002BE6
S3150802FDF0E6D17B681B6808333B613B6953E8003FE1
S3150802FE00FB60FB6823F00103BB647B681B6808334D
S3150802FE10BA6CFA61BB61B969FA6941E800237B6188
S3150802FE207B69002BE5D17B682022C3F88C207B688E
S3150802FE30002283F88420032312E07B682022C3F879
S3150802FE4088207B682022C3F88C207B680022DA6629
S3150802FE507B6800221A677B68002283F884200023C5
S3150802FE6018465837BD4680BD80B584B000AFF860E5
S3150802FE70B9603B601346FB7149E0BB69B3F1FF3FCA
S3150802FE8045D0F6F7A5FA02463B68D31ABA699A42EA
S3150802FE9002D3BB69002B01D1032348E0FB681B6828
S3150802FEA01B6803F00403002B31D0FB681B68DB696F
S3150802FEB003F00803082B10D1FB681B6808221A6294
S3150802FEC0F86800F05BF9FB680822C3F89020FB6823
S3150802FED0002283F88420012329E0FB681B68DB697A
S3150802FEE003F40063B3F5006F11D1FB681B684FF486
S3150802FEF000621A62F86800F041F9FB682022C3F82A
S3150802FF009020FB68002283F8842003230FE0FB6815
S3150802FF101B68DA69BB681340BA689A420CBF0123A8
S3150802FF200023DBB21A46FB799A42A6D0002318466A
S3150802FF301037BD4680BD000080B4A3B000AFF8609C
S3150802FF40B9601346FB80FB68BA689A65FB68FA884B
S3150802FF50A3F85C20FB68FA88A3F85E20FB680022F7
S3150802FF605A67FB689B68B3F5805F0ED1FB681B690D
S3150802FF70002B05D1FB6840F2FF12A3F860202DE0A2
S3150802FF80FB68FF22A3F8602028E0FB689B68002B29
S3150802FF900DD1FB681B69002B04D1FB68FF22A3F86D
S3150802FFA060201BE0FB687F22A3F8602016E0FB684E
S3150802FFB09B68B3F1805F0DD1FB681B69002B04D1E6
S3150802FFC0FB687F22A3F8602008E0FB683F22A3F8BB
S3150802FFD0602003E0FB680022A3F86020FB68002289
S3150802FFE0C3F89020FB682222C3F88C20FB681B68A2
S3150802FFF008337B667B6E53E8003F3B663B6E43F0F5
S315080300000103C7F88430FB681B680833D7F88420D4
S315080300103A67FB66F96E3A6F41E80023BB66BB6E27
S31508030020002BE3D1FB685B6EB3F1005F4FD1FB682E
S31508030030B3F86830FA889A4249D3FB689B68B3F5E4
S31508030040805F07D1FB681B69002B03D1FB68474A0E
S315080300505A6702E0FB68464A5A67FB681B69002B26
S315080300601AD0FB681B683B653B6D53E8003FFB648E
S31508030070FB6C43F48073C7F88030FB681B681A4629
S31508030080D7F88030FB65BA65B96DFA6D41E8002388
S315080300907B657B6D002BE4D1FB681B680833FB6328
S315080300A0FB6B53E8003FBB63BB6B43F08053FB67B3
S315080300B0FB681B680833FA6FBA647B64796CBA6C9D
S315080300C041E800233B643B6C002BE5D146E0FB6823
S315080300D09B68B3F5805F07D1FB681B69002B03D1C7
S315080300E0FB68244A5A6702E0FB68234A5A67FB6897
S315080300F01B69002B19D0FB681B68BB62BB6A53E8F4
S31508030100003F7B627B6A43F490737B67FB681B68DB
S315080301101A467B6F7B633A63396B7A6B41E8002334
S31508030120FB62FB6A002BE6D118E0FB681B687B6160
S315080301307B6953E8003F3B613B6943F02003BB6798
S31508030140FB681B681A46BB6F3B62FA61F9693A6A30
S3150803015041E80023BB61BB69002BE6D1002318469F
S315080301608C37BD465DF8047B704700BF0D0A03084C
S315080301709D060308D90403081503030880B495B03C
S3150803018000AF78607B681B687B637B6B53E8003F33
S315080301903B633B6B23F49073FB647B681B681A46CB
S315080301A0FB6C3B64FA63F96B3A6C41E80023BB6367
S315080301B0BB6B002BE6D17B681B6808333B623B6A43
S315080301C053E8003FFB61FB6923F0805323F00103E7
S315080301D0BB647B681B680833BA6CFA62BB62B96A8C
S315080301E0FA6A41E800237B627B6A002BE3D17B68CA
S315080301F0DB6E012B18D17B681B68FB60FB6853E831
S31508030200003FBB60BB6823F010037B647B681B68F5
S315080302101A467B6CBB617A617969BA6941E800233E
S315080302203B613B69002BE6D17B682022C3F88C200F
S315080302307B680022DA667B6800225A6700BF543758
S31508030240BD465DF8047B704780B584B000AF78601F
S315080302507B68DB6DFB60FB680022A3F85E20FB6806
S315080302600022A3F85620F868F6F732F800BF1037CD
S31508030270BD4680BD80B584B000AF78607B68DB6D12
S31508030280FB60FB680022A3F85E20FB681B680F224D
S315080302901A62FB681B689A69FB681B6842F00802C6
S315080302A09A61FB682022C3F88C20FB680022DA6671
S315080302B0F868FFF767FA00BF1037BD4680BD80B5FB
S315080302C088B000AF78607B681B68FB60FB6853E8FF
S315080302D0003FBB60BB6823F04003FB617B681B6878
S315080302E01A46FB69BB617A617969BA6941E80023F1
S315080302F03B613B69002BE6D17B682022C3F8882043
S315080303007B6800229A677868FFF732FA00BF2037BE
S31508030310BD4680BD80B59CB000AF78607B68B3F8F6
S315080303206030A7F86E307B68D3F88C30222B40F008
S31508030330C3807B681B685B6AA7F86C30B7F86C30B8
S31508030340D9B2B7F86E30DAB27B689B6D0A40D2B27F
S315080303501A707B689B6D5A1C7B689A657B68B3F831
S315080303605E309BB2013B9AB27B68A3F85E207B683A
S31508030370B3F85E309BB2002B40F0A6807B681B68FF
S31508030380FB64FB6C53E8003FBB64BB6C23F49073BC
S31508030390BB667B681B681A46BB6EBB657A65796D57
S315080303A0BA6D41E800233B653B6D002BE6D17B68BC
S315080303B01B680833BB63BB6B53E8003F7B637B6BEC
S315080303C023F001037B667B681B6808337A6E7A64BD
S315080303D03B64396C7A6C41E80023FB63FB6B002BA7
S315080303E0E5D17B682022C3F88C207B6800225A67F4
S315080303F07B6800221A677B681B68354A934224D0B8
S315080304007B681B68334A93421FD07B681B685B680B
S3150803041003F40003002B18D07B681B687B627B6A96
S3150803042053E8003F3B623B6A23F080633B667B6885
S315080304301B681A463B6E3B63FA62F96A3A6B41E8F4
S315080304400023BB62BB6A002BE6D17B68DB6E012BFC
S315080304502ED17B680022DA667B681B683B613B69A1
S3150803046053E8003FFB60FB6823F01003FB657B68DA
S315080304701B681A46FB6DFB61BA61B969FA6941E8FB
S3150803048000237B617B69002BE6D17B681B68DB69EC
S3150803049003F01003102B03D17B681B6810221A6222
S315080304A07B68B3F85C3019467868FFF775F90BE093
S315080304B07868F5F7EDFE07E07B681B689A697B6841
S315080304C01B6842F008029A6100BF7037BD4680BDBB
S315080304D0002400440024005480B59CB000AF786023
S315080304E07B68B3F86030A7F86E307B68D3F88C3036
S315080304F0222B40F0C3807B681B685B6AA7F86C30C5
S315080305007B689B6DBB66B7F86C20B7F86E301340F3
S315080305109AB2BB6E1A807B689B6D9A1C7B689A6538
S315080305207B68B3F85E309BB2013B9AB27B68A3F84B
S315080305305E207B68B3F85E309BB2002B40F0A68042
S315080305407B681B68BB64BB6C53E8003F7B647B6CAE
S3150803055023F490737B667B681B681A467B6E7B6500
S315080305603A65396D7A6D41E80023FB64FB6C002B11
S31508030570E6D17B681B6808337B637B6B53E8003FD4
S315080305803B633B6B23F001033B667B681B680833BD
S315080305903A6E3A64FB63F96B3A6C41E80023BB6332
S315080305A0BB6B002BE5D17B682022C3F88C207B68C4
S315080305B000225A677B6800221A677B681B68354ADC
S315080305C0934224D07B681B68334A93421FD07B68C7
S315080305D01B685B6803F40003002B18D07B681B6851
S315080305E03B623B6A53E8003FFB61FB6923F0806388
S315080305F0FB657B681B681A46FB6DFB62BA62B96AC0
S31508030600FA6A41E800237B627B6A002BE6D17B68A2
S31508030610DB6E012B2ED17B680022DA667B681B68AA
S31508030620FB60FB6853E8003FBB60BB6823F010031D
S31508030630BB657B681B681A46BB6DBB617A617969C2
S31508030640BA6941E800233B613B69002BE6D17B6825
S315080306501B68DB6903F01003102B03D17B681B6847
S3150803066010221A627B68B3F85C3019467868FFF77C
S3150803067093F80BE07868F5F70BFE07E07B681B68D1
S315080306809A697B681B6842F008029A6100BF703753
S31508030690BD4680BD002400440024005480B5ACB098
S315080306A000AF78607B68B3F86030A7F8AA307B6838
S315080306B01B68DB69C7F8AC307B681B681B68C7F81F
S315080306C0A4307B681B689B68C7F8A0307B68D3F89F
S315080306D08C30222B40F087817B68B3F86830A7F803
S315080306E09E302AE17B681B685B6AA7F89C30B7F8DB
S315080306F09C30D9B2B7F8AA30DAB27B689B6D0A4048
S31508030700D2B21A707B689B6D5A1C7B689A657B68A4
S31508030710B3F85E309BB2013B9AB27B68A3F85E20BE
S315080307207B681B68DB69C7F8AC30D7F8AC3003F0D5
S315080307300703002B53D0D7F8AC3003F00103002B83
S3150803074011D0D7F8A43003F48073002B0BD07B6841
S315080307501B6801221A627B68D3F8903043F00102C2
S315080307607B68C3F89020D7F8AC3003F00203002B5C
S3150803077011D0D7F8A03003F00103002B0BD07B6808
S315080307801B6802221A627B68D3F8903043F004028E
S315080307907B68C3F89020D7F8AC3003F00403002B2A
S315080307A011D0D7F8A03003F00103002B0BD07B68D8
S315080307B01B6804221A627B68D3F8903043F002025E
S315080307C07B68C3F890207B68D3F89030002B06D05B
S315080307D07868F5F77DFD7B680022C3F890207B686F
S315080307E0B3F85E309BB2002B40F0A7807B681B688A
S315080307F03B673B6F53E8003FFB66FB6E23F480734E
S31508030800C7F898307B681B681A46D7F89830FB6791
S31508030810BA67B96FFA6F41E800237B677B6F002BD2
S31508030820E4D17B681B680833FB65FB6D53E8003F1F
S31508030830BB65BB6D23F0805323F00103C7F89430DF
S315080308407B681B680833D7F89420BA667B66796E8B
S31508030850BA6E41E800233B663B6E002BE1D17B6809
S315080308602022C3F88C207B6800225A677B68002203
S315080308701A677B681B68624A934226D07B681B68A3
S31508030880604A934221D07B681B685B6803F40003C4
S31508030890002B1AD07B681B68BB64BB6C53E8003F0C
S315080308A07B647B6C23F08063C7F890307B681B6896
S315080308B01A46D7F890307B653A65396D7A6D41E803
S315080308C00023FB64FB6C002BE4D17B68DB6E012BF6
S315080308D030D17B680022DA667B681B687B637B6B97
S315080308E053E8003F3B633B6B23F01003C7F88C3098
S315080308F07B681B681A46D7F88C303B64FA63F96B36
S315080309003A6C41E80023BB63BB6B002BE4D17B68DD
S315080309101B68DB6903F01003102B03D17B681B6884
S3150803092010221A627B68B3F85C3019467868FEF7BA
S3150803093033FF02E07868F5F7ABFCB7F89E30002B77
S3150803094006D0D7F8AC3003F02003002B7FF4CAAEE9
S315080309507B68B3F85E30A7F88A30B7F88A30002B7D
S3150803096049D07B68B3F86830B7F88A209A4242D2EE
S315080309707B681B6808333B623B6A53E8003FFB61AD
S31508030980FB6923F08053C7F884307B681B680833F8
S31508030990D7F88420FA62BB62B96AFA6A41E8002387
S315080309A07B627B6A002BE3D17B68174A5A677B68AD
S315080309B01B68FB60FB6853E8003FBB60BB6843F0FA
S315080309C02003C7F880307B681B681A46D7F880303F
S315080309D0BB617A617969BA6941E800233B613B697E
